:100000000C9499020C94C4020C94C4020C94C40283
:100010000C94A0080C94C4020C94C4020C94C40266
:100020000C94C4020C94D32E0C94C4020C94C402FD
:100030000C94C4020C9443570C94C4020C94C40254
:100040000C94C4020C94C4020C94BB5F0C94C402C4
:100050000C9476610C940C620C94C4020C94C4024F
:100060000C94C4020C94C4020C94F55D0C94C4026C
:100070000C94AF610C9459620C94C4020C94C402A9
:100080000C94C4020C94C4020C94C4022D33002DB1
:1000900032002D31002030002B31002B32002B3369
:1000A000002B340020430020432300204400204440
:1000B0002300204500204600204623002047002042
:1000C000472300204100204123002042004D53548B
:1000D000004D494400434C4B00322F3100312F3149
:1000E00000312F3200312F3400312F3800312F31C1
:1000F0003600312F34380053494E005452490053D2
:1001000041570053515500532F4800445732004483
:100110005733004457340044573500445736005491
:100120005731005457320054573300545734004568
:10013000585000485244005346540046555A005304
:10014000504B0053545000313025003235250035D6
:1001500030250037352500393025004348524F4DB2
:100160004154494320004D414A4F52202020202035
:10017000006D696E6F7220202020200050454E5483
:1001800041544F4E494300444F5249414E20202094
:100190002000504852594749414E2020004C5944B4
:1001A00049414E20202020004D49584F4C59444988
:1001B000414E004C4F435249414E20202000464FB3
:1001C00052574152442020004241434B5741524430
:1001D000200050494E472D504F4E470052414E444B
:1001E0004F4D2020200053594E0042504D00545294
:1001F00058004356525800434C4B004E4300505455
:1002000052004C454E0053434C0054524947004C59
:10021000464F005741560046525100414D50005341
:100220005450004E5445004F4354004C454E470037
:1002300055544D0050524F00525452470050554CA7
:100240000042415200E601EA013D02F701F701FBDD
:1002500001FB01FB01FE01020206020A020F02136A
:100260000217021B024102230227022B020602FB95
:1002700001FB01FB0141023002340238024102302D
:100280000234022B024102020206020A02BE01C827
:1002900001D201DC015B01660171017C01870192E1
:1002A000019D01A801B30147014B014F01530157C3
:1002B00001F700FB00FF00030107010B010F011311
:1002C0000117011B011F01230127012B012F0133FE
:1002D0000137013B013F014301D900DD00E100E5A9
:1002E00000E900ED00F200CD00D100D5008C008FB8
:1002F000009200950098009B009E00A100A400A71A
:1003000000AB00AE00B200B500B800BC00BF00C337
:1003100000C600CA0020202020002E2E2E2E2E2EB9
:100320002E2E2E2E2E2E2E2E2E2E004441437320A6
:1003300063616C6962726174696F6E0020696E69D5
:100340007469616C697A6174696F6E200020202085
:100350002020454550524F4D2020202020002B00CA
:100360002D00546F74616C204163632076616C755D
:100370006520005B5341564544215D0045585400BB
:10038000202020202020202020202020202020206D
:1003900000202020200020202020002020202000DD
:1003A00020202020004F6E004F6666004F6E004FE9
:1003B00066660020204C464F73202043562F47612D
:1003C000746520006261722075746D2070726F20F8
:1003D00072747267006261722075746D2070726F42
:1003E000206C656E67006C666F20776176206672A0
:1003F0007120616D702000435620547261636B2040
:100400005363616C653A2000626172206E746520EE
:100410006F6374206C656E670020202000312F0010
:1004200046494C4C00626172206C656E2073636CAF
:10043000207472696700455854002020506174741C
:1004400065726E20506C617920200020202042616E
:1004500072202020205374657020200073796E2054
:1004600062706D2070756C20636C6B20002054727C
:10047000636B20646972656374696F6E200020503D
:1004800074726E20646972656374696F6E20002BEC
:10049000002D00202053687566666C652076616CBF
:1004A0007565200076312E303335000000210024A0
:1004B0000027002A0000002200250028002B000051
:1004C000002000230026002900020202020202028C
:1004D00002040404040404040403030303030303E5
:1004E0000301010101010101010102040810204082
:1004F00080010204081020408001020408102040FE
:100500008001020408102040800000000102000861
:1005100009000000000403070600000000000000BE
:1005200000000000000000000000242A8D5CD4635D
:100530001D2A11241FBECFEFD0E4DEBFCDBF16E0D1
:10054000A0E0B1E0E2E0F8ED00E00BBF02C00790F0
:100550000D92A83FB107D9F71BBE13E3A8EFB6E091
:1005600001C01D92AD3CB107E1F715E0C0E3D5E055
:1005700004C02297FE010E94B96BCA32D107C9F7A5
:100580000E946A640C94F46B0C940000CF93DF9388
:10059000BC018230910510F462E070E0A091CB3391
:1005A000B091CC33ED01E0E0F0E040E050E021C05C
:1005B000888199818617970769F48A819B81309792
:1005C00019F09383828304C09093CC338093CB3310
:1005D000FE0134C06817790738F44115510519F048
:1005E0008417950708F4AC01FE018A819B819C0168
:1005F000E9012097E9F641155105A9F1CA01861BC9
:10060000970B049708F4BA01E0E0F0E02AC08D915E
:100610009C91119784179507F9F46417750781F475
:1006200012968D919C911397309719F09383828342
:1006300004C09093CC338093CB33FD0132964CC0F1
:10064000CA01861B970BFD01E80FF91F6193719397
:1006500002978D939C9340C0FD01828193819C0100
:10066000D9011097A1F68091C9339091CA33892B93
:1006700041F480912101909122019093CA3380939B
:10068000C93340912301509124014115510541F492
:100690004DB75EB780911F0190912001481B590B07
:1006A0002091C9333091CA33CA01821B930B86173C
:1006B000970780F0AB014E5F5F4F8417950750F0AE
:1006C000420F531F5093CA334093C933F9016193CA
:1006D000719302C0E0E0F0E0CF01DF91CF91089587
:1006E000CF93DF93009709F450C0EC0122971B824F
:1006F0001A82A091CB33B091CC33109709F140E02E
:1007000050E0AC17BD0708F1BB83AA83FE0121911D
:100710003191E20FF31FAE17BF0779F48D919C91D1
:100720001197280F391F2E5F3F4F39832883129668
:100730008D919C9113979B838A834115510571F488
:10074000D093CC33C093CB3320C012968D919C9123
:100750001397AD01009711F0DC01D3CFFA01D383D9
:10076000C28321913191E20FF31FCE17DF0769F4A5
:1007700088819981280F391F2E5F3F4FFA013183FD
:1007800020838A819B8193838283DF91CF91089517
:10079000A0E0B0E0EEECF3E00C94C56BEC01A880B7
:1007A000B980CA80DB80A114B104C104D10441F432
:1007B00084E2A82E89EDB82E8BE5C82E87E0D82ECE
:1007C000C601B5012DE133EF41E050E00E949C6B82
:1007D00027EA31E440E050E00E94286B7B018C0165
:1007E000C601B5012DE133EF41E050E00E949C6B62
:1007F000CA01B9012CEE34EF4FEF5FEF0E94286B76
:100800006E0D7F1D801F911F97FF04C061507040C7
:1008100080409048688379838A839B839B01AC01E5
:100820005F77B901CA01CDB7DEB7EAE00C94E16B9E
:100830000E94C803089585E291E00E94C8030895CC
:1008400060932501709326018093270190932801DE
:100850000895A0E0B0E0EFE2F4E00C94BF6B6C010F
:10086000009729F4CB010E94C6026C01C1C08EEF33
:10087000882E8FEF982E8C0C9D1C8601060F171F5B
:100880000815190508F4B2C0F401A081B181A617BA
:10089000B707B8F0A530B10508F4AAC0CD01049798
:1008A0008617970708F4A4C01297A61BB70BF80188
:1008B000A193B193D4016D937C93CF010E947003F7
:1008C00097C07B01EA1AFB0AEEEFFFEFEE0EFF1E68
:1008D00036016A0E7B1EC091CB33D091CC334424B9
:1008E0005524AA24BB244AC0C615D705E1F5488182
:1008F00059814E155F05B8F1CA0104978E159F0501
:10090000B0F41296A40FB51FF401B183A0832A811D
:100910003B814114510431F0D20113963C932E9344
:10092000129766C03093CC332093CB3361C08A8159
:100930009B81F80193838283425050404E195F0996
:10094000518340834114510431F0D20113961C931A
:100950000E93129704C01093CC330093CB33F40161
:100960007183608345C088819981A816B90608F40F
:100970005C012E018A819B819C01E901209709F08D
:10098000B3CF8091C9339091CA3386159705E9F4A6
:10099000A616B706D0F42091230130912401211529
:1009A000310541F42DB73EB780911F019091200190
:1009B000281B390B02171307C8F41093CA3300938E
:1009C000C933D4016D937C9313C0CB010E94C6023E
:1009D000EC01009759F0F40140815181B6010E9469
:1009E0000505C6010E9470036E0102C0CC24DD24FF
:1009F000C601CDB7DEB7E0E10C94DB6BFB01DC0197
:100A000005900D920020E1F70895FB01DC0102C082
:100A100001900D9241505040D8F70895FB01DC0140
:100A20008D91019080190110D9F3990B0895FB0164
:100A3000DC0101900D920020E1F70895FB019F0178
:100A4000E8944230C4F04532B4F44A3029F497FBBC
:100A50001EF4909581959F4F642F77270E94536BCA
:100A6000805D8A330CF0895D8193CB010097A1F7FB
:100A700016F45DE251931082C9010C945505FB01F7
:100A80009F01423074F0453264F4642F77270E944E
:100A9000536B805D8A330CF0895D8193CB010097A5
:100AA000A1F71082C9010C945505DC01FC01672FE8
:100AB00071917723E1F7329704C07C916D93708335
:100AC0006291AE17BF07C8F30895FC011482138228
:100AD00090E0672B09F091E090838181981779F07D
:100AE0008281882319F4913009F4938392819130A3
:100AF00021F48081882309F494838081828380811A
:100B000081830895AF92BF92CF92DF92EF92FF92CE
:100B10000F931F93482F9091F90680E02091F806DB
:100B200030E0282B392B442321F0413009F056C006
:100B300056C04091C22F5091C32FEBE0F7E060E028
:100B400070E081E0E82EF12C012D112D1382C901F6
:100B5000062E02C0969587950A94E2F7982F917019
:100B600090838181981761F18281882349F59130C2
:100B700039F5938386818F5F8683813019F08230C7
:100B8000F9F40DC057016801062E04C0AA0CBB1C65
:100B9000CC1CDD1C0A94D2F74A295B2911C01682AD
:100BA00057016801062E04C0AA0CBB1CCC1CDD1C1E
:100BB0000A94D2F7D601C501809590954823592310
:100BC000808181836F5F7F4F37966031710509F0B7
:100BD000BDCF4093C22F5093C32F02C002C0A901C2
:100BE000CA011F910F91FF90EF90DF90CF90BF90BF
:100BF000AF9008952F923F924F925F927F928F9283
:100C00009F92AF92BF92CF92DF92EF92FF920F939B
:100C10001F93CF93DF931C017090A309472D50E0E1
:100C2000FA01EC54F14D80808294A0EF8A22209149
:100C30009E2E30E09090A80ACBE0D7E060E070E014
:100C40008A01000F111FCA01E6E0880F991FEA957B
:100C5000E1F7080F191F83E994E0FC012E9FC00102
:100C60002F9F900D3E9F900D1124080F191F82EAAF
:100C7000A82E8EE2B82EA40EB51E86E299E0289F1B
:100C80006001299FD00C389FD00C11247A01EC0C04
:100C9000FD1C82EB9AE0E80EF91E882D860F482E87
:100CA0005524F801E40DF51DEE0FFF1FEB53F54F32
:100CB0008081482F4170282F26952170C101062E72
:100CC00002C0969587950A94E2F7382F31703883E1
:100CD0008981381709F46DC0942F8A81882309F01F
:100CE00059C0313009F056C0F5013083442309F46E
:100CF00048C0222329F4F7018081882309F046C0E7
:100D00001E82F0E17F16D9F0F801E60FF71FEE0F13
:100D1000FF1FDF01AB53B54F8C9183708C931196FD
:100D20008C911197887F846011968C93EA53F54FCC
:100D3000808187708083F501308390E02BC0FB01B8
:100D4000EE0FFF1FE60FF71FEC0DFD1DDF01A05F8B
:100D5000BC4E8C918E7F8C93EF5EFC4E80818770B1
:100D600080839C9111968C911197887F8460119655
:100D70008C931197917098619C9390E0992493942F
:100D800009C0F7018081882319F491E021E002C0B5
:100D900091E020E0F801E40DF51DEE0FFF1FEB538D
:100DA000F54F80818C7F220F892B822B8083888155
:100DB00089836F5F7F4F27966031710509F06DCF92
:100DC0009092A80ADF91CF911F910F91FF90EF9021
:100DD000DF90CF90BF90AF909F908F907F905F906B
:100DE0004F903F902F9008957F928F929F92AF9255
:100DF000BF92CF92DF92EF92FF920F931F93CF9308
:100E0000DF934C01C090A3094C2D50E020919E2E01
:100E100030E0FA01EC54F14DD080D294B0EFDB22F7
:100E2000E091A80ACBE0D7E060E070E086E299E0CC
:100E3000289F7001299FF00C389FF00C1124772413
:100E400073948A01000F111FCA01F6E0880F991FE1
:100E5000FA95E1F7080F191F83E994E0DC012A9F56
:100E6000C0012B9F900D3A9F900D1124080F191F60
:100E7000B2EAAB2EBEE2BB2EA40EB51EC401062EF6
:100E800002C0969587950A94E2F7482F41704883EF
:100E90008981481709F464C08A81882309F05FC0FA
:100EA000413009F05CC08D2D860F282F30E090E096
:100EB000F901EE0FFF1FE20FF31FEE0DFF1DE05FC4
:100EC000FC4E808180FF91E0F901EE0FFF1FE20FE1
:100ED000F31FEE0DFF1DE05FFC4E80818E7F892B9E
:100EE00080839923D9F5B0E1CB16D1F0F801E60F54
:100EF000F71FEE0FFF1FDF01AB53B54F8C918370CF
:100F00008C9311968C911197887F846011968C93A5
:100F1000EA53F54F808187708083F50170821EC08F
:100F2000FB01EE0FFF1FE60FF71FEE0DFF1DDF01A8
:100F3000A05FBC4E8C918E7F8C93EF5EFC4E8081C7
:100F4000877080839C9111968C911197887F846023
:100F500011968C931197917098619C93E1E049836D
:100F60006F5F7F4F27966031710509F087CFE0935F
:100F7000A80ADF91CF911F910F91FF90EF90DF9022
:100F8000CF90BF90AF909F908F907F900895BF9229
:100F9000CF92DF92EF92FF920F931F93CF93DF9345
:100FA000EC01B0909C08C0902B025091DD2ED090A7
:100FB000E5092091DB2E3091DC2EEBE7F7E060E0D5
:100FC00070E011E0E12EF12C012D112D462F13823E
:100FD000CE01062E02C0969587950A94E2F7982FC7
:100FE000917090838181981709F452C0828188237F
:100FF00009F04EC0913009F04BC09383BB2029F11A
:10100000552381F0C901062E02C0969587950A9452
:10101000E2F780FD23C0CC24C39450E0DD2420E01F
:1010200030E036C0D801C701062E04C0880F991FD2
:10103000AA1FBB1F0A94D2F79C0120953095CC249F
:10104000C39451E0DD24D39423C0C901062E02C00D
:10105000969587950A94E2F780FF0EC0D801C701E4
:1010600004C0880F991FAA1FBB1F4A95D2F780950D
:101070009095282339230CC0D801C701062E04C03F
:10108000880F991FAA1FBB1F0A94D2F7282B392B50
:10109000808181836F5F7F4F37966031710509F0E2
:1010A00095CFC0922B025093DD2ED092E50930935C
:1010B000DC2E2093DB2EDF91CF911F910F91FF90BB
:1010C000EF90DF90CF90BF90089581E00E9482055D
:1010D000AC019093C12F8093C02F20E030E0CA0173
:1010E000022E02C0969587950A94E2F780FF02C00F
:1010F000822F08952F5F3F4F2031310581F70895EA
:1011000081E00E948205AC019093BF2F8093BE2F97
:1011100060E020E030E0CA01022E02C0969587957B
:101120000A94E2F780FF05C0613011F4822F089520
:1011300061E02F5F3F4F2031310569F780E008956E
:101140001F920F920FB60F920BB60F921124EF92CF
:10115000FF920F931F932F933F934F935F938F9320
:101160009F93AF93BF93EF93FF9380B18170809370
:10117000862F9091862F8091872F9817B9F18091B3
:10118000862F882379F581E08093882F10923C097F
:10119000EEE5FFE281930FE2EF36F007D9F72C9AE4
:1011A0002C981092380910924E0110924D0180E057
:1011B00090E021E0FC01E25BF64F1082FC01E65377
:1011C000F64F1082FC01E955F64F2083FC01E059EF
:1011D000F64F1082FC01EF57F64F208301968131C4
:1011E000910541F78091862F8093872F809129095F
:1011F000823009F084C080B190E095958795817028
:1012000080937B2F90917B2F80917C2F981709F4EE
:1012100040C080917C2F882311F02C9A01C02C981B
:1012200090917B2F913091F580919D09882321F435
:1012300090937E2F9093350220916F2F3091702FD5
:101240004091712F5091722F8091772F9091782F2C
:10125000A091792FB0917A2F79018A01E81AF90AC1
:101260000A0B1B0BE0923102F09232020093330220
:101270001093340281E080937D2F2093772F309359
:10128000782F4093792F50937A2F03C081E0809379
:10129000802F80917B2F80937C2F809131029091C1
:1012A0003202A0913302B0913402885B9B40A0408F
:1012B000B04060F088EB9BE0A0E0B0E080933102AA
:1012C00090933202A0933302B093340280913102A2
:1012D00090913202A0913302B09134028D5291402C
:1012E000A040B04060F48CE291E0A0E0B0E08093D8
:1012F000310290933202A0933302B0933402FF91F3
:10130000EF91BF91AF919F918F915F914F913F91DD
:101310002F911F910F91FF90EF900F900BBE0F90A8
:101320000FBE0F901F901895E82F592F4091102F46
:101330003091112F2091C42F222381F0213051F4BC
:101340008DB38093C62F9DB38091C52F809589233F
:101350008DBB04C08FB7F8948093C62F4CBD3DBDA4
:101360005D985EBD00000DB407FEFDCF8EB5EEBDED
:1013700000000DB407FEFDCF8EB57EBD00000DB49C
:1013800007FEFDCF8EB56EBD00000DB407FEFDCF8C
:101390008EB55D9A222339F08091C62F213011F449
:1013A0008DBB08958FBF0895682F592F4091102F3E
:1013B0003091112F2091C42F222381F0213051F43C
:1013C0008DB38093C62F9DB38091C52F80958923BF
:1013D0008DBB04C08FB7F8948093C62F4CBD3DBD24
:1013E0005C985EBD00000DB407FEFDCF8EB56EBDEE
:1013F00000000DB407FEFDCF8EB55C9A222339F0B4
:101400008091C62F213011F48DBB08958FBF0895B0
:101410004091102F3091112F2091C42F222381F061
:10142000213051F48DB38093C62F9DB38091C52F89
:10143000809589238DBB04C08FB7F8948093C62F05
:101440004CBD3DBD5C981EBC00000DB407FEFDCF39
:101450008EB51EBC00000DB407FEFDCF8EB55C9AA4
:10146000222339F08091C62F213011F48DBB0895CD
:101470008FBF08959C013F7030616091102F509193
:10148000112F4091C42F442381F0413051F48DB38A
:101490008093C62F9DB38091C52F809589238DBBE6
:1014A00004C08FB7F8948093C62F6CBD5DBD1298B1
:1014B0003EBD00000DB407FEFDCF8EB52EBD000071
:1014C0000DB407FEFDCF8EB5129A442339F08091FA
:1014D000C62F413011F48DBB08958FBF08959C0134
:1014E0003F7030616091102F5091112F4091C42FA7
:1014F000442381F0413051F48DB38093C62F9DB3C6
:101500008091C52F809589238DBB04C08FB7F89437
:101510008093C62F6CBD5DBD13983EBD00000DB419
:1015200007FEFDCF8EB52EBD00000DB407FEFDCF2A
:101530008EB5139A442339F08091C62F413011F4AF
:101540008DBB08958FBF08959C013F7030696091F5
:10155000102F5091112F4091C42F442381F041301E
:1015600051F48DB38093C62F9DB38091C52F809584
:1015700089238DBB04C08FB7F8948093C62F6CBDB0
:101580005DBD13983EBD00000DB407FEFDCF8EB5C6
:101590002EBD00000DB407FEFDCF8EB5139A442377
:1015A00039F08091C62F413011F48DBB08958FBF63
:1015B00008954091102F3091112F2091C42F222394
:1015C00081F0213051F48DB38093C62F9DB380916B
:1015D000C52F809589238DBB04C08FB7F894809365
:1015E000C62F4CBD3DBD5E9A1EBC00000DB407FE6B
:1015F000FDCF8EB51EBC00000DB407FEFDCF8EB52D
:101600001EBC00000DB407FEFDCF8EB51EBC000051
:101610000DB407FEFDCF8EB51EBC00000DB407FE55
:10162000FDCF8EB580935C2F80935D2F5E98222333
:1016300039F08091C62F213011F48DBB08958FBFF2
:1016400008959C0143B148704093122F93B1947058
:101650009093132F442311F58091142F8823F1F0D8
:10166000992319F0260F371F19C08091A3088823EA
:1016700081F080911D2F813041F0813010F0823057
:1016800069F42A30310554F007C02031310534F0B7
:1016900003C02115310511F0261B370B4093142F81
:1016A000C9010895482F53B152705093182F93B128
:1016B00091709093192F5523D9F480911A2F882374
:1016C000B9F0992369F08FEF90E0841B9109262FE0
:1016D00030E08217930714F44FEF0AC0460F08C09A
:1016E000461720F4442321F0462F02C04111461B27
:1016F00050931A2F842F90E00895CF92DF92EF92AB
:10170000FF920F931F93CF93DF93EC01F42EE22E01
:10171000680118811093AD2F812F0E94520B88838E
:10172000F81608F0F88288818E1508F0E882888122
:10173000811739F08093AD2F81E0F601808380938B
:101740002B02DF91CF911F910F91FF90EF90DF90CF
:10175000CF9008959F92AF92BF92CF92DF92EF9277
:10176000FF920F931F937B018C0159016A0193B083
:1017700082E098229092182F93B191709093192F34
:101780009920D9F580911A2F8823B9F1992329F04E
:10179000C801B7010E9413692EC08091A308882355
:1017A000D1F080911D2F813059F0813010F08230BE
:1017B00021F5C801B70120E030E040E251E406C065
:1017C000C801B70120E030E040E851E40E94C16A5E
:1017D00088239CF00AC0C801B70120E030E040E057
:1017E00050E00E947769882341F0C801B701A60143
:1017F00095010E9412697B018C0190921A2FB7010A
:10180000C8011F910F91FF90EF90DF90CF90BF9094
:10181000AF909F90089523B122702093182F93B119
:1018200091709093192F1092AC2F1092AB2F22230E
:1018300079F480911A2F882359F0992319F081E0C7
:1018400090E002C08FEF9FEF9093AC2F8093AB2F6F
:1018500020931A2F8091AB2F9091AC2F0895EF9287
:10186000FF920F931F93CF93DF93582F20919E2EBB
:10187000803109F04DC030E0A0E0B0E086E299E0B0
:10188000289F7001299FF00C389FF00C1124062F1F
:1018900010E0C42FD0E0742F7295770F770F707C13
:1018A000469546954770562F5295550F550F507CCB
:1018B000669566956770FD01EE0FFF1FEA0FFB1F2F
:1018C000EE0DFF1DE05FFC4E2081922F92959695C4
:1018D000969593703181832F8770880F880F892B9D
:1018E00090E08017910734F42F73252B2083387FE5
:1018F000362B08C08C179D0734F02F73272B2083BD
:10190000387F342B31831196A034B105A1F686C0FF
:1019100030E0A0E0B0E083E994E0289FE001299F57
:10192000D00D389FD00D1124062F10E0242F30E069
:10193000F42EF294FF0CFF0C80ECF82246954695AD
:101940004770762F7295770F770F707C6695669546
:101950006770852F90E0FC01689415F8EE0FFF1F6B
:101960001694E1F7880F991FE80FF91FEC0FFD1F80
:10197000EA0FFB1FEE0FFF1FEB53F54F908192957F
:1019800096959695937081818770880F880F892B23
:1019900090E080179107ECF4852F90E0FC016894AB
:1019A00015F8EE0FFF1F1694E1F7880F991FE80F47
:1019B000F91FEC0FFD1FEA0FFB1FEE0FFF1FEB538C
:1019C000F54F80818F73872B80838181887F862B61
:1019D0001FC082179307ECF0852F90E0FC016894FC
:1019E00015F8EE0FFF1F1694E1F7880F991FE80F07
:1019F000F91FEC0FFD1FEA0FFB1FEE0FFF1FEB534C
:101A0000F54F80818F738F2980838181887F842B1C
:101A100081831196A034B10509F09BCFDF91CF915E
:101A20001F910F91FF90EF9008952F923F924F9248
:101A30005F926F927F928F929F92AF92BF92CF925E
:101A4000DF92EF92FF920F931F93DF93CF93CDB767
:101A5000DEB760970FB6F894DEBF0FBECDBF8091A2
:101A6000E308882351F0809109028F5F8093090277
:101A7000883018F087E0809309028091DC08882381
:101A800049F080910902815080930902883010F05A
:101A900010920902DE011196E7EBF6E080E1019079
:101AA0000D928150E1F780919E2E482F50E086E202
:101AB00099E0489FF001499FF00D589FF00D1124C7
:101AC000E65FFC4EE081E33018F4E13048F405C0F5
:101AD000E33049F0E93048F403C0ACE0AA2E05C079
:101AE000F7E0AF2E02C0E5E0AE2E80919D0988237D
:101AF00009F444C08091A209813009F03FC080916F
:101B0000A70A8823D9F180916F0990E0FC01EE0FBC
:101B1000FF1FE80FF91F86E299E0489F9001499F57
:101B2000300D589F300D1124E20FF31FEE5EFC4E76
:101B30009091AA2F9F708081807F892B80838091D4
:101B40006F0990E0FC01EE0FFF1FE80FF91FE20F95
:101B5000F31FE05FFC4E8081817C806380838091F5
:101B60006F0990E0FC01EE0FFF1FE80FF91FE20F75
:101B7000F31FE05FFC4E808181608083B090AA2FCC
:101B80000BEE17E0EE24FF242E010894411C511C9B
:101B90008A2C992446E2642E49E0742E332433942F
:101BA00037E0232EF80113828091010990910209F8
:101BB0000E2C02C0969587950A94E2F7982F9170A3
:101BC00090838181981709F4CBC08281882309F022
:101BD000C4C0913009F0C1C09383F201EE0DFF1D26
:101BE000E0818E2F90E06A2D70E00E94536B9B0184
:101BF00080910902860F80930A02883010F02092AB
:101C00000A02289DC001299D900D389D900D112438
:101C10002E2F281B80919E2E90E0869DF001879D9F
:101C2000F00D969DF00D1124E65FFC4E808183300F
:101C300018F4813058F405C0833069F0893080F49D
:101C400005C0E22FF0E0E356FE4F09C0E22FF0E0BE
:101C5000EF56FE4F04C0E22FF0E0E856FE4FB08092
:101C600090E0FC01EE0FFF1FE80FF91FEE0FFF1FC2
:101C7000EE0FFF1FEB0DF11DE356FE4FE081F0E08C
:101C8000EE0FFF1FE958FE4F80910A02D82EDD0C9F
:101C9000CC24808191818C0D9D1D0E943A0A5F9A0F
:101CA0003092A70A80919D09882309F456C080913B
:101CB000A209813009F051C020919E2E30E0809120
:101CC0006F0990E0FC01EE0FFF1FE80FF91FA9015B
:101CD000469D9001479D300D569D300D1124E20F19
:101CE000F31FEE5EFC4E9B2D9F708081807F892BC1
:101CF000808380916F0990E0FC01EE0FFF1FE80FD9
:101D0000F91FE20FF31FEE5EFC4E90910A029770EE
:101D10009295907F80818F78892B808380916F0945
:101D200090E0FC01EE0FFF1FE80FF91FE20FF31F19
:101D3000E05FFC4E8081817C8861808380916F09A7
:101D400090E0FC01EE0FFF1FE80FF91FE20FF31FF9
:101D5000E05FFC4E808181608083F8018081818317
:101D60000894E11CF11C095F1F4FF0E1EF16F1042C
:101D700009F018CFB092AA2F809101099091020921
:101D8000892B21F58091A70A882301F15F98109291
:101D9000A70A80916F0990E020919E2E30E0FC010F
:101DA000EE0FFF1FE80FF91F86E299E0AC01249FB8
:101DB000C001259F900D349F900D1124E80FF91F4D
:101DC000E05FFC4E8081817C8861808360960FB6E5
:101DD000F894DEBF0FBECDBFCF91DF911F910F9161
:101DE000FF90EF90DF90CF90BF90AF909F908F903B
:101DF0007F906F905F904F903F902F900895EF925B
:101E0000FF920F931F9300EE1EE27801E80EF11C83
:101E100060912E0970912F0980E090E00E940F6A76
:101E200020910E2F020F111DD8015496EC91F0E075
:101E3000EE0FFF1FEE0FFF1FE55FFD4F2081318189
:101E4000428153810E94C56A9B01AC0160E070E051
:101E500080E792E40E947B6921E338E04CEA5CEB86
:101E60000E947B6920E030E040E853E40E9413695F
:101E70000E94E369F70162831F910F91FF90EF9039
:101E800008953F924F925F926F927F928F929F92AE
:101E9000AF92BF92CF92DF92EF92FF920F931F9378
:101EA000CF93DF9360909C0860921A099090A308EA
:101EB000909219097090F70870921B09809095080C
:101EC00080921C098091790880931D092091B108A6
:101ED00020931E098091DB0880931F099091E208EE
:101EE00090932009482F50E0440F551F440F551F71
:101EF000692F70E003E0660F771F0A95E1F7A22FC4
:101F0000B0E015E0AA0FBB1F1A95E1F790911209F6
:101F1000990F942B80911609982B962B8091170975
:101F20008295807F892B8A2B80930909E090340960
:101F3000F090350921E0E216F10419F480912901AD
:101F400005C080E0E114F10409F481E080930F09F9
:101F5000C7010397029720F08CE0E816F10419F40A
:101F60000091290106C000E0E2E0EE16F10409F458
:101F700001E000931209F4E0EF16F10421F02CE0E7
:101F8000E216F10419F4A090290105C0809180089F
:101F9000811181E0A82EA09213098091DF2E882361
:101FA00021F081E08093100906C08091B8088093E9
:101FB00010098091BF088093110920918708209310
:101FC000140981E090E000907D0802C0880F991FFD
:101FD0000A94E2F78093220980917608809315098C
:101FE000B090CD08B09216098091A209882341F0E3
:101FF00081E08093230910912309E2EAFEE216C0F2
:102000008091A12E882361F480913309882341F4C3
:102010008091A80A882321F480910F2F882319F03A
:1020200080912901E6CF10922309E5CF8081882392
:1020300011F01091290131968EE2E23BF807B1F7D9
:1020400010932309E5E0EE16F10421F481E080937A
:10205000170902C010921709C090DB2ED090DC2E19
:10206000D0922809C0922709F8E0EF16F10419F47C
:102070008091290102C080918E0880931809E09117
:102080009D0930E0EE2309F431E030930E09EE2390
:1020900011F081E002C08091290180932109462B33
:1020A000572B8B2D90E0482B592B4A2B5B2B809183
:1020B000170990E0F4E0880F991FFA95E1F7482B93
:1020C000592B882D90E076E0880F991F7A95E1F7DB
:1020D000482B592B822F90E09695982F882797951B
:1020E0008795482B592B972D80E0482B592B962DFF
:1020F000990F990F80E0482B592B992D990F990F23
:10210000990F80E0482B592B20912109922F92950D
:10211000907F80E0482B592B912F9295990F990F22
:10212000907C80E0482B592B932F9295990F907EAD
:1021300080E0482B592B802F90E0880F991F482B67
:10214000592B9A2D990F80E0482B592B50930B094E
:1021500040930A096090A309C62DD0E081E090E089
:102160009C01062C02C0220F331F0A94E2F7309321
:1021700025092093240945E0E416F10409F451C22D
:1021800066E0E616F10484F473E0E716F10409F45E
:10219000E3C0F4E0EF16F1040CF018C222E0E216FE
:1021A000F10409F048C210C049E0E416F10409F452
:1021B000D3C06CE0E616F10409F408C277E0E71634
:1021C000F10409F038C2C8C0BB2041F00090A40956
:1021D00002C0880F991F0A94E2F729C2EE2309F47E
:1021E0006CC09091D72E992309F44BC08091D82EC2
:1021F000482F50E04F70507060E070E020E030E019
:10220000E92FF0E001E0E02EF12C012D112D10C09E
:10221000C901840F951F5701680104C0AA0CBB1C9B
:10222000CC1CDD1C8A95D2F76A297B292F5F3F4F92
:10223000E217F3076CF780912901FE01E65DFE4F7E
:10224000E081C35CD64F288140E050E0882311F440
:1022500041E050E08091A5098F7002C0440F551FE6
:102260008A95E2F740955095642375238E2F90E070
:102270002F7002C0880F991F2A95E2F768277927E7
:102280005AC040912901FE01E65DFE4F8081C35C8A
:10229000D64F288190E02F7002C0880F991F2A9591
:1022A000E2F750E02091A5092F7002C0440F551F9E
:1022B0002A95E2F784279527BAC19091D72E9923C2
:1022C00009F43EC08091D82E482F50E04F705070D6
:1022D00060E070E020E030E0E92FF0E011E0E12E76
:1022E000F12C012D112D10C0C901840F951F57012C
:1022F000680104C0AA0CBB1CCC1CDD1C8A95D2F75B
:102300006A297B292F5F3F4FE217F3076CF7809113
:10231000290120E030E0882311F421E030E08091B1
:10232000A5098F7002C0220F331F8A95E2F720950E
:1023300030956223732370930409609303097BC172
:102340008091290190E02091A5092F7002C0880F8B
:10235000991F2A95E2F76BC1992009F04FC1FE0140
:10236000EC54F14D7080372C3294B0EF3B22209129
:102370009E2E30E040E050E000E010E060E070E0D1
:102380004E01880C991CCE01F6E0880F991FFA9532
:10239000E1F7880E991E83E994E06C012C9DC00141
:1023A0002D9D900D3C9D900D1124880E991EE1E00D
:1023B000AE2EB12CC12CD12C86E299E0289F2001B1
:1023C000299F500C389F500C1124832D840FA82F67
:1023D000B0E020E1621669F4FD01EE0FFF1FEA0F85
:1023E000FB1FE40DF51DE05FFC4E808180FF3AC0CD
:1023F0000DC0A80DB91DAA0FBB1FAB53B54F8C91D3
:10240000982F917081FF0FC09923E1F0D601C5018B
:10241000042E04C0880F991FAA1FBB1F0A94D2F76D
:10242000682B792B1FC0992369F0D601C501042EB2
:1024300004C0880F991FAA1FBB1F0A94D2F7082B4C
:10244000192B10C0D601C501042E04C0880F991F96
:10245000AA1FBB1F0A94D2F7809590956823792311
:10246000082319234F5F5F4F4034510509F0ADCF6A
:1024700000930709109308096093050970930609F2
:10248000FE01EB53F14D30817316B1F4FE01E65DB0
:10249000FE4F8081FE01E35CF64F208190E02F70BB
:1024A00002C0880F991F2A95E2F7862797279093F5
:1024B00004098093030904C070930409609303091D
:1024C00080912609883C08F17316B9F4FE01E65D97
:1024D000FE4F8081C35CD64F288190E02F7002C0F0
:1024E000880F991F2A95E2F780279127862B972B33
:1024F000909304098093030906C0062B172B1093B1
:102500000409009303091092260947E0E416F10438
:1025100029F069E0E616F10409F08DC07720A1F4F6
:1025200080913B09803108F086C02091290130E07C
:1025300002C0220F331F8A95E2F780910309909120
:1025400004098227932773C071E0771679F42091EC
:102550003B09203208F06FC0203108F46CC0809134
:10256000290190E030E02051304024C082E078160C
:1025700079F420913B09203308F05DC0203208F443
:102580005AC08091290190E030E02052304012C0C2
:10259000E3E07E1609F04FC020913B09203408F09B
:1025A0004AC0203308F447C08091290190E030E010
:1025B0002053304002C0880F991F2A95E2F72091DE
:1025C0000309309104092827392718C08091290967
:1025D0008823C9F081E00E94820520919A093091F8
:1025E0009B0940910D0950E059014A9D90014B9D76
:1025F000300D5A9D300D1124282B392B30930409AE
:102600002093030918C0009196091091970981E061
:102610000E948205082B192B1093040900930309CB
:102620000AC080919409909195098C299D299093D5
:1026300004098093030960910A0970910B09809144
:10264000030990910409409109090E949409DF91BE
:10265000CF911F910F91FF90EF90DF90CF90BF909F
:10266000AF909F908F907F906F905F904F903F9032
:102670000895DF92EF92FF920F931F93CF93DF9312
:1026800020919E2E803109F48CC0622F70E0282F9B
:1026900030E084E890E0289FD001299FB00D389F5A
:1026A000B00D112486E299E0689FA001699F500D4A
:1026B000789F500D1124FD01E40FF51FE555F54FEE
:1026C000E656FF4FE190A950B34EA656BF4FED928C
:1026D00080818C931296329680818C9382918E9316
:1026E000F901E950F34E4555554F420F531FDA019A
:1026F00017968C91878350E0E90106E0CC0FDD1F2F
:102700000A95E1F7220F331FC20FD31F83E994E02C
:10271000689F8001699F100D789F100D11240C0F88
:102720001D1F852F90E09E01280F391F220F331F98
:10273000B9016F5E724EF801E80FF91FEE0FFF1F2F
:10274000DF01AB53B54F8C91482F42954695469586
:10275000437011969C919770990F990F942B492F64
:102760004295440F440F407C8F73842BDB018C9384
:1027700096959695977011968C911197887F892BD5
:1027800011968C932E5E324EEA53F54F9081987FCE
:10279000F90180818770892B80835F5FE51608F6D9
:1027A00081C030E086E299E0A901489F9001499FED
:1027B000300D589F300D1124F901E555F54FEF59B3
:1027C000F74FD080D092582582918093572532962A
:1027D000819180935925808180935A2534978081F7
:1027E0008093562500E0E901802F90E0DC01AA0FDC
:1027F000BB1FA80FB91F9D01245A3A4DAD014C0FC4
:102800005D1F90E1E92E93E1F92EE40EF51EF7012C
:102810001081912F9170F90180818E7F892B8083A7
:10282000BD01625A7A4DFA01EE5EFC4E9081FB01C9
:1028300080818078E92FE0779F70892B8E2BFB01B8
:102840008083912F9E73F9018081817C892B808305
:10285000A35ABA4D4F5E5C4EFA019081987F8C91DD
:102860008770892B8C931295169516951370D70146
:1028700011969C919770990F990F912B492F429522
:10288000440F440F407CF90180818F73842B808337
:10289000969596958181887F892B81830F5FD016CD
:1028A00008F0A2CFDF91CF911F910F91FF90EF9091
:1028B000DF900895CF92DF92EF92FF920F931F93D4
:1028C000CF93DF93462F20919E2E803109F4A3C031
:1028D000622F70E0C82FD0E050E084E890E0489F7D
:1028E000D001499FB00D589FB00D1124A950B34E8F
:1028F000A656BF4FCD90C89FF001C99FF00DD89F3D
:10290000F00D112486E299E0689F9001699F300DD7
:10291000789F300D1124E20FF31FE555F54FE65671
:10292000FF4FC1928C918083329612968C91808356
:102930008E9182932555354F2C0F3D1FFA01E9509A
:10294000F34E8781D90117968C93DD248E01000FF9
:10295000111FCE0126E0880F991F2A95E1F7080F75
:10296000191F83E994E0FC016E9FC0016F9F900DD9
:102970007E9F900D1124080F191F7A0196E0EE0C2E
:10298000FF1C9A95E1F7440F551FE40EF51E8D2D9F
:1029900090E09801280F391F220F331FB9016B53A4
:1029A000754FF701E80FF91FEE0FFF1FDF01AF5E54
:1029B000B24E8C91482F429546954695437011969C
:1029C0009C919770990F990F942B492F4295440F22
:1029D000440F407C8F73842BDB018C9396959695E6
:1029E000977011968C911197887F892B11968C93F3
:1029F0002A53354FEE5EF24E9081987FF901808127
:102A00008770892B8083D394CD1408F6CE55D14D91
:102A100081E0888386C030E0D090582586E299E036
:102A2000A901489F9001499F300D589F300D1124F6
:102A3000F901E555F54FEF59F74FD08280915725B1
:102A40008293329680915925819380915A25808373
:102A5000349780915625808300E0E901802F90E033
:102A6000DC01AA0FBB1FA80FB91FAD014C0F5D1FE2
:102A70009A01205F3C4E8CE5E82E85E2F82EEA0EA6
:102A8000FB1EF7011081912F9170F90180818E7FDB
:102A9000892B8083BA016E5E7C4EFD01E25AFA4DAD
:102AA0009081FB0180818078E92FE0779F70892BEE
:102AB0008E2BFB018083912F9E73F9018081817C95
:102AC000892B80834F5E5C4EA35ABA4D9C91987FB0
:102AD000DA018C918770892B8C9312951695169537
:102AE0001370F70191819770990F990F912B492FCE
:102AF0004295440F440F407CD9018C918F73842BF5
:102B00008C939695969511968C911197887F892B29
:102B100011968C930F5FD01608F0A0CF81E08093C0
:102B2000A80A81E080932B02DF91CF911F910F9132
:102B3000FF90EF90DF90CF900895CF93DF93209197
:102B40009E2E30E0C82FD0E084E890E0C89FF001CE
:102B5000C99FF00DD89FF00D112486E299E0AC01D9
:102B6000249FC001259F900D349F900D1124E80FE4
:102B7000F91FE555F54FE656FF4F8FE0819388E149
:102B80008083329681E08083129260E070E0AE0133
:102B9000440F551FCE01E6E0880F991FEA95E1F733
:102BA000480F591F83E994E0FC012E9FC0012F9F1D
:102BB000900D3E9F900D1124480F591FFA01E60F0A
:102BC000F71FEE0FFF1FDF01AB53B54F82E08C9371
:102BD00011968C911197887F846011968C93EA539B
:102BE000F54F8081877080836F5F7F4F6034710500
:102BF00029F7CE55D14D81E0888380932B02DF9158
:102C0000CF910895CF93DF9380919E2E90E026E29E
:102C100039E0A901849F9001859F300D949F300D6C
:102C20001124F901E555F54FEF59F74F8FE08083F7
:102C300088E18293329681E08193108234971082EA
:102C400040E050E0B901FA01EE0FFF1FE40FF51F5D
:102C5000E60FF71FDF01A05FBC4E8C918E7F8C9337
:102C60009F012E5E3C4EE9018881807880638883D5
:102C70008C91817C88618C93EF5EFC4E80818770A3
:102C800080838C918F738C9311968C911197887F90
:102C900011968C934F5F5F4F40345105A1F681E050
:102CA0008093A80A80932B02DF91CF9108951F9300
:102CB00010E0812F0E9439131F5F1131D1F78091ED
:102CC000E02E8093F72E8091E22E8093F92E809152
:102CD000E42E9091E52EA091E62EB091E72E809300
:102CE000FB2E9093FC2EA093FD2EB093FE2E809190
:102CF000F22E8093092F8091F42E80930B2F8091D8
:102D0000E12E8093F82E8091E32E8093FA2E80910D
:102D1000E82E9091E92EA091EA2EB091EB2E8093AF
:102D2000FF2E9093002FA093012FB093022F80913C
:102D3000F32E80930A2F8091F52E80930C2F1F91F4
:102D400008951F9310E0812F612F0E945A141F5F76
:102D50001131C9F78091F72E8093E02E8091F92EE2
:102D60008093E22E8091FB2E9091FC2EA091FD2E5F
:102D7000B091FE2E8093E42E9093E52EA093E62E44
:102D8000B093E72E8091092F8093F22E80910B2F24
:102D90008093F42E8091F82E8093E12E8091FA2E6C
:102DA0008093E32E8091FF2E9091002FA091012F10
:102DB000B091022F8093E82E9093E92EA093EA2EF3
:102DC000B093EB2E80910A2F8093F32E80910C2FDD
:102DD0008093F52E1F9108951F9310E0812F0E947C
:102DE0009D151F5F1031D1F70E9402161F910895A3
:102DF0002F923F924F925F926F927F928F929F920B
:102E0000AF92BF92CF92DF92EF92FF920F931F93F8
:102E1000DF93CF9300D000D0CDB7DEB720919E2EA8
:102E2000803109F0F7C0A22EBB2486E299E0A89E6B
:102E30009001A99E300DB89E300D1124F901E45F78
:102E4000FC4E9080D901A05FBC4E9C918824839455
:102E50008922F901EE5EFC4E80810FE0702E78220F
:102E6000F82EF2941FE0F12247E0F422E92EE694D6
:102E70005FE1E522F901EF5EFC4EC080C694C69486
:102E8000C694929596959695937011961C9117708D
:102E9000110F110F192BDD24D3943C832B836EC0AB
:102EA0002D2D30E0C9010197AC01440F551F480F8B
:102EB000591F8B819C81480F591FBA01605F7C4E5E
:102EC0002901440C551C420E531E480E591ED201B6
:102ED000A05FBC4EBA83A9839C919170FB01808155
:102EE0008E7F892B808332E1232E33E1332E240E13
:102EF000351E92012E5E3C4ED9019C919F70F101CE
:102F00008081807F892B80839C9190778F78892B1B
:102F10008083A981BA818C918295869586958370EC
:102F200011969C919770990F990F982B292F2295A4
:102F3000220F220F207CFB0180818F73822B8083E4
:102F4000969596958181887F892B81834F5E5C4E13
:102F500021E133E1420E531ED2019C91987FFA0188
:102F600080818770892B8083A981BA819C919E730F
:102F7000FB018081817C892B8083D3949D1408F090
:102F80008FCF892D90E0FC01EE0FFF1FE80FF91F96
:102F900086E299E09C01A29EC001A39E900DB29E84
:102FA000900D1124E80FF91FAF01405F5C4EDA016C
:102FB0008C918E7F88298C939F012E5E3C4ED90187
:102FC0008C918078B7E0FB22F29490EFF922872968
:102FD0008F29D9018C93912F9295990F990F907CFD
:102FE000DA018C918F73892B8C93EF5EFC4ECC0CA5
:102FF000CC0CCC0C169516951C291083BFE1EB2246
:10300000EE0CFA018081817C8E29808381E080939F
:10301000A80AF1C0C22EDD24E82EFF2484E890E047
:10302000E89ED001E99EB00DF89EB00D112486E215
:1030300099E09C01C29EC001C39E900DD29E900D4E
:103040001124A80FB91FFD01EB5BF44F5080FD0167
:10305000EB53F54F8081442443944822082F069572
:103060000170382F369536953F70829586958695F6
:10307000837011811770110F110F182BAA53B54FC0
:10308000AC90A694A694A694BB24B3943701660C86
:10309000771C4701B6E0880C991CBA95E1F7A301AB
:1030A000480D591D83E994E0DC01CA9EC001CB9E06
:1030B000900DDA9E900D1124480F591F5C834B83AD
:1030C00059C0EB2DF0E031974B815C814E0F5F1FB3
:1030D0003196440F551F75EC272E7AE0372E240EBB
:1030E000351E8B819C81E80FF91FEE0FFF1FBF017A
:1030F0006B53754FDB019C919170D1018C918E7F48
:10310000892B8C93DB019C9192708D7F892BD1014F
:103110008C93DB019C919C73837C892BD1018C93D4
:10312000DB012C91229526952695237011969C9172
:103130009770990F990F922B292F2295220F220F0A
:10314000207C8F73822BD1018C9396959695119646
:103150008C911197887F892B11968C934A53554FE8
:10316000EA53F54F9081987FFA0180818770892B0F
:103170008083B3945B1408F0A4CFF301E80DF91D2C
:1031800083E994E0AC01C49EC001C59E900DD49E1D
:10319000900D1124E80FF91FE50DF11DEE0FFF1F33
:1031A000DF01AB53B54F0170000F02703F70330F5A
:1031B000330F0429812F8295880F880F807C032B81
:1031C000082B0C931695169511968C911197887F64
:1031D000812B11968C93EA53F54FAA0CAA0CAA0CDA
:1031E000808187708A29808382EA9EE2E80EF91E38
:1031F00081E0D7018C938091340990913509893011
:10320000910511F0079719F481E080932B020F903C
:103210000F900F900F90CF91DF911F910F91FF9022
:10322000EF90DF90CF90BF90AF909F908F907F9066
:103230006F905F904F903F902F9008952F923F9204
:103240004F925F926F927F928F929F92AF92BF92B6
:10325000CF92DF92EF92FF920F931F93DF93CF9362
:1032600000D000D000D0CDB7DEB740919E2E803187
:1032700009F003C1642E772486E299E0689EA001DC
:10328000699E500D789E500D1124FA01E45FFC4EAA
:10329000208130E0F901EE0FFF1FE20FF31FE40F72
:1032A000F51FBF01605F7C4EDB019C91332433949A
:1032B0003922DF01AE5EBC4E8C91BFE02B2E28225E
:1032C000E82EE294AFE0EA22B7E0EB22B92EB69402
:1032D0008FE1B822EF5EFC4EA080A694A694A6943F
:1032E0009295969596959370DB011196FC90B7E0B8
:1032F000FB22FF0CFF0CF92A1E821D8269012601A8
:103300000894410851084A0172C0C601ED81FE814E
:103310008E1B9F0B9C01220F331F280F391F280D76
:10332000391DA901405F5C4EFB01EE0FFF1FE60F48
:10333000F71FE80DF91D8F01005F1C4ED8019C910D
:103340009170DA018C918E7F892B8C93B9016E5E1E
:103350007C4E7A836983BF016E5E7C4EDB019C915B
:103360009F70A981BA818C91807F892B8C93DB011E
:103370009C9190778F78892BA981BA818C93D80101
:103380008C91829586958695837011969C91977005
:10339000990F990F982B692F6295660F660F607CC5
:1033A000DA018C918F73862B8C9396959695119656
:1033B0008C911197887F892B11968C932F5E3C4EB0
:1033C000EF5EFC4E9081987FF90180818770892B98
:1033D0008083D8019C919E73FA018081817C892B26
:1033E00080832D813E812F5F3F4F3E832D83B2012D
:1033F0008D819E81681B790B8C159D0509F085CF09
:1034000086E299E0689EA001699E500D789E500D5D
:103410001124DA01A05FBC4E8C918E7F83298C939E
:103420009A012E5E3C4EF90180818078F7E0EF2210
:10343000E29410EFE12282298E29F90180839F2DE9
:103440009295990F990F907C8C918F73892B8C9307
:103450004F5E5C4EAA0CAA0CAA0CF694F694FA28BD
:10346000FA01F082FFE1BF22BB0C8C91817C8B2999
:103470008C9381E08093A80AF6C0842E9924282F8B
:1034800030E03E832D8384E890E0289FF001299F5F
:10349000F00D389FF00D112486E299E0BC01869E64
:1034A000C001879E900D969E900D1124E80FF91F84
:1034B000EB5BF44F408150E0220F331F8D819E81E2
:1034C000E6E0880F991FEA95E1F7280F391F83E995
:1034D00094E0DC018A9EC0018B9E900D9A9E900D17
:1034E0001124280F391FF901E40FF51FEE0FFF1FFC
:1034F000DF01AB53B54F8C91332433943822082F1E
:1035000006950170B82EB694B6946FE0B6228295F7
:1035100086958695837011961C911770110F110F67
:10352000182BEA53F54FA080A694A694A694EE24F7
:10353000FF246A012601089441085108390154C04A
:10354000D601AE19BF09A60DB71DAA0FBB1FBC83BC
:10355000AB83AD014B53554FD301A80FB91FAA0F31
:10356000BB1FBD016B53754FFB0190819170FA0138
:1035700080818E7F892B8083FB01908192708D7F6B
:10358000892BFA018083FB0190819C73837C892BBA
:10359000FA018083FB0120812295269526952370D0
:1035A00091819770990F990F922B292F2295220FB5
:1035B000220F207C8F73822BFA018083969596953B
:1035C0008181887F892B81834B815C814A53554F50
:1035D000AA53B54F9C91987FDA018C918770892B03
:1035E0008C930894E11CF11CC2018E199F09EC1404
:1035F000FD0409F0A5CF84E890E02D813E81289F4D
:10360000F001299FF00D389FF00D112486E299E01A
:10361000BC01869EC001879E900D969E900D112440
:10362000E80FF91FDF01AB53B54F0170000F0270B7
:103630007FE0B722BB0CBB0C0329812F8295880F3A
:10364000880F807C0B29082B0C93EA53F54FAA0CAA
:10365000AA0CAA0C169516951A2910832E55314DD1
:1036600081E0D9018C93809134099091350989309A
:10367000910511F0079719F481E080932B022696AB
:103680000FB6F894DEBF0FBECDBFCF91DF911F9173
:103690000F91FF90EF90DF90CF90BF90AF909F90F1
:1036A0008F907F906F905F904F903F902F900895F4
:1036B000CF93DF93782F6F5F20919E2E8031C9F5D5
:1036C00030E086E299E0289FA001299F500D389FA5
:1036D000500D11242BC0862F90E0FC01EE0FFF1F30
:1036E000E80FF91FE40FF51FDF01A05FBC4E8C91BE
:1036F0008E7F8C939F012E5E3C4EE90188818078FD
:10370000806388838C91817C88618C93EF5EFC4E12
:103710008081877080838C918F738C9311968C91AC
:103720001197887F846011968C936F5F603498F254
:1037300088C030E083E994E0289FA001299F500DC4
:10374000389F500D11247AC0262F30E0872F90E04B
:10375000FC01B6E0EE0FFF1FBA95E1F7880F991F45
:10376000E80FF91FE40FF51FE20FF31FEE0FFF1F25
:10377000EB53F54F80818E7F8083872F90E0FC0193
:10378000B6E0EE0FFF1FBA95E1F7880F991FE80F1B
:10379000F91FE40FF51FE20FF31FEE0FFF1FEB53AE
:1037A000F54F808182608083872F90E0FC01B6E036
:1037B000EE0FFF1FBA95E1F7880F991FE80FF91F69
:1037C000E40FF51FE20FF31FEE0FFF1FEB53F54F52
:1037D0008081837C8083872F90E0FC01B6E0EE0F30
:1037E000FF1FBA95E1F7880F991FE80FF91FE40F43
:1037F000F51FE20FF31FEE0FFF1FEB53F54F808114
:103800008F7380838181887F84608183872F90E09C
:10381000FC01B6E0EE0FFF1FBA95E1F7880F991F84
:10382000E80FF91FE40FF51FE20FF31FEE0FFF1F64
:10383000EA53F54F8081877080836F5F603408F4AE
:1038400083CFDF91CF910895DF92EF92FF920F9394
:103850001F93CF93DF9380919E2E90E026E239E074
:10386000829FF001839FF00D929FF00D1124E5558A
:10387000F54F10821182C0E0D0E034E8E32EF12C45
:1038800006E219E0DD24D3944C2F80919E2E282F40
:1038900030E0CE9DF001CF9DF00DDE9DF00D1124A6
:1038A000209FC001219F900D309F900D1124E80FA3
:1038B000F91FEB5BF44FE081DC01A555B54F8C910E
:1038C0008E1718F4EC93C093B32ECE9DF001CF9DCC
:1038D000F00DDE9DF00D1124209FC001219F900D61
:1038E000309F900D1124E80FF91FEA5BF44FE0813F
:1038F000DC01A555B54F11968C9111978E1710F4D8
:103900001196EC93FE01E955F64FD082CE9DF00161
:10391000CF9DF00DDE9DF00D1124209FC001219F51
:10392000900D309F900D1124E80FF91FEB5BF44FC1
:10393000842F60810E94581B2196C031D10509F067
:10394000A3CF80919E2E282F30E086E299E0289F19
:10395000F001299FF00D389FF00D1124E555F54F2A
:10396000EF59F74F9081E156F8408081891720F494
:10397000908380E18093B32E86E299E0289FF00146
:10398000299FF00D389FF00D1124E555F54FE05AB1
:10399000F74F9081E056F8408181891708F49183B0
:1039A00081E08093B70986E299E0289FF001299F82
:1039B000F00D389FF00D1124E45FFC4E80E1608132
:1039C0000E94581BDF91CF911F910F91FF90EF90B4
:1039D000DF90089580912909882319F0833038F504
:1039E00020C020912E0930912F0980E690E0AC0193
:1039F000249FC001259F900D349F900D11246CE3EE
:103A000070E00E94536B9B0140E050E060E874E876
:103A10008EE190E00E949C6B309389002093880097
:103A2000089584EF91E09093890080938800089531
:103A3000E1E8F0E0108280818093800080818A60DC
:103A400080830E94EA1CEFE6F0E080818260808340
:103A500008959F92AF92BF92CF92DF92EF92FF9222
:103A60000F931F93DF93CF9300D000D00F92CDB769
:103A7000DEB7809134099091350982309105D1F0FB
:103A80000C97C1F080911D2F90E061E070E00E94E2
:103A9000210B982F843008F093E090931D2F809194
:103AA000BA2F981739F09093BA2F81E080932C02A7
:103AB00080932B028091222F882309F4B7C00091B4
:103AC000A30960919E2E0031A1F4862F90E026E29A
:103AD00039E07C01E29EC001E39E900DF29E900DC4
:103AE0001124835F9C4E61E041E027E008EA1AE080
:103AF00020C010E084E890E09C01029FC001039F79
:103B0000900D129F900D1124462F50E026E239E0CF
:103B1000B901469F9001479F300D569F300D1124EB
:103B2000820F931F0E55114D885B944F61E041E069
:103B300027E00E947D0B80919C08882339F48091B6
:103B4000340990913509029709F070C04091A3099A
:103B500060919E2E4031A1F4262F30E086E299E05C
:103B6000289FF001299FF00D389FF00D1124E55595
:103B7000F54FEE59F74F8081E256F84083831FC01E
:103B8000262F30E086E299E0289FD001299FB00DD2
:103B9000389FB00D1124242F30E084E890E0289F56
:103BA000F001299FF00D389FF00D1124EA0FFB1F43
:103BB000E85BF44F8081A555B54F13968C9320E0B8
:103BC00030E004E810E066E279E0FF24F3948091AD
:103BD0009E2E90E0209FF001219FF00D309FF00D70
:103BE0001124DC01A69FC001A79F900DB69F900DE8
:103BF0001124E80FF91FE85BF44FDC01A555B54F20
:103C0000AD014D5F5F4F13968C9113978083F9013F
:103C1000EE55F14DF0822F5F3F4F20313105B9F65F
:103C2000FD01EE59F74FDA018C9180838091212FAD
:103C3000882309F4C1C00091A30960919E2E003130
:103C4000A1F4862F90E026E239E0FC01E29FC0015A
:103C5000E39F900DF29F900D1124825F9C4E61E0D6
:103C600040E023E008EA1AE020C010E084E890E099
:103C70007C010E9DC0010F9D900D1E9D900D112485
:103C8000462F50E026E239E0B901469F9001479F58
:103C9000300D569F300D1124820F931F0E55114D7C
:103CA000895B944F61E040E023E00E947D0B8091AE
:103CB0009C08882339F48091340990913509029742
:103CC00009F07AC02091A30960919E2E203171F4F1
:103CD000462F50E086E299E0489FF001499FF00DA1
:103CE000589FF00D1124E25FFC4E1AC0462F50E0A1
:103CF00030E084E890E0289FF001299FF00D389F84
:103D0000F00D112486E299E0DC014A9FC0014B9F2F
:103D1000900D5A9F900D1124E80FF91FE95BF44FA5
:103D2000208183E994E0489FF001499FF00D589F5E
:103D3000F00D1124EE0FFF1FE355F54F208320E017
:103D400030E094E8E92EF12C06E219E063E974E032
:103D5000DD24D39480919E2E90E02E9DF0012F9D26
:103D6000F00D3E9DF00D1124809FA001819F500D0C
:103D7000909F500D1124E40FF51FE95BF44F869FCF
:103D8000D001879FB00D969FB00D1124AA0FBB1FC5
:103D9000A355B54F8C918083F901EE55F14DD0823A
:103DA0002F5F3F4F20313105A9F6FA01E25FFC4E4B
:103DB0008C918083D092A80A809134099091350922
:103DC0008630910509F468C3873091056CF4823020
:103DD0009105E1F08230910514F40C949629059731
:103DE00014F00C949629C8C08830910509F4F0C2EB
:103DF000883091050CF468C48930910509F457C6E0
:103E00000C9711F00C9496290C9480298091B1089C
:103E1000882309F469C080919E2E90E0A6E2EA2EE4
:103E2000A9E0FA2E8E9DF0018F9DF00D9E9DF00D64
:103E30001124E555F54FD080CF0161E040E02FE33C
:103E400001EA1EE20E947D0B80919E2E90E08E9DE5
:103E5000F0018F9DF00D9E9DF00D1124E555F54F5D
:103E600080818D1591F120E030E064E870E046E259
:103E700059E011E080919E2E90E0269FF001279F4F
:103E8000F00D369FF00D11247C01E49EC001E59EEB
:103E9000900DF49E900D1124E80FF91FEB5BF44F89
:103EA000DC01A555B54F8C918083F901EE55F14D9C
:103EB00010832F5F3F4F20313105E1F6FD01EF59AF
:103EC000F74F8C9180831093A80A8091A309082F43
:103ED00010E00C54114DD801FC908F2D90E061E062
:103EE00070E00E94210BCFC680912E0961E00E94F4
:103EF000520B90932F0980932E098F31910530F446
:103F00008EE190E090932F0980932E0980912E09E5
:103F100090912F098A3F910530F08AEF90E09093BD
:103F20002F0980932E0920912E0930912F0980911D
:103F3000B72F9091B82F2817390749F03093B82F31
:103F40002093B72F0E94EA1C81E080932B0280917E
:103F50002909882311F00C9496298091F22E882348
:103F600019F080E00E94FF0E8091F32E882311F457
:103F70000C94962981E0EFC280911D2F8130A9F029
:103F8000813040F0823009F4A4C0833011F00C94E9
:103F90009629F9C18091EA08882309F463C68091C3
:103FA000A308882309F05EC646C60091A309609164
:103FB0009E2E0031A1F4862F90E026E239E07C01AC
:103FC000E29EC001E39E900DF29E900D1124845F4D
:103FD0009C4E61E040E02FE308EA1AE020C010E0C8
:103FE00084E890E09C01029FC001039F900D129F06
:103FF000900D1124462F50E026E239E0B901469F8A
:104000009001479F300D569F300D1124820F931F52
:104010000E55114D8B5B944F61E040E02FE30E9401
:104020007D0B80919E2E90E026E239E0829FF00188
:10403000839FF00D929FF00D1124E555F54F1082EE
:1040400020E030E064E870E046E259E080919E2E86
:1040500090E0269FF001279FF00D369FF00D112470
:10406000DC01A49FC001A59F900DB49F900D112469
:10407000E80FF91FEB5BF44FE081DC01A555B54F6C
:104080008C918E1718F4EC932093B32E2F5F3F4F33
:1040900020313105D9F680919E2E90E026E239E05C
:1040A000829FF001839FF00D929FF00D1124E55542
:1040B000F54FEF59F74F9081E156F840808189170D
:1040C00010F00C949629908380E18093B32E0C9489
:1040D00096292091A30960919E2E203171F4262FFC
:1040E00030E086E299E0289FF001299FF00D389F8B
:1040F000F00D1124E55FFC4E1AC030E0462F50E071
:1041000084E890E0289FF001299FF00D389FF00D82
:10411000112486E299E07C014E9DC0014F9D900DD7
:104120005E9D900D1124E80FF91FEA5BF44F10819A
:104130001831A9F0193128F41C30A9F01031B1F46C
:1041400010C0103341F0103619F0103279F405C068
:1041500010927D080BC081E007C082E005C083E0BB
:1041600003C084E001C085E080937D0880917D08D4
:1041700061E00E94520B982F863008F095E09093F2
:104180007D088091B62F981711F40C94962990937E
:10419000B62F81E080932B02E091A309E03119F45E
:1041A0008093A80A04C0F0E0EE55F14D8083809121
:1041B0007D088230A9F0833028F4882351F08130C3
:1041C00011F509C08430A1F0843060F08530D9F455
:1041D00015C010E601C010E3EE24FFE1FF2E13C06E
:1041E00010E2FACF18E1E4E0EE2E7BE1F72E0BC0EF
:1041F00010E168E0E62E57E1F52E05C01CE04AE02C
:10420000E42E35E1F32E8091A3096E2D4F2D0E94EF
:104210002F0C2091A30960919E2E203171F4262F3E
:1042200030E086E299E0289FF001299FF00D389F49
:10423000F00D1124E55FFC4E1AC030E0462F50E02F
:1042400084E890E0289FF001299FF00D389FF00D41
:10425000112486E299E09C01429FC001439F900D8A
:10426000529F900D1124E80FF91FEA5BF44F108361
:104270008091CD08882311F40C9496294091A309CC
:1042800060919E2E4031A1F4262F30E086E299E025
:10429000289FF001299FF00D389FF00D1124E5555E
:1042A000F54FE05AF74F8081E056F84081831FC0F8
:1042B000262F30E086E299E0289FD001299FB00D9B
:1042C000389FB00D1124242F30E084E890E0289F1F
:1042D000F001299FF00D389FF00D1124EA0FFB1F0C
:1042E000EA5BF44F8081A555B54F11968C9300E0A1
:1042F00010E024E8A22EB12C96E2C92E99E0D92E26
:104300009924939480919E2E90E00A9DD0010B9D5C
:10431000B00D1A9DB00D11248C9DF0018D9DF00DF6
:104320009C9DF00D1124AE0FBF1FAA5BB44FE55545
:10433000F54F81818C93802F6E2D4F2D0E942F0C75
:10434000F801EE55F14D90820F5F1F4F00311105BE
:10435000C9F680E16E2D4F2D0E942F0C80919E2E6C
:1043600090E026E239E0829FF001839FF00D929F5A
:10437000F00D1124E555F54F8181E05AF74F808308
:104380009092A80AD3C78091EA088823D9F0809137
:104390009E2E90E04091A30926E239E0829FF00131
:1043A000839FF00D929FF00D1124E555F54FE40F1A
:1043B000F11D90E08781882309F491E0978381E0E3
:1043C00080932B0283EA99E061E040E020E175C030
:1043D00080911E2F813009F0A9C780911D2F813057
:1043E000F9F0813038F0823009F446C0833009F0AA
:1043F0009DC74CC08091290961E00E94520B982F03
:10440000833008F092E0909329098091B52F981796
:1044100009F48CC79093B52F81E080932A0929C0B5
:104420008091300961E00E94520B9C018E31910510
:1044300018F42EE130E005C08B3F910510F02AEF13
:1044400030E030933109209330098091B42F90E00F
:104450002817390709F46AC72093B42F0E94EA1C71
:10446000809130099091310990932F0980932E0902
:1044700081E08093330958C787E399E061E042E027
:104480002AE003E319E00E947D0B50C78DE299E01A
:1044900061E040E023E0F5CF80911D2F813081F075
:1044A000813030F08230A9F0833009F03FC756C028
:1044B0008EE09FE261E040E021E000E010E0E3CF29
:1044C00080910E2F90E08052914D61E040E024E019
:1044D00030C08091EA08882389F080910E2FE82F60
:1044E000F0E0E052F14D90E08289882309F491E0F8
:1044F000928B81E080930F2F80932B0280910E2F5F
:10450000282F30E0F901E052F14D82898823A1F48F
:1045100080919C08F9013296882329F0CF018052BE
:10452000914D6AE004C0CF018052914D61E040E0BE
:104530002EEF0FE01FE2A7CF813009F0F7C6C901C7
:104540008C50914D61E040E025E00FE01FE20E94B9
:104550007D0B80910E2F0E94FF0EE8C680919C0873
:1045600000910E2F882389F010E0000F111F000F1B
:10457000111F0C51114DD8016D917D918D919C9120
:104580002DEC3CEC4CEC5DE310C010E0000F111F73
:10459000000F111F0C51114DD8016D917D918D911E
:1045A0009C912AE037ED43E25CE30E94AA0BF801FC
:1045B000608371838283938380910E2FC82EDD24C4
:1045C000F601EE0FFF1FEE0FFF1FEC51F14DE080E3
:1045D000F18002811381C801B70120E030E040E0A2
:1045E00050E00E94776988235CF40F2EF0E0EF2EF4
:1045F000F0E0FF2EF0E00F2FF0E01F2FF02D14C0A1
:10460000C801B70120E030E040E85FE30E94C16AE2
:10461000181654F40F2EF0E0EF2EF0E0FF2EF0E825
:104620000F2FFFE31F2FF02DCC0CDD1CCC0CDD1C5D
:1046300024EE3EE2C20ED31ED601ED92FD920D9302
:104640001C931397E0910E2FF0E0EE0FFF1FEE0F7B
:10465000FF1FE20FF31FE080F18002811381C80188
:10466000B7012091B02F3091B12F4091B22F5091CE
:10467000B32F0E947769882369F0E092B02FF092FF
:10468000B12F0093B22F1093B32F81E080930F2F9F
:1046900080932B028091EA08882309F447C6E091B1
:1046A0000E2FF0E0EE0FFF1FEE0FFF1FEC51F14D4C
:1046B00080E090E0A0E8BFE380839183A283B3838E
:1046C00081E080930F2F30C620919E2E30E08091A4
:1046D0003B0990E0DC01AA0FBB1FA80FB91F86E2BF
:1046E00099E0F901E89F9001E99F300DF89F300DA6
:1046F0001124A20FB31FFD01EE5EFC4E8081082F36
:104700000F70829587708A83F901E555F54FE15A5C
:10471000F74F1081EF55F840A05FBC4E8C91869505
:104720008F71898380911D2F8130A1F1813038F004
:10473000823009F401C1833009F0F8C566C1809167
:10474000AA0A882309F48EC2813009F0EFC5812FAF
:1047500061E00E94520B482F893008F048E08091B8
:10476000AE2F481739F04093AE2F81E08093A80A0E
:1047700080932B0280919E2E90E026E239E0829F6A
:10478000F001839FF00D929FF00D1124E65FFC4E27
:104790004083CCC50E940B0C402F480FA02FB0E0E7
:1047A000642F70E0CD01861B970B8130910551F588
:1047B000212F30E0F901EE0FFF1FE20FF31FEE0F84
:1047C000FF1FEE0FFF1FAE0FBF1FA356BE4F9C91E2
:1047D000E60FF71FE356FE4F8081981709F441500A
:1047E000F901EE0FFF1FE20FF31FEE0FFF1FEE0F99
:1047F000FF1FE40FF11DE356FE4F8081981771F5FE
:1048000041502CC08F5F9F4F49F5212F30E0F901B7
:10481000EE0FFF1FE20FF31FEE0FFF1FEE0FFF1F44
:10482000AE0FBF1FA356BE4F9C91E60FF71FE35676
:10483000FE4F8081981709F44F5FF901EE0FFF1FBB
:10484000E20FF31FEE0FFF1FEE0FFF1FE40FF11D2E
:10485000E356FE4F8081981709F44F5F4F3F41F4B4
:104860008A8181508A838F3F09F41A824BE00AC003
:104870004C3040F08A818F5F8A83873010F087E068
:104880008A8340E04C3008F04BE08091AF2F48170E
:1048900039F04093AF2F81E08093A80A80932B02D8
:1048A0004093DE098091CE08882321F120E030E09A
:1048B00066E279E080919E2E90E0F901EE0FFF1FF5
:1048C000E20FF31F7C01E69EC001E79E900DF69E6D
:1048D000900D1124E80FF91FEE5EFC4E9091DE0959
:1048E0009F708081807F892B80832F5F3F4F203492
:1048F000310501F780913B0990E020919E2E30E038
:10490000FC01EE0FFF1FE80FF91F86E299E0BC01E2
:10491000269FC001279F900D369F900D1124E80F10
:10492000F91FEE5EFC4E4F70808180789A819770FF
:104930009295907F842BE1C48091CE088823B1F1B9
:104940000E940B0C8093DF098823C9F140E050E0FE
:1049500066E279E080919E2E90E0FA01EE0FFF1F53
:10496000E40FF51FDC01A69FC001A79F900DB69F25
:10497000900D1124E80FF91FEE5EFC4E2081822F6E
:1049800082958F709091DF09890F87708295807F63
:104990002F78282B20834F5F5F4F40345105D1F68D
:1049A00081E08093A80A80932B0209C0CE01029671
:1049B00061E040E027E008EA1AE00E947D0B809168
:1049C000EA08882311F083E08A8380913B0990E014
:1049D00020919E2E30E0FC01EE0FFF1FE80FF91F23
:1049E00086E299E07C012E9DC0012F9D900D3E9D99
:1049F000900D1124E80FF91FEE5EFC4E9A8197701E
:104A00009295907F80818F7878C4E05AF74FCE01DD
:104A1000019661E041E0208108EA1AE00E947D0BE6
:104A200089818093DD098091CE08882329F120E0D7
:104A300030E046E259E080919E2E90E0F901EE0FC1
:104A4000FF1FE20FF31FBC01649FC001659F900D23
:104A5000749F900D1124E80FF91FE05FFC4E9091B8
:104A6000DD099F71990F8081817C892B80832F5F65
:104A70003F4F20343105F9F680913B0990E02091B9
:104A80009E2E30E0FC01EE0FFF1FE80FF91F86E2BB
:104A900099E0DC012A9FC0012B9F900D3A9F900D59
:104AA0001124E80FF91FE05FFC4E99817BC31D8242
:104AB0001091A30960919E2EB0913B091031A1F590
:104AC0008B2F90E0262F30E0FC01EE0FFF1FE80F48
:104AD000F91F86E299E07901E89E9001E99E300D88
:104AE000F89E300D1124E20FF31FDF01A05FBC4ED2
:104AF0009C91492F429546954695437011968C910D
:104B00008770880F880F842B8983255F3C4ED901DD
:104B1000FC90EF5EFC4E80818695869586958A8313
:104B200096959F719C8375C04B2F50E070E0812F4C
:104B300090E0FC01A6E0EE0FFF1FAA95E1F7880FB9
:104B4000991FE80FF91F83E994E0689FD001699FDE
:104B5000B00D789FB00D1124EA0FFB1FE40FF51F75
:104B6000EE0FFF1FEB53F54F90819295969596951A
:104B7000937081818770880F880F892B8983212FFB
:104B800030E084E890E0289FF001299FF00D389FE5
:104B9000F00D112486E299E07C016E9DC0016F9DAD
:104BA000900D7E9D900D1124E80FF91FEA5BF44FE4
:104BB000F080F90196E0EE0FFF1F9A95E1F7220FC2
:104BC000331FE20FF31FEA0FFB1FE40FF51FEE0F79
:104BD000FF1FEB53F54F8081869586958F708A83F2
:104BE000812F90E09C01E6E0220F331FEA95E1F768
:104BF000880F991F280F391FA20FB31FA40FB51FCD
:104C0000AA0FBB1FAA53B54F8C91869586958695A2
:104C10008B8380911D2F813009F44CC0813038F096
:104C2000823009F489C1833009F080C37BC280914E
:104C3000EA088823B9F090E08091D62E882309F401
:104C400091E09093D62E992351F0E091A309F0E0E2
:104C5000DF01AB53B14D8C91EC54F14D808381E079
:104C600080932B028091D62E882309F05FC3809118
:104C7000A309082F10E00C54114DD801FC908F2D82
:104C800061E00E94520BF80180838091A309E82F14
:104C9000F0E0EC54F14D8081843008F083E08083B3
:104CA000E091A309F0E0EC54F14D8081F81609F091
:104CB0003AC33CC3F8E1FF16C9F0FF1540F05CE0D1
:104CC000E52EFE14F9F020E1F21631F515C030E3BF
:104CD000F31631F040E6F41619F050E2F516E1F45F
:104CE000CE01019661E040E02FE111C0CE010196B6
:104CF00061E044E02BE10BC0CE01019661E048E0A9
:104D000027E105C0CE01019661E04AE025E18E0170
:104D10000B5F1F4F0E947D0B8091EA08882331F0C2
:104D200080E1898381E08D8380932B028D818823AC
:104D300009F46AC04091A30960919E2EB0913B098D
:104D4000A981403159F58B2F90E0262F30E0FC01EE
:104D5000EE0FFF1FE80FF91F86E299E0BC01269FC6
:104D6000C001279F900D369F900D1124E80FF91F69
:104D7000E05FFC4E9A2F9295990F990F907C80815D
:104D80008F73892B8083A695A695A7708181887FD4
:104D90008A2B818381E08093A80A36C0262F30E0D9
:104DA000842F90E0FC0106E0EE0FFF1F0A95E1F76B
:104DB000880F991FE80FF91F83E994E07C012E9D6D
:104DC000C0012F9D900D3E9D900D1124E80FF91FFD
:104DD000EB0FF11DEE0FFF1FEB53F54F9A2F92953E
:104DE000990F990F907C80818F73892B8083A69572
:104DF000A695A7708181887F8A2B8183E42FF0E0BC
:104E0000EE55F14D81E080838091CE08882309F42E
:104E10008DC280919E2E90E026E239E0829FF001C3
:104E2000839FF00D929FF00D1124E555F54F898178
:104E300085838091A309803199F520E030E046E236
:104E400059E080919E2E90E0F901EE0FFF1FE20FD6
:104E5000F31F849FD001859FB00D949FB00D112446
:104E6000EA0FFB1FE05FFC4EA555B54F15969C91D0
:104E700015979295990F990F907C80818F73892B4C
:104E8000808315969C919695969597708181887FE1
:104E9000892B81832F5F3F4F2034310591F6FAC073
:104EA00040E050E0E3E9EE2EE4E0FE2E06E219E0F9
:104EB00020919E2E30E06091A309862F90E0FC01A6
:104EC00076E0EE0FFF1F7A95E1F7880F991FE80F44
:104ED000F91F2E9DC0012F9D900D3E9D900D112418
:104EE000E80FF91FE40FF51FEE0FFF1FEB53F54F0F
:104EF000209FD001219FB00D309FB00D1124A555EA
:104F0000B54F15969C9115979295990F990F907C96
:104F100080818F73892B808315969C9196959695A9
:104F200097708181887F892B81834F5F5F4F4034E9
:104F3000510509F0BDCFF0C0CE01029661E040E01E
:104F40002FE08E010B5F1F4F0E947D0B8091EA08BE
:104F5000882329F01A8281E08D8380932B028D8132
:104F6000882309F458C04091A30960919E2EB09106
:104F70003B09AA81403111F58B2F90E0262F30E0BC
:104F8000FC01EE0FFF1FE80FF91F86E299E0AC016C
:104F9000249FC001259F900D349F900D1124E80F90
:104FA000F91FEF5EFC4EAA0FAA0FAA0F808187702F
:104FB0008A2B808381E08093A80A2DC0262F30E0C1
:104FC000842F90E0FC0166E0EE0FFF1F6A95E1F789
:104FD000880F991FE80FF91F83E994E0BC01269F11
:104FE000C001279F900D369F900D1124E80FF91FE7
:104FF000EB0FF11DEE0FFF1FEB53F54FAF70AA0F34
:10500000AA0F8081837C8A2B8083E42FF0E0EE5509
:10501000F14D81E080838091CE08882309F486C118
:1050200080919E2E90E026E239E0829FF001839FDE
:10503000F00D929FF00D1124E555F54F8A81848380
:105040008091A309803151F520E030E046E259E03B
:1050500080919E2E90E0D901AA0FBB1FA20FB31F13
:10506000849FF001859FF00D949FF00D1124AE0FE9
:10507000BF1FAF5EBC4EE555F54F9481990F990F58
:10508000990F8C918770892B8C932F5F3F4F203421
:105090003105F1F681E08093A80A48C140E050E074
:1050A000A3E9EA2EA4E0FA2E06E219E020919E2E52
:1050B00030E06091A309862F90E0DC01F6E0AA0FB2
:1050C000BB1FFA95E1F7880F991FA80FB91F2E9DF6
:1050D000C0012F9D900D3E9D900D1124A80FB91F6A
:1050E000A40FB51FAA0FBB1FAB53B54F209FF001F4
:1050F000219FF00D309FF00D1124E555F54F94815F
:105100009F70990F990F8C91837C892B8C934F5FA3
:105110005F4F4034510551F6E62FF0E0EE55F14D6A
:1051200081E0ECC00091A309003109F040C0CE013C
:10513000049661E041E02F2D08EA1AE00E947D0B01
:105140008C818093DD098091CE08882341F090E026
:105150008091DD098C839F5F9034D1F706C08091E8
:10516000EA08882329F0F694FC8281E08093A80A5B
:1051700080913B0990E020919E2E30E0FC01EE0FE3
:10518000FF1FE80FF91F86E299E0DC012A9FC001AA
:105190002B9F900D3A9F900D1124E80FF91FE05FAF
:1051A000FC4E9C819F71990F8081817CA6C0EBE5AC
:1051B000F1E02CE08081F81621F021503197222374
:1051C000C9F7215010E00E55114DCE01039661E054
:1051D00040E00E947D0B8091EA08882351F01B82F9
:1051E000E091A309F0E0EE55F14D81E080838093DA
:1051F0002B028091CE08882309F456C080919E2E00
:1052000090E026E239E0829FF001839FF00D929FAB
:10521000F00D1124E555F54F8B81868360E070E039
:1052200093E9C92E94E0D92E86E2E82E89E0F82E83
:1052300040919E2E50E01091A3094C9DD0014D9DB0
:10524000B00D5C9DB00D1124812F90E09C0106E013
:10525000220F331F0A95E1F7880F991F280F391F76
:10526000A20FB31FA60FB71FAA0FBB1FAA53B54F9C
:105270004E9DF0014F9DF00D5E9DF00D1124E55502
:10528000F54F9681990F990F990F8C918770892B03
:105290008C936F5F7F4F6034710551F6E12FF0E022
:1052A000EE55F14D81E0808340913B0980919E2E27
:1052B00090E023E934E0829FF001839FF00D929FFC
:1052C000F00D11248091A30990E09C0166E0220F6B
:1052D000331F6A95E1F7880F991F280F391FE20FD6
:1052E000F31FE40FF11DEE0FFF1FEA53F54F9B81F3
:1052F000990F990F990F80818770892B808316C031
:105300008091892F90E061E070E00E94210B982F3E
:10531000873008F096E09093892F8091B92F9817E5
:1053200029F09093B92F81E080932B020F900F907A
:105330000F900F900F90CF91DF911F910F91FF90E1
:10534000EF90DF90CF90BF90AF909F900895CF9255
:10535000EF920F938130910509F046C06F5F7F4F48
:1053600009F067C080E58093102F1092112F83E21F
:105370009FE260E071E00E94DF678AE29FE260E006
:1053800071E00E94DF6781E39FE260E071E00E94CC
:10539000DF6788E39FE260E071E00E94DF678FE3F0
:1053A0009FE260E071E00E94DF6786E49FE260E0D8
:1053B00071E00E94DF678DE49FE260E071E00E948F
:1053C000DF6784E59FE260E071E00E94DF678CE8C0
:1053D0009FE262E143E124E105E176E1E72E57E156
:1053E000C52E0E94105C25C0892B19F56F5F7F4F79
:1053F00001F584E59FE20E9406698DE49FE20E9428
:10540000066986E49FE20E9406698FE39FE20E949C
:10541000066988E39FE20E94066981E39FE20E9499
:1054200006698AE29FE20E94066983E29FE20E9487
:1054300006690F91EF90CF90089580E090E06FEFB4
:105440007FEF0E94A729089581E090E06FEF7FEF42
:105450000E94A72908950E940360209107073091B8
:1054600008074091090750910A07621B730B840BD0
:10547000950B663071058105910508F470C00E9496
:105480000360609307077093080780930907909360
:105490000A074091102F3091112F2091C42F222301
:1054A00081F0213051F48DB38093C62F9DB380914C
:1054B000C52F809589238DBB04C08FB7F894809346
:1054C000C62F4CBD3DBD5E9A1EBC00000DB407FE4C
:1054D000FDCF8EB58093FD061EBC00000DB407FE07
:1054E000FDCF8EB58093FF061EBC00000DB407FEF5
:1054F000FDCF8EB5809301071EBC00000DB407FEE2
:10550000FDCF8EB5809303071EBC00000DB407FECF
:10551000FDCF8EB5809305075E98222339F08091E8
:10552000C62F213011F48DBB01C08FBF93B1907293
:105530009093152FEDEFF6E0A8EFB6E02081818182
:10554000281709F42C933296119687E0E730F80774
:10555000A9F78091162F981711F49093172F409167
:10556000102F3091112F2091C42F222381F0213050
:1055700051F48DB38093C62F9DB38091C52F809534
:1055800089238DBB04C08FB7F8948093C62F4CBD80
:105590003DBD5E9A1EBC00000DB407FEFDCF8EB56A
:1055A0008093FE061EBC00000DB407FEFDCF8EB535
:1055B000809300071EBC00000DB407FEFDCF8EB522
:1055C000809302071EBC00000DB407FEFDCF8EB510
:1055D000809304071EBC00000DB407FEFDCF8EB5FE
:1055E000809306075E98222339F08091C62F2130E0
:1055F00011F48DBB01C08FBF83B180728093162FD1
:105600000895DF92EF92FF920F931F93CF93DF9352
:105610000E942B2AE090FA06D090FC060091FB062F
:1056200010E0B801647070708AE998E00E94650526
:10563000B8016870707081EA98E00E946505B80151
:105640006170707085EF98E00E946505FF24B701D6
:10565000627070708EEE98E00E94650502701070A6
:105660008EE798E0B8010E946505B701647070701C
:1056700089ED98E00E946505B7016870707080EE52
:1056800098E00E946505B7016078707085E898E041
:105690000E946505CD2DD0E0BE01617070708BE574
:1056A00098E00E946505BE016270707082E698E025
:1056B0000E946505B701607270708FEA98E00E94E1
:1056C0006505B7016074707083E998E00E94650514
:1056D000B7016071707084EC98E00E94650521E06C
:1056E000E222FF248BEC98E0B7010E946505BE0121
:1056F0006072707089E698E00E946505BE01607175
:10570000707087EE98E00E9465057091F90660E080
:105710008091F80690E0682B792B82ED98E00E944A
:1057200065051092AC081092AB08D695C795D69532
:10573000C795CE018170682F8093A8088091A90831
:10574000681711F18091AA08882371F4613061F41F
:105750006093AB080E9403606093FC087093FD089F
:105760008093FE089093FF089091AA08913041F42D
:105770008091A808882321F49093AC081092AD087A
:105780008091A8088093AA088091A8088093A9080E
:105790008091AA088823B1F00E9403602091FC0840
:1057A0003091FD084091FE085091FF08621B730B79
:1057B000840B950B695E73408040904018F081E047
:1057C0008093AD08EEE0F7E010821182379687E013
:1057D000EE37F807C9F7DF91CF911F910F91FF9036
:1057E000EF90DF9008951F93CF93DF9310E0C0E018
:1057F000D0E081E792E3BE0140E00E94AF5F2196D6
:1058000081E792E3BE0143E60E94AF5F219681E704
:1058100092E3BE0144E60E94AF5F219681E792E3E6
:10582000BE0141E00E94AF5F219681E792E3BE0195
:1058300043E00E94AF5F2196CA30D105D1F61F5FC9
:105840001038A9F6DF91CF911F9108952F923F92C2
:105850004F925F926F927F928F929F92AF92BF9280
:10586000CF92DF92EF92FF920F931F93CF93DF932C
:10587000C0EEDEE214E0A12EB12CAC0EBD1EEE2473
:10588000FF24C82EDD2416010894211C311CB2E02F
:105890004B2E512C4C0C5D1CA3E06A2E712C6C0C11
:1058A0007D1CF4E08F2E912C8C0C9D1CB7016C0D8F
:1058B0007D1D81E792E348810E94AF5FB1016E0DCB
:1058C0007F1D81E792E34A810E94AF5F82010E0D46
:1058D0001F1DF50161917191819191915F0120E00E
:1058E00030E048EC52E40E94C56A0E94E3699B01E3
:1058F000AC0181E792E3B801422F0E94AF5FB30190
:105900006E0D7F1D81E792E34A890E94AF5FB4016B
:105910006E0D7F1D81E792E34C890E94AF5F219657
:1059200085E090E0E80EF91E9EE2C23ED90709F03C
:10593000BDCFDF91CF911F910F91FF90EF90DF903E
:10594000CF90BF90AF909F908F907F906F905F901F
:105950004F903F902F9008954F925F926F927F9259
:105960008F929F92AF92BF92CF92DF92EF92FF926F
:105970000F931F93CF93DF93C0EEDEE234E0C32E8C
:10598000D12CCC0EDD1E00E010E0E82EFF24270114
:105990000894411C511C22E0622E712C6E0C7F1C5D
:1059A00093E0892E912C8E0C9F1C84E0A82EB12CA4
:1059B000AE0CBF1CB8016E0D7F1D81E792E30E9403
:1059C000A85F853008F084E08883B201600F711F02
:1059D00081E792E30E94A85F8F3F09F48EEF8A83EC
:1059E000B301600F711F81E792E30E94A85F8536C3
:1059F00008F084E6682F70E0882777FD8095982F5F
:105A00000E94116A20E030E048EC52E40E947B6979
:105A1000F6016083718382839383B401600F711FE9
:105A200081E792E30E94A85F811181E08A8BB50132
:105A3000600F711F81E792E30E94A85F843008F035
:105A400083E08C8B1C861E86188A0B5F1F4F219665
:105A500084E090E0C80ED91E0A30110509F0AACFE3
:105A6000DF91CF911F910F91FF90EF90DF90CF903A
:105A7000BF90AF909F908F907F906F905F904F906E
:105A8000089510920E2F1092F62E80E00E94AC2CFA
:105A90000895AF92BF92CF92DF92EF92FF920F9351
:105AA0001F939091EC2E9F5F9093EC2E8091ED2EA2
:105AB0008F5F8093ED2E8091F62E882349F080E051
:105AC00098E00E946F0A80E098E00E94A40A2DC12D
:105AD000892F90E04091E22E20E031E0241B310933
:105AE000821793070CF48AC01092EC2E9091E02E4E
:105AF0009430D9F58091EE2E882309F074C060E0CF
:105B000070E080E090E020E031E040E050E00E9472
:105B10006C66E090E42EF090E52E0091E62E109158
:105B2000E72E0E94116AA80197010E94C56A5B01D5
:105B30006C01C801B70120E030E040E053EC0E9466
:105B4000C56A20E030E040E053E40E9413699B0105
:105B5000AC01C601B5010E9413690E94E369F4E03B
:105B6000660F771FFA95E1F73AC0A090E42EB09047
:105B7000E52EC090E62ED090E72E8091EE2EF92FE4
:105B8000E0E0E80FF11DEB54FD4F608170E08827E5
:105B900077FD8095982F0E94116AA60195010E94B9
:105BA000C56A7B018C01C601B50120E030E040E010
:105BB00053EC0E94C56A20E030E040E053E40E94CC
:105BC00013699B01AC01C801B7010E94136920E071
:105BD00030E040E851E40E94C56A0E94E369709396
:105BE000A42F6093A32F8091A32F9091A42F0E94A4
:105BF0006F0A8091EE2E8F5F8093EE2E8091ED2EB6
:105C000090E04091E32E20E031E0241B310982171F
:105C100093070CF48AC01092ED2E9091E12E9430EF
:105C2000D9F58091EF2E882309F074C060E070E010
:105C300080E090E020E031E040E050E00E946C66BF
:105C4000E090E82EF090E92E0091EA2E1091EB2ED4
:105C50000E94116AA80197010E94C56A5B016C014C
:105C6000C801B70120E030E040E053EC0E94C56A73
:105C700020E030E040E053E40E9413699B01AC0156
:105C8000C601B5010E9413690E94E369E4E0660F52
:105C9000771FEA95E1F73AC0A090E82EB090E92E80
:105CA000C090EA2ED090EB2E8091EF2EF92FE0E0FD
:105CB000E80FF11DEB54FD4F608170E0882777FD00
:105CC0008095982F0E94116AA60195010E94C56ACD
:105CD0007B018C01C601B50120E030E040E053ECCF
:105CE0000E94C56A20E030E040E053E40E9413695E
:105CF0009B01AC01C801B7010E94136920E030E0AC
:105D000040E851E40E94C56A0E94E3697093A22FA3
:105D10006093A12F8091A12F9091A22F0E94A40A9D
:105D20008091EF2E8F5F8093EF2E80913909882329
:105D300061F190913A0980912909813069F4E091EB
:105D40003709F0E0EE0FFF1FE95CFE4F0190F08194
:105D5000E02DF695E7950AC0E0913709F0E0EE0FE7
:105D6000FF1FE95CFE4F0190F081E02D9F5F909353
:105D70003A099150892F90E08E179F0730F00E94CA
:105D8000080A10923A0910923909809126098F5F0A
:105D9000809326091F910F91FF90EF90DF90CF9095
:105DA000BF90AF9008951F920F920FB60F920BB64F
:105DB0000F9211242F933F934F935F936F937F9391
:105DC0008F939F93AF93BF93EF93FF930E94492DBF
:105DD000FF91EF91BF91AF919F918F917F916F91C3
:105DE0005F914F913F912F910F900BBE0F900FBE7F
:105DF0000F901F901895FF920F931F93F82E0CE8A9
:105E00001FE2C8016F2D41E00E94255BC80165E1DA
:105E100073E00E94A364C8016F2D41E00E94255BDE
:105E20001F910F91FF9008950F931F930CE81FE2AD
:105E3000C80164E040E00E94255BC80163E773E0AD
:105E40000E94A36481E080931C2F1F910F910895FD
:105E50008CE89FE260E873E00E94A36408950F93CA
:105E60001F930CE81FE2C80160E040E00E94255B40
:105E7000C8016BE273E00E94A364C80160E041E0E6
:105E80000E94255B0E94282FC80160E041E00E942B
:105E9000255BC8016AE173E00E94A3641F910F9122
:105EA00008950F931F930CE81FE2C80160E040E0E3
:105EB0000E94255BC8016DE473E00E94A364C801E1
:105EC00060E041E00E94255B0E94282FC80160E04D
:105ED00041E00E94255BC8016CE373E00E94A3646B
:105EE0001F910F9108950F931F93CF93DF93C0E0FD
:105EF000D0E0082F10E006C08CE89FE261EA0E9423
:105F0000C6642196C017D107BCF3DF91CF911F91D2
:105F10000F91089588E00E94FB2EE0910E2FF0E093
:105F2000E052F14D8489823019F1833038F48823AE
:105F300009F440C0813009F047C031C0843031F0ED
:105F4000843020F1853009F03FC009C08CE89FE221
:105F500060E00E94F35A8CE89FE261E011C08CE897
:105F60009FE260E00E94F35A8CE89FE261E01FC06C
:105F70008CE89FE260E00E94F35A8CE89FE263E0C5
:105F80000E94F35A8CE89FE262E011C08CE89FE225
:105F900060E00E94F35A8CE89FE263E008C08CE85E
:105FA0009FE260E00E94F35A8CE89FE266E00E9464
:105FB000F35A08958CE89FE260E00E94F35A8CE85F
:105FC0009FE267E00E94F35A08951F93882319F017
:105FD0008FEF8093A52F2091A30940919E2E203111
:105FE00071F4242F30E086E299E0289FF001299F88
:105FF000F00D389FF00D1124E55FFC4E19C030E024
:1060000050E084E890E0289FF001299FF00D389F30
:10601000F00D112486E299E09C01429FC001439F4C
:10602000900D529F900D1124E80FF91FEA5BF44F79
:1060300010818091A52F181709F452C088E00E94A2
:10604000FB2E183109F1193130F41C3059F01031A0
:1060500009F044C010C0103371F11036A9F11032AC
:10606000E9F51BC08CE89FE260E00E94F35A8CE8DF
:106070009FE264E031C08CE89FE260E00E94F35A46
:106080008CE89FE261E011C08CE89FE260E00E9432
:10609000F35A8CE89FE261E01FC08CE89FE260E069
:1060A0000E94F35A8CE89FE263E00E94F35A8CE866
:1060B0009FE262E011C08CE89FE260E00E94F35A28
:1060C0008CE89FE263E008C08CE89FE260E00E94F9
:1060D000F35A8CE89FE266E00E94F35A1093A52FD2
:1060E0001F910895CF92DF92EF92FF920F931F932B
:1060F000CF93DF93EC018B017A01690163E27FE2C8
:106100000E94F966882321F58CE89FE260E041E077
:106110000E94255B8CE89FE260EA73E00E94A36422
:106120008C819D81029720F48CE89FE261E003C09E
:106130008CE89FE260E041E00E94255B8CE89FE2F2
:10614000BE010E94CE6583E29FE2BE010E94D96833
:10615000C8016AE27FE20E94F9668823E1F48CE8D4
:106160009FE264E041E00E94255B8CE89FE26BE9DE
:1061700073E00E94A3648CE89FE264E041E00E9427
:10618000255B8CE89FE2B8010E94CE658AE29FE21F
:10619000B8010E94D968C70161E37FE20E94F966F5
:1061A000882361F5C70160E070E00E94A366882340
:1061B00029F58CE89FE268E041E00E94255B8CE8CD
:1061C0009FE266E973E00E94A364F70184819581F0
:1061D000029720F48CE89FE269E003C08CE89FE21C
:1061E00068E041E00E94255B8CE89FE2B7010E94D5
:1061F000CE6581E39FE2B7010E94D968C60168E3DA
:106200007FE20E94F966882329F58CE89FE26CE022
:1062100041E00E94255B8CE89FE261E973E00E9407
:10622000A364F60184819581029720F48CE89FE2B3
:106230006DE003C08CE89FE26CE041E00E94255BCA
:106240008CE89FE2B6010E94CE6588E39FE2B6012A
:106250000E94D968DF91CF911F910F91FF90EF902D
:10626000DF90CF9008959F92AF92BF92CF92DF922E
:10627000EF92FF920F931F93DF93CF93CDB7DEB7CB
:10628000C35AD1400FB6F894DEBF0FBECDBF809188
:106290002B02882311F40C94E43C10922B02809181
:1062A000222F882309F471C08CE89FE260E040E06F
:1062B0000E94255B8CE89FE263E974E00E94A3647E
:1062C0008CE89FE260E041E00E94255B0E94282F5D
:1062D0008CE89FE262E041E00E94255B8CE89FE24F
:1062E00061E974E00E94A3648CE89FE265E041E00C
:1062F0000E94255B87E00E94732F8CE89FE26EE08E
:1063000041E00E94255B8CE89FE26FE874E00E9408
:10631000A3642091A30940919E2E203171F4242F73
:1063200030E086E299E0289FF001299FF00D389F28
:10633000F00D1124E35FFC4E19C030E050E084E81A
:1063400090E0289FF001299FF00D389FF00D112457
:1063500086E299E09C01429FC001439F900D529FAD
:10636000900D1124E80FF91FE85BF44F60816C5F1A
:106370008CE89FE241E00E94255B8CE89FE26BED98
:106380000E94C6648BE090E078C08091212F882322
:1063900009F479C08CE89FE260E040E00E94255B50
:1063A0008091340990913509029729F48CE89FE295
:1063B0006EE774E004C08CE89FE26DE674E00E9432
:1063C000A3648CE89FE260E041E00E94255B0E94AC
:1063D000282F8CE89FE263E041E00E94255B20913A
:1063E000A30940919E2EDE01AF56BE4F2031B9F475
:1063F000242F30E086E299E0289FF001299FF00DDC
:10640000389FF00D1124E25FFC4E8081E82FF0E010
:10641000EE0FFF1FE357FD4F6591749122C030E0EE
:1064200050E084E890E0289FF001299FF00D389F0C
:10643000F00D112486E299E09C01429FC001439F28
:10644000900D529F900D1124E80FF91FE95BF44F56
:106450008081E82FF0E0EE0FFF1FE357FD4F6591BD
:106460007491CD010E94FE048CE89FE2BE016F563C
:106470007E4F0E94CB658AE090E09093A1098093C3
:10648000A0090C94E43C8091340990913509863040
:10649000910509F431C68730910574F48530910572
:1064A00014F00C94A03C833091050CF004C20297C8
:1064B00011F00C94E43CF0C08830910569F088300C
:1064C00091050CF415C48930910509F457C70C9750
:1064D00011F00C94E43C7EC38091A0099091A10935
:1064E0000897A9F088E39FE263E071E00E941368D7
:1064F000BC0181E39FE20E94D968BC018AE29FE26D
:106500000E94D968BC0183E29FE20E94D968809111
:106510001E2F813011F00C94E43C8091A0099091E1
:10652000A109089761F480915C01813041F4809168
:106530002C02882321F480911C2F8823D1F188E03C
:1065400090E09093A1098093A00980911E2F8093E1
:106550005C0110922C0210921C2F8CE89FE260E0EC
:1065600040E00E94255B8CE89FE26CE574E00E94AD
:10657000A36480911D2FE82FF0E0EE0FFF1FEB5B6F
:10658000FD4F659174918E010F5F1F4FC8010E94EE
:10659000FE04E0911D2FF0E0E35DFD4F8CE89FE2EB
:1065A000608140E00E94255B8CE89FE2B8010E9478
:1065B000CB6580912909E82FF0E0EE0FFF1FE9512C
:1065C000FD4F659174918E010F5F1F4FC8010E94AE
:1065D000FE0480912D09E82FF0E0EE0FFF1FE75237
:1065E000FD4F6591749185E0E82EF12CEC0EFD1EB7
:1065F000C7010E94FE048FE39FE2B8010E94136866
:106600008E01075F1F4F6091300970913109C801F9
:106610004AE00E942C6886E49FE2B8010E94D96893
:10662000C8010E9406698E01005F1F4FC80160917A
:1066300037094AE00E948E688DE49FE2B8010E940B
:10664000D968C8010E94066984E59FE2B7010E94EB
:10665000136817E1A12EB12CAC0EBD1EC5016FE36E
:106660007FE20E94F068BEE1CB2ED12CCC0EDD1E65
:10667000C60166E47FE20E94F068A5E2EA2EF12CF2
:10668000EC0EFD1EC7016DE47FE20E94F0688E01F2
:10669000045D1F4F0C94883C8CE89FE260E040E072
:1066A0000E94255B80911F2F882309F445C08CE848
:1066B0009FE26BE474E00E94A3648CE89FE260E0D8
:1066C00041E00E94255B0E94282F8CE89FE264E055
:1066D00041E00E94255BE091A309F0E0EC54F14D0C
:1066E000608170E06F5F7F4F8CE89FE24AE050E08E
:1066F0000E94B8658CE89FE26BE041E00E94255B58
:1067000080919E2E90E026E239E0829FF001839FE7
:10671000F00D929FF00D1124E555F54F608170E06A
:106720006F5F7F4F8CE89FE24AE050E00E94B865BF
:1067300081E08093202F77C08091A0099091A109DA
:10674000029749F48091202F882329F480911C2FEF
:10675000882309F468C082E090E09093A1098093B7
:10676000A0091092202F10921C2F8CE89FE26AE360
:1067700074E00E94A3648CE89FE260E041E00E9424
:10678000255B0E94282F8CE89FE262E041E00E9496
:10679000255B6091A4096F5B8CE89FE20E94C66450
:1067A0006091A50970E06F5F7F4F8091A40990E030
:1067B000F4E0880F991FFA95E1F7681B790B8CE8D4
:1067C0009FE24AE050E00E94B8658091A50980935D
:1067D000A92F8CE89FE269E041E00E94255B8CE8EC
:1067E0009FE265E00E94F35A8CE89FE261E071E06D
:1067F0000E94CB6580912909882359F460912E0964
:1068000070912F098CE89FE24AE050E00E945565A4
:1068100006C08CE89FE266E374E00E94A364809166
:106820002E098093A82F9091A5098091A92F9817E0
:1068300019F182E00E94FB2E6091A4096F5B8CE845
:106840009FE20E94C6646091A50970E06F5F7F4F70
:106850008091A40990E0E4E0880F991FEA95E1F7A0
:10686000681B790B8CE89FE24AE050E00E94B86513
:106870008091A5098093A92F8091A82F90E0209165
:106880002E0930912F098217930711F40C94E43CE0
:106890008BE00E94FB2E60912E0970912F098CE8ED
:1068A0009FE24AE050E00E94556580912E09809356
:1068B000A82F0C94E43C8091A0099091A109039722
:1068C000C1F088E39FE263E071E00E941368BC01BD
:1068D00081E39FE20E94D968BC018AE29FE20E94A4
:1068E000D968BC0183E29FE20E94D96881E00E94DE
:1068F000E52F8091A0099091A109039741F480911F
:106900002C02882321F480911C2F882381F18CE8AC
:106910009FE260E040E00E94255B8CE89FE265E238
:1069200074E00E94A36480911D2FE82FF0E0EE0F29
:10693000FF1FEB57FD4F659174918E010F5F1F4F45
:10694000C8010E94FE04E0911D2FF0E0E35DFD4FC1
:106950008CE89FE2608140E00E94255B8CE89FE22A
:10696000B8010E94CB6510922C0210921C2F8E0150
:106970000D5C1F4FE091A309F0E0EB53F14D6081F6
:1069800070E06F5F7F4FC8014AE00E945D68CE01F2
:10699000CA96B8010E94FB688091D62E882311F414
:1069A00060E201C06EE74AE3C42ED12CCC0EDD1E9E
:1069B000C6010E9497678C0131E4E32EF12CEC0EA6
:1069C000FD1EE091A309F0E0EC54F14D608170E010
:1069D0006F5F7F4FC7014AE00E945D68C801B70141
:1069E0000E94A867BC018E01085B1F4FC8010E946E
:1069F000F0688FE39FE2B8010E94D968C8010E9445
:106A00000669C7010E940669C6010E940C69CE0191
:106A1000C3960E9406692091A30940919E2E2031C1
:106A200071F4242F30E086E299E0289FF001299F3D
:106A3000F00D389FF00D1124E45FFC4E19C030E0DA
:106A400050E084E890E0289FF001299FF00D389FE6
:106A5000F00D112486E299E09C01429FC001439F02
:106A6000900D529F900D1124E80FF91FEB5BF44F2E
:106A70008081682F70E06F5F7F4F8E01015B1F4F39
:106A8000C8014AE00E945D6886E49FE2B8010E9466
:106A9000D968C8010E9406698DE49FE260E070E059
:106AA0000E9413684091A309403189F48E010A5A6B
:106AB0001F4FC80165E071E00E94DF6784E59FE237
:106AC000B8010E94D968C8010E94066945C080913A
:106AD0009E2E90E026E239E0829FF001839FF00D28
:106AE000929FF00D1124E555F54FE40FF11D8781BC
:106AF000882311F460E201C06BE224E6C22ED12C9F
:106B0000CC0EDD1EC6010E94C0689DE5E92EF12C69
:106B1000EC0EFD1E6091A30970E06F5F7F4FC7010F
:106B20004AE00E945D68C601B7010E94A867BC01E7
:106B30008E0105591F4FC8010E94F06884E59FE24D
:106B4000B8010E94D968C8010E940669C7010E9465
:106B50000669C6010E940C6982E7A82EB12CAC0E12
:106B6000BD1EC5016FE37FE20E94F06809E7C02EF9
:106B7000D12CCC0EDD1EC60166E47FE20E94F068D7
:106B800010E8E12EF12CEC0EFD1EC7016DE47FE252
:106B90000E94F0688E0109571F4FC80164E57FE22B
:106BA0000E94F068C501B601A70198010E947230E9
:106BB000C8010E940669C7010E940669C6010E94B9
:106BC0000669C5010E94066980E00E94E52F83E006
:106BD00090E053CC8091A0099091A1090C9721F4E9
:106BE00080911C2F8823B1F18CE89FE260E040E0A7
:106BF0000E94255B0E94282F8CE89FE262E040E023
:106C00000E94255B8CE89FE260E274E00E94A3642E
:106C10008CE89FE260E041E00E94255B0E94282F03
:106C20008CE89FE262E041E00E94255B8CE89FE2F5
:106C30006DE174E00E94A364E091892FF0E0EA5CCA
:106C4000FD4F8CE89FE260814AE050E00E9466655B
:106C500010921C2F8E0102571F4FE091892FF0E0F8
:106C6000EA5CFD4FC80160814AE00E948E6883E2C1
:106C70009FE2B8010E94F966F82EC8010E940669D9
:106C8000FF2099F58CE89FE264E041E00E94255BDB
:106C90008CE89FE269E174E00E94A3648CE89FE2C3
:106CA00064E041E00E94255BE091892FF0E0EA5C1E
:106CB000FD4F8CE89FE260814AE050E00E946665EB
:106CC0008E010B561F4FE091892FF0E0EA5CFD4FDB
:106CD000C80160814AE00E948E6883E29FE2B801A9
:106CE0000E94D968C8010E9406698CE090E0C5CB7B
:106CF0008091AA0A882321F0813009F0FAC1A1C14C
:106D00008091A0099091A109079721F480915C01DD
:106D10008823A9F088E39FE263E071E00E94136892
:106D2000BC0181E39FE20E94D968BC018AE29FE234
:106D30000E94D968BC0183E29FE20E94D9688091D9
:106D4000A0099091A109079771F49091AA0A8091E6
:106D50005C01981741F480912C02882321F48091E2
:106D60001C2F8823A1F18CE89FE260E040E00E94A4
:106D7000255B8CE89FE268E074E00E94A364809148
:106D80001D2FE82FF0E0EE0FFF1FEB59FD4F65912F
:106D900074918E010F5F1F4FC8010E94FE04E091A5
:106DA0001D2FF0E0E35DFD4F8CE89FE2608140E045
:106DB0000E94255B8CE89FE2B8010E94CB65809120
:106DC000AA0A80935C0110922C0210921C2F209131
:106DD0009E2E30E080913B0990E0FC01EE0FFF1FFA
:106DE000E80FF91F06E219E0209FD001219FB00DA6
:106DF000309FB00D1124EA0FFB1FEE5EFC4E208188
:106E00002F70A65FBC4E8C9190E0FC01EE0FFF1F2F
:106E1000E80FF91FEE0FFF1FEE0FFF1FE20FF11D2E
:106E2000E356FE4F8081E82FF0E0EE0FFF1FE550A4
:106E3000FD4F65917491CE0101960E94FE048091F0
:106E40003B0990E020919E2E30E0FC01EE0FFF1FE9
:106E5000E80FF91F209FC001219F900D309F900DDA
:106E60001124E80FF91FEE5EFC4E80818295877039
:106E7000E82FF0E0EE0FFF1FE351FD4F6591749195
:106E8000CE0105960E94FE048E0104561F4FE0912C
:106E9000A309F0E0EB53F14D608170E06F5F7F4F2D
:106EA000C8014AE00E945D68CE018D559F4FB80130
:106EB0000E94FB688091D62E882311F460E201C005
:106EC0006EE793EAC92ED12CCC0EDD1EC6010E94BE
:106ED00097678C018AEAE82EF12CEC0EFD1EE091FA
:106EE000A309F0E0EC54F14D608170E06F5F7F4FDB
:106EF000C7014AE00E945D68C801B7010E94A86707
:106F0000BC018E010F541F4FC8010E94F0688FE32F
:106F10009FE2B8010E94D968C8010E940669C701B2
:106F20000E940669C6010E940C69CE0184569F4FDB
:106F30000E9406698E0108541F4FC801BE016F5F91
:106F40007F4F0E94DF6786E49FE2B8010E94D96804
:106F5000C8010E9406698E0101541F4FC801BE017D
:106F60006B5F7F4F0E94DF678DE49FE2B8010E9454
:106F7000D968C8010E9406698E010A531F4F80918B
:106F80003B0990E020919E2E30E0FC01EE0FFF1FA8
:106F9000E80FF91F86E299E0AC01249FC001259F0C
:106FA000900D349F900D1124E80FF91FE05FFC4E07
:106FB000608166956F71C80170E04AE00E942C689C
:106FC00084E59FE2B8010E94D968C8010E94066961
:106FD000ADECAA2EB12CAC0EBD1EC5016FE37FE255
:106FE0000E94F068F4EDCF2ED12CCC0EDD1EC60130
:106FF00066E47FE20E94F068EBEDEE2EF12CEC0EE1
:10700000FD1EC7016DE47FE20E94F0688E010E5103
:107010001F4FC80164E57FE20E94F068C501B60118
:10702000A70198010E947230C8010E940669C70139
:107030000E940669C6010E940669C5010E94066990
:1070400058C08091A0099091A109079741F48091BF
:107050005C01813021F480911C2F8823C1F08CE8E1
:107060009FE260E040E00E94255B8CE89FE260E0E8
:1070700040E00E94255B8CE89FE267EF73E00E948E
:10708000A3648091AA0A80935C0110921C2F109235
:107090001D2F8CE89FE260E041E00E94255B0E948A
:1070A000282F8CE89FE262E041E00E94255B8091FE
:1070B0009E2E90E026E239E0829FF001839FF00D42
:1070C000929FF00D1124E65FFC4E8081E82FF0E0E6
:1070D000EE0FFF1FEB56FD4F659174918E01065622
:1070E0001E4FC8010E94FE048CE89FE2B8010E9476
:1070F000CB6587E090E0C1C98091A0099091A1097A
:107100000697A9F088E39FE263E071E00E941368AC
:10711000BC0181E39FE20E94D968BC018AE29FE240
:107120000E94D968BC0183E29FE20E94D968E09185
:107130000E2FF0E0E052F14D92898091A72F981721
:1071400071F081E39FE263E071E00E941368E091D7
:107150000E2FF0E0E052F14D82898093A72F8091AD
:10716000A0099091A109069741F480912C028823EF
:1071700021F480911C2F8823B1F18CE89FE260E01C
:1071800040E00E94255B8CE89FE266EE73E00E947F
:10719000A36480911D2FE82FF0E0EE0FFF1FE35A4C
:1071A000FD4F659174918E010F5F1F4FC8010E94C2
:1071B000FE04E0911D2FF0E0E35DFD4F8CE89FE2BF
:1071C000608140E00E94255B8CE89FE2B8010E944C
:1071D000CB6586E090E09093A1098093A00910927E
:1071E0002C0210921C2FE0910E2FF0E0E052F14D96
:1071F0008081E82FF0E0EE0FFF1FEF54FD4F659107
:1072000074917E010894E11CF11CC7010E94FE04E8
:107210008E0107511F4F60910E2F70E06F5F7F4FFF
:10722000C8014AE00E945D688FE39FE2B8010E94B6
:10723000D968C8010E9406698E0100511F4FC8011C
:10724000B7010E94DF6786E49FE2B8010E94D96817
:10725000C8010E94066980910E2FE82FF0E0E052ED
:10726000F14D82899E0129503F4F882331F0C90199
:1072700060E070E00E94DF6708C0628170E06F5FCD
:107280007F4FC9014AE00E945D688E0109501F4F7F
:107290008DE49FE2B8010E94D968C8010E94066986
:1072A0008E0102501F4FE0910E2FF0E0EE0FFF1FF6
:1072B000EE0FFF1FEC51F14D60817181828193814E
:1072C00020E030E048EC52E40E94C56A0E94E36985
:1072D0009B01AC01C801622F4AE00E948E6884E5E0
:1072E0009FE2B8010E94D968C8010E94066935E092
:1072F000A32E31E0B32EAC0EBD1EC5016FE37FE2BD
:107300000E94F0682CE0C22E21E0D22ECC0EDD1EB1
:10731000C60166E47FE20E94F06893E1E92E91E005
:10732000F92EEC0EFD1EC7016DE47FE20E94F068AD
:107330008E01065E1E4FC80164E57FE20E94F06880
:10734000C501B601A70198010E947230C8010E94D0
:107350000669C7010E940669C6010E940669C50147
:107360000E940669E0910E2FF0E0E052F14D828913
:10737000882309F429C30E948A2F26C38091A0097B
:107380009091A1090997A9F088E39FE263E071E079
:107390000E941368BC0181E39FE20E94D968BC018E
:1073A0008AE29FE20E94D968BC0183E29FE20E94C8
:1073B000D9688CE89FE260E040E00E94255B809104
:1073C000A3092091A0093091A109803109F044C09E
:1073D0002930310569F480912C02882349F4809189
:1073E000A62F803129F480911C2F882309F475C0C1
:1073F0008CE89FE265ED73E00E94A36480911D2FED
:10740000E82FF0E0EE0FFF1FE358FD4F65917491F8
:107410008E010F5F1F4FC8010E94FE04E0911D2FD7
:10742000F0E0E35DFD4F8CE89FE2608140E00E9468
:10743000255B8CE89FE2B8010E94CB6589E090E073
:107440009093A1098093A00910921C2F10922C02F6
:1074500080E18093A62F41C02930310561F48091ED
:107460002C02882341F48091A62F803121F0809155
:107470001C2F882391F18CE89FE264EC73E00E945A
:10748000A36480911D2FE82FF0E0EE0FFF1FEB5853
:10749000FD4F659174918E010F5F1F4FC8010E94CF
:1074A000FE04E0911D2FF0E0E35DFD4F8CE89FE2CC
:1074B000608140E00E94255B8CE89FE2B8010E9459
:1074C000CB6589E090E09093A1098093A009109288
:1074D0001C2F10922C021092A62F80919E2EA82F66
:1074E000B0E06091A30980913B09282F30E083E947
:1074F00094E0A89FA001A99F500DB89F500D1124A2
:10750000862F90E0FC0116E0EE0FFF1F1A95E1F7C1
:10751000880F991FE80FF91FE40FF51FE20FF31F03
:10752000EE0FFF1FEA53F54F908096949694969431
:10753000603161F5F901EE0FFF1FE20FF31F86E2E4
:1075400099E09C01A29FC001A39F900DB29F900D56
:107550001124E80FF91FDF01A05FBC4E9C919295AA
:1075600096959695937011968C918770880F880FD9
:10757000892BA82EBB2440EF5FEFA40EB51EEF5E53
:10758000FC4EC080C694C694C6943DC0862F90E041
:10759000FC01A6E0EE0FFF1FAA95E1F7880F991FE7
:1075A000E80FF91FE40FF51FE20FF31FEE0FFF1FA7
:1075B000EB53F54F908192959695969593708181B6
:1075C0008770880F880F892BA82EBB2480EF9FEF30
:1075D000A80EB91E862F90E0FC0106E0EE0FFF1FFB
:1075E0000A95E1F7880F991FE80FF91FE40FF51FBF
:1075F000E20FF31FEE0FFF1FEB53F54FC080C69451
:10760000C6949FE0C9222AE02C1590F4EC2DF0E0FE
:10761000EE0FFF1FEF56FD4F659174918E010F5FC6
:107620001F4FC8010E94FE048DE49FE2B80106C00E
:10763000CC2039F48DE49FE268E071E00E94136889
:107640003DC038E0C31629F48DE49FE26CE071E0A0
:10765000F5CF49E0C41629F48DE49FE260E171E0C2
:10766000EDCF5AE0C51629F48DE49FE264E171E0A4
:10767000E5CFE8E2EE2EE1E0FE2EEC0EFD1EC701A6
:1076800068E171E00E94F9678E010F5D1E4F6C2D5D
:1076900070E06F5F7F4FC8014AE00E945D68C701DC
:1076A000B8010E94A867BC018DE49FE20E94D968DE
:1076B000C8010E940669C7010E940C698E01015D24
:1076C0001E4FE091A309F0E0EB53F14D608170E0B3
:1076D0006F5F7F4FC8014AE00E945D68CE018A5CFF
:1076E0009E4FB8010E94FB688091D62E882311F42A
:1076F00060E201C06EE776E3C72E71E0D72ECC0EB4
:10770000DD1EC6010E9497678C016DE3E62E61E0E5
:10771000F62EEC0EFD1EE091A309F0E0EC54F14DC5
:10772000608170E06F5F7F4FC7014AE00E945D6833
:10773000C801B7010E94A867BC018E010C5B1E4FF7
:10774000C8010E94F0688FE39FE2B8010E94D968E7
:10775000C8010E940669C7010E940669C6010E940D
:107760000C69CE01815D9E4F0E940669B7FC23C063
:1077700052E5E52E51E0F52EEC0EFD1EC7016BE142
:1077800071E00E94F9678E01055B1E4FC801B501CB
:107790004AE00E945D68C701B8010E94A867BC0169
:1077A00086E49FE20E94D968C8010E940669C70169
:1077B0000E940C6910C08E01075A1E4FC801B50106
:1077C0004AE00E945D6886E49FE2B8010E94D968A1
:1077D000C8010E9406698091A309803121F580913A
:1077E0003B0990E020919E2E30E0FC01EE0FFF1F40
:1077F000E80FF91F86E299E0AC01249FC001259FA4
:10780000900D349F900D1124E80FF91FE05FFC4E9E
:10781000608166956F71CE0182599E4F70E04AE09B
:107820000E942C680DC08EE6A82E81E0B82EAC0E0A
:10783000BD1E992041F4C50168E071E00E94DF6738
:10784000EE24FF2428C007E6E02E01E0F02EEC0E27
:10785000FD1EC7016DE171E00E94F9678E01005ABB
:107860001E4FE92DF0E0E15BFE4F608180E891E082
:1078700070E00E94676BC8014AE00E945D68C70122
:10788000B8010E94A867BC01C5010E94F068EE24FF
:10789000E394FF24F3948E0102591E4F84E59FE286
:1078A000B8010E94D968C8010E940669FF2029F02A
:1078B000CE01805A9E4F0E940669EE2029F0CE012B
:1078C00089599E4F0E940C6915E7A12E11E0B12E37
:1078D000AC0EBD1EC5016FE37FE20E94F068BCE7FD
:1078E000CB2EB1E0DB2ECC0EDD1EC60166E47FE2BE
:1078F0000E94F068A3E8EA2EA1E0FA2EEC0EFD1E2D
:10790000C7016DE47FE20E94F0688E0106571E4FAA
:10791000C80164E57FE20E94F068C501B601A701D5
:1079200098010E947230C8010E940669C7010E9436
:107930000669C6010E940669C5010E94066944C025
:1079400085E090E09093A1098093A0098CE89FE2E4
:1079500060E040E00E94255B8CE89FE263EB73E00F
:107960000E94A3648CE89FE260E041E00E94255BF6
:107970000E94282F8CE89FE262E041E00E94255B94
:107980008091F62E882329F08CE89FE26FEA73E05D
:1079900004C08CE89FE26CEA73E00E94A3648CE868
:1079A0009FE26AE041E00E94255B8091E50988231F
:1079B00029F08CE89FE268EA73E004C08CE89FE25B
:1079C00065EA73E00E94A364CD55DE4F0FB6F894CC
:1079D000DEBF0FBECDBFCF91DF911F910F91FF9002
:1079E000EF90DF90CF90BF90AF909F900895CF928F
:1079F000DF92EF92FF920F931F937B018C01E1EDD9
:107A0000CE2EE0E3DE2E980144275527205BC601E9
:107A1000622F0E94495C5527412F302F2F2DC60120
:107A2000622F0E94D55CC6016E2D0E94D55C1F910D
:107A30000F91FF90EF90DF90CF9008950F931F93D9
:107A400060E070EC84E090E00E94F73C01ED10E310
:107A5000C801609129090E94D55CC8016091300974
:107A60000E94D55CC80160912C090E94D55CC801B8
:107A700060912B090E94D55CC80160912D090E947C
:107A8000D55CC801609137090E94D55CC8010E948D
:107A9000185D6AE070E080E090E00E9411601F9144
:107AA0000F9108951F93CF93DF9380912A09882324
:107AB00071F110912909113099F0113018F012303C
:107AC00021F513C0809130099091310990932F09CD
:107AD00080932E090E94181D81E08093350215C005
:107AE0000E94181D1093350210C080E293E0A0E0C0
:107AF000B0E08093310290933202A0933302B093AE
:107B000034020E94181D1092350210922A098091A9
:107B10003309882351F08091AB08882331F00E940B
:107B20001E3D109233090E94142F809134099091C8
:107B30003509089711F01092330980912909823094
:107B400009F0E6C0C2EFDEE210E08881882309F484
:107B5000DAC02091310230913202409133025091CB
:107B60003402DA01C901825A9840A040B0408651DF
:107B70009340A040B04068F4CA01B9010E940F6A66
:107B80009B01AC010E94136929EC3EE84DE059E3EA
:107B9000A7C0DA01C90189519740A040B040895877
:107BA0009140A040B04068F4CA01B9010E940F6A38
:107BB0009B01AC010E94136928EA37EA4FE059E3C0
:107BC0008FC0DA01C901895E9540A040B040805362
:107BD0009140A040B04068F4CA01B9010E940F6A08
:107BE0009B01AC010E94136927E830EC41E159E3A5
:107BF00077C0DA01C90181519540A040B040883D6D
:107C00009105A105B10568F4CA01B9010E940F6A86
:107C10009B01AC010E94136925E432EF45E159E371
:107C20005FC0DA01C90189569440A040B040883A4B
:107C30009105A105B10568F4CA01B9010E940F6A56
:107C40009B01AC010E9413692CE531E948E159E33D
:107C500047C0DA01C901895A9340A040B040803C36
:107C60009105A105B10568F4CA01B9010E940F6A26
:107C70009B01AC010E94136922EE3CE34CE159E305
:107C80002FC0DA01C90189549340A040B04080362A
:107C90009105A105B10568F4CA01B9010E940F6AF6
:107CA0009B01AC010E94136920EA3EE640E259E3E1
:107CB00017C0DA01C901855F9140A040B0408455EA
:107CC0009140A040B040E0F4CA01B9010E940F6A9F
:107CD0009B01AC010E9413692EEE33E943E259E3A4
:107CE0000E94C56A9B01AC0160E070E080E792E40D
:107CF0000E947B690E94E36970932F0960932E09AB
:107D0000812F0E94FF0E1F5F2196123009F01DCFB8
:107D1000DF91CF911F9108953F924F925F926F92A2
:107D20007F928F929F92AF92BF92CF92DF92EF920B
:107D3000FF920F931F93DF93CF9300D000D000D01A
:107D4000CDB7DEB7062FC82EDD24EE24FF24603128
:107D500009F433C1262F30E040E050E029833A8314
:107D60004B835C83C701B60123E130E040E050E083
:107D70000E94286B29813A814B815C81620F731FBD
:107D8000841F951FE7E0660F771F881F991FEA95EC
:107D9000D1F70E94F73C3324402E552484E890E02C
:107DA000489E4001499E900C589E900C112452010F
:107DB000AA0CBB1CC20166E0880F991F6A95E1F707
:107DC000A80EB91E50C043E954E0249FF001259F3E
:107DD000F00D349FF00D1124EA0DFB1DE30DF11D94
:107DE000EE0FFF1FDF01AB53B54F2C91022F06950D
:107DF000017010E0000F111F822F869586958F70FD
:107E000090E0880F991F880F991F082B192B822F3C
:107E1000817090E0082B192B2295269526952370CA
:107E200011968C918770880F880F822B90E0B6E0B6
:107E3000880F991FBA95E1F7082B192BEA53F54FD4
:107E40008081887F8E831D828D819E81082B192BD6
:107E500081ED90E3602F0E94D55C81ED90E3612F6E
:107E60000E94D55C339480919E2E282F30E0E6E26C
:107E70006E2EE9E07E2E269DF001279DF00D369DA9
:107E8000F00D1124E80DF91DEB5BF44F8081831593
:107E900008F099CF81ED90E30E94185D6AE070E0F0
:107EA00080E090E00E941160C701B60120E839E04F
:107EB00040E050E00E94286B7B018C0120E038E01C
:107EC00040E050E0E20EF31E041F151F69817A8125
:107ED0008B819C8126E030E040E050E00E94286BDE
:107EE000E60EF71E081F191FC801B7010E94F73CD4
:107EF00081ED90E360E00E94D55C80919E2E90E041
:107F0000869DF001879DF00D969DF00D1124E80DE2
:107F1000F91DEB5BF44F81ED90E360810E94D55C2D
:107F200080919E2E90E0869DF001879DF00D969D9C
:107F3000F00D1124E80DF91DEA5BF44F81ED90E39B
:107F400060810E94D55C80919E2E90E0869DF0011C
:107F5000879DF00D969DF00D1124E80DF91DE85B4D
:107F6000F44F81ED90E360810E94D55C80919E2E5C
:107F700090E0869DF001879DF00D969DF00D1124F7
:107F8000E80DF91DE95BF44F81ED90E360810E94FB
:107F9000D55C80919E2E90E0869DF001879DF00D2E
:107FA000969DF00D1124E555F54FE40DF51D81ED7D
:107FB00090E367810E94D55CF6C0C701B60120E856
:107FC00039E040E050E00E94286B6B017C01605872
:107FD000774F8F4F9F4F0E94F73C80919E2E90E0ED
:107FE00006E219E0809FF001819FF00D909FF00D57
:107FF0001124E45FFC4E81ED90E360810E94D55C2A
:1080000080919E2E90E0809FF001819FF00D909FC7
:10801000F00D1124E55FFC4E81ED90E360810E943C
:10802000D55C80919E2E90E0809FF001819FF00DA5
:10803000909FF00D1124E35FFC4E81ED90E3608191
:108040000E94D55C80919E2E90E0809FF001819FE0
:10805000F00D909FF00D1124E25FFC4E81ED90E356
:1080600060810E94D55C80919E2E90E0809FF001FF
:10807000819FF00D909FF00D1124E65FFC4E81ED85
:1080800090E360810E94D55C00E076E2A72E79E063
:10809000B72E12C0802F90E0FC01EE0FFF1FE80FFB
:1080A000F91FE20FF31FEE5EFC4E60816F7781EDEA
:1080B00090E30E94D55C0F5F80919E2E90E08A9D98
:1080C00090018B9D300D9A9D300D1124F901E45FD4
:1080D000FC4E80810817F0F281ED90E30E94185D5C
:1080E0006AE070E080E090E00E941160C701B60194
:1080F0006050774F8F4F9F4F0E94F73CFF2456E20E
:10810000C52E59E0D52E3EC08F2D90E0FC01EE0F1C
:10811000FF1FE80FF91FE20FF31FDF01A05FBC4E46
:108120002C91022F06950F7110E0000F111F422FA6
:10813000429546954695437011968C918770880FAD
:10814000880F842B90E0A6E0880F991FAA95E1F78D
:10815000082B192B217030E0022B132BEF5EFC4E05
:108160008081F8EF9F2E982288240829192981ED13
:1081700090E3602F0E94D55C81ED90E3612F0E9417
:10818000D55CF39480919E2E90E08C9D90018D9D06
:10819000300D9C9D300D1124F901E45FFC4E80816F
:1081A0008F1508F0B1CF81ED90E30E94185D6AE071
:1081B00070E080E090E00E94116026960FB6F8947F
:1081C000DEBF0FBECDBFCF91DF911F910F91FF900A
:1081D000EF90DF90CF90BF90AF909F908F907F9067
:1081E0006F905F904F903F9008952F923F924F92E3
:1081F0005F927F928F929F92AF92BF92CF92DF92C7
:10820000EF92FF920F931F93DF93CF9300D000D094
:10821000CDB7DEB77724C8C0003109F43FC0C7012D
:10822000B6010E94F73C10E081ED90E362E00E940D
:10823000D55C81ED90E364E00E94D55C1F5F103453
:1082400099F781ED90E30E94185D6AE070E080E0AC
:1082500090E00E941160C501B4010E94F73C81EDDD
:1082600090E361E00E94D55C81ED90E36FE00E94B5
:10827000D55C81ED90E368E10E94D55C81ED90E3EF
:1082800061E00E94D55C81ED90E360E00E94D55CE6
:1082900081ED90E360E00E94D55C44C069817A8101
:1082A0008B819C810E94F73C81ED90E36FE00E94FE
:1082B000D55C81ED90E368E10E94D55C81ED90E3AF
:1082C00061E00E94D55C81ED90E360E00E94D55CA6
:1082D00081ED90E360E00E94D55C10E081ED90E3D9
:1082E00060E30E94D55C1F5F1034C1F781ED90E31D
:1082F0000E94185D6AE070E080E090E00E941160EA
:10830000C201B1010E94F73C10E081ED90E368E109
:108310000E94D55C81ED90E364E00E94D55C1F5F14
:10832000103499F781ED90E30E94185D6AE070E0E7
:1083300080E090E00E9411600F5F86E090E0A0E096
:10834000B0E0880E991EAA1EBB1E80E890E0A0E057
:10835000B0E0C80ED91EEA1EFB1E013109F05CCF49
:10836000272D26952695269581E090E0A0E0B0E0A7
:1083700004C0880F991FAA1FBB1F2A95D2F79C0122
:10838000AD018091BB2F9091BC2F822B932B9093AA
:10839000BC2F8093BB2F60E070E040E00E94940906
:1083A000739490E8791651F1672D70E080E090E0C9
:1083B00020E839E040E050E00E94286B6B017C012E
:1083C000812CA8E09A2EA12CB12C860E971EA81EF7
:1083D000B91EDC01CB018058974FAF4FBF4F898347
:1083E0009A83AB83BC83212CF9E03F2E412C512C86
:1083F0002C0C3D1C4E1C5F1C00E00ECF60E070ECAE
:1084000084E090E00E94F73C81ED90E360E00E9400
:10841000D55C81ED90E368E70E94D55C81ED90E347
:1084200061E00E94D55C81ED90E361E00E94D55C43
:1084300081ED90E361E00E94D55C81ED90E30E94C4
:10844000185D6AE070E080E090E00E94116081EDCC
:1084500090E367E570E00E94535C81ED90E36FEF7D
:108460000E94D55C81ED90E36DEF0E94D55C81EDBB
:1084700090E360E00E94D55C81ED90E361E00E94B2
:10848000D55C81ED90E363E00E94D55C81ED90E3E3
:108490000E94185D6AE070E080E090E00E94116048
:1084A0000F900F900F900F90CF91DF911F910F9130
:1084B000FF90EF90DF90CF90BF90AF909F908F9004
:1084C0007F905F904F903F902F90089560E070EC08
:1084D00084E090E00E94F73C81ED90E30E94185DFB
:1084E00081ED90E364E540E80E942D5D81ED90E32D
:1084F0000E94665C833008F082E08093290981ED58
:1085000090E30E94665C90E08E31910518F48EE154
:1085100090E005C08B3F910510F08AEF90E09093BA
:1085200031098093300981ED90E30E94665C8823D5
:1085300011F481E003C0813108F080E180932C09BF
:1085400081ED90E30E94665C882311F481E003C012
:10855000813108F080E180932B0981ED90E30E9446
:10856000665C843008F083E080932D0981ED90E310
:108570000E94665C823010F482E003C08B3008F009
:108580008AE08093370908951F930E9466421092F3
:108590003C0910924E0110924D0110921E2F83E063
:1085A00090E0909335098093340980E00E94BC608C
:1085B0000E948A6680916800816080936800D89AE2
:1085C00080916B00836080936B001092E50980912D
:1085D00030099091310990932F0980932E091091C1
:1085E0002909113059F0113018F0123081F40BC004
:1085F0000E94181D81E08093350209C00E94181D59
:108600001093350204C00E94181D1092350210927A
:108610002A0980913809882311F02C9A01C02C98DE
:108620001F9108952F923F924F925F926F927F9287
:108630008F929F92AF92BF92CF92DF92EF92FF9272
:108640000F931F93DF93CF93CDB7DEB7A0970FB6ED
:10865000F894DEBF0FBECDBF062F90E0A0E0B0E0E3
:10866000BC01CD0120E839E040E050E00E94286BD9
:108670005B016C01412C78E0572E612C712C4A0C67
:108680005B1C6C1C7D1CA60195012058374F4F4F79
:108690005F4F29873A874B875C87CA01AA27BB2788
:1086A000382F305B3E83D601C5018050974FAF4FC6
:1086B000BF4F8A839B83AC83BD83CD01AA27BB2791
:1086C000E82FE05BE98310E086E299E09C01029FDD
:1086D000C001039F900D129F900D112435E4832E4D
:1086E0003BE0932E880E991EAC014E54554F58878F
:1086F0004F83222433249A8B898B8555954FDC0137
:10870000AF59B74FBC8BAB8BFC01E05AF74FFE8BD8
:10871000ED8B9C012E59374F388F2F8BAC014D5963
:10872000574F5A8F498FDC01A15AB74FBC8FAB8F7F
:1087300083E994E0089FF001099FF00D189FF00D68
:108740001124FE8FED8FF0E12F16310409F4D4C00F
:10875000C301B2010E94F73C81ED90E30E94185DD5
:10876000930144275527205B81ED90E3622F46E07B
:108770000E942D5D81ED90E30E94665C81ED90E3A7
:108780000E94665CD4018C9381ED90E30E94665C4C
:10879000F401818381ED90E30E94665CD40113961D
:1087A0008C9381ED90E30E94665CF401828381EDFD
:1087B00090E30E94665CAF81B8858C93F401E08001
:1087C000FF240894E11CF11CEE0CFF1C0027F7FCB1
:1087D0000095102FC601B5010E94F73C81ED90E392
:1087E0000E94185D960144275527205B81ED90E398
:1087F000622F4E2D0E942D5DEE249101220F331F1A
:10880000C10116E0880F991F1A95E1F7280F391F4B
:108810004D8D5E8D240F351F38A32F8F67C081EDDE
:1088200090E30E94665C8C0181ED90E30E94665C9F
:108830008E871D86A80150708D859E85482B592BEB
:108840006E2D70E0EF8DF8A1E60FF71FEE0FFF1F02
:10885000EB53F54F242F217030813C7FCA01827089
:108860009070969587958170880F322B382BCA01AE
:108870008C73907096958795969587958F70282F15
:10888000220F220F337C322B3083882311F4337C68
:108890003083EF8DF8A1E60FF71FEE0FFF1FDF010A
:1088A000AB53B54FCA01807C977016E096958795BB
:1088B0001A95E1F7382F3295330F330F307C2C9116
:1088C0002F73232B2C9386958695877011962C9168
:1088D0001197287F282B11962C93EA53F54F952F4B
:1088E000987F80818770892B8083E394D4018C9159
:1088F0008E1508F094CFD4C069857A858B859C85C8
:108900000E94F73C81ED90E30E94185D81ED90E3B9
:108910006E8140E80E942D5D81ED90E30E94665CCF
:10892000EB89FC89808381ED90E30E94665CAD89D0
:10893000BE898C9381ED90E30E94665CEF89F88D8F
:10894000808381ED90E30E94665CA98DBA8D8C9343
:1089500081ED90E30E94665CEB8DFC8D8083893015
:1089600008F088E0AB8DBC8D8C9300E024C081EDD5
:1089700090E30E94665C202F30E0F901EE0FFF1FAC
:10898000E20FF31F29893A89E20FF31FEE5EFC4ED6
:1089900090819078282F30E02077307054E0359522
:1089A00027955A95E1F727702295207F8F70982B95
:1089B000922B90830F5FAB89BC89EC90E016B8F6E0
:1089C0006A817B818C819D810E94F73C81ED90E3DF
:1089D0000E94185D2E2D30E02F5F3F4F220F331F76
:1089E000442737FD4095542F81ED90E36981422F54
:1089F0000E942D5DEE244EC081ED90E30E94665CE6
:108A00008C0181ED90E30E94665C888B1F8610705C
:108A1000EF85F8890E2B1F2B8E2D90E0AC01440FB3
:108A2000551F480F591F29893A89420F531FFA01D0
:108A3000E05FFC4E702F7170C8018E739070969538
:108A400087958F71880F9801207C3770B6E0369536
:108A50002795BA95E1F7622F6295660F660F607CE5
:108A6000872B862B808326952695812F8695869544
:108A70008695FA01EF5EFC4E982F990F990F990F8A
:108A80002770292B2083815E8F71803110F0277031
:108A90002083E394AB89BC898C918E1508F0ACCF10
:108AA0000894211C311CE4E8F0E08E0E9F1E26E0A5
:108AB00030E040E050E0420E531E641E751E4F81B0
:108AC00058854F5F5F4F58874F8380E890E0A0E064
:108AD000B0E0A80EB91ECA1EDB1E91E129163104B2
:108AE00009F031CEA0960FB6F894DEBF0FBECDBF11
:108AF000CF91DF911F910F91FF90EF90DF90CF907A
:108B0000BF90AF909F908F907F906F905F904F90AD
:108B10003F902F9008954F925F926F927F928F9225
:108B20009F92AF92BF92CF92DF92EF92FF920F93FC
:108B30001F93CF93DF9381E00E94820590930209F7
:108B40008093010980919D09882379F080913409EF
:108B500090913509089749F483E090E090933509A6
:108B60008093340981E080932B02809134099091A5
:108B70003509059711F01092CA0880913409909137
:108B800035098430910531F00C9721F01092A2093B
:108B90001092DF2E8091802F882379F00E9403604D
:108BA0006093822F7093832F8093842F9093852FCF
:108BB00081E08093812F1092802F8091812F8823D4
:108BC000F1F080919D098823D1F00E9403602091EB
:108BD000822F3091832F4091842F5091852F621BDB
:108BE000730B840B950B6B3F71058105910538F074
:108BF00081E080937F2F109235021092812F809117
:108C00005E08882341F080919C08882321F480919C
:108C10003502882329F480917E2F882309F44DC0E2
:108C200021E020939D0910925B011092882F1092F1
:108C30007E2F10923C0981E090E0A0E0B0E08093AC
:108C4000732F9093742FA093752FB093762F2C9839
:108C50002C9A109238092093D92E109268081092FD
:108C60004E0110924D0180E090E0FC01E25BF64F76
:108C70001082FC01E653F64F1082FC01E955F64FD5
:108C80002083FC01E059F64F1082FC01E25AF04DBE
:108C90002083FC01EF57F64F208301968131910527
:108CA00021F78091F22E882311F01092EE2E809100
:108CB000F32E882311F01092EF2E8091882F8823B5
:108CC00041F080919D09882321F01092882F109205
:108CD000680880916508882341F080919C0888236A
:108CE00021F480913502882341F480915B2F882301
:108CF00021F480917F2F882339F15F981092DB094E
:108D0000109238091092A20910927F2F80915B2F48
:108D1000882311F010926808809168088F5F809313
:108D20006808813019F0823079F405C080935B01C6
:108D300010929D0909C010925B0181E080939D090A
:108D40001092680810923C0980919C088823E1F0F9
:108D50008091DC08882321F08091A3090E94F816F5
:108D60008091E308882321F08091A3090E941E19B5
:108D700080918108882309F4ABC08CE090E0909347
:108D8000350980933409A1C0809134099091350947
:108D90008230910569F48091DC08882311F00E94EB
:108DA00057168091E3088823D9F00E94A11618C0B5
:108DB0000397B1F48091DC08882341F08091A309E6
:108DC0000E9439138091A30980931D268091E308A6
:108DD000882331F08091A30960911D260E945A14C6
:108DE0008091F108882391F08091340990913509A0
:108DF000039719F083E090E002C082E090E0909346
:108E000035098093340981E080932B028091810899
:108E10008823E1F08091340990913509049719F085
:108E200084E090E002C083E090E090933509809365
:108E300034098091A309803121F481E08093DF2EF1
:108E400002C01092DF2E81E080932B028091C70830
:108E5000882331F18091CA088F5F8093CA088130DE
:108E600019F08230D1F40FC0809134099091350906
:108E700090939F0980939E0985E090E09093350937
:108E8000809334090AC080919E0990919F09909324
:108E90003509809334091092CA0881E080932B022F
:108EA0008091340990913509059711F01092CA0804
:108EB00080913409909135090797029710F010922C
:108EC0001E2F80919008882319F081E080932B0257
:108ED00080915E088823E9F080919C088823C9F07E
:108EE00080919D098823A9F488E090E0909335094A
:108EF0008093340980911E2F8F5F80931E2F8230C4
:108F000018F081E080931E2F10921D2F81E0809336
:108F10002B0280919608882321F081E08093222FF4
:108F200007C080919708882329F01092222F81E0B2
:108F300080932B0280918808882321F081E0809320
:108F4000212F07C080918908882329F01092212FB2
:108F500081E080932B022091340930913509C901B9
:108F60000397029768F02730310551F02930310519
:108F700039F02630310521F02C30310509F0F7C4E5
:108F80008091010990910209892B11F41092000936
:108F90008091A3088823F1F18091D508882369F096
:108FA00083E090E090933509809334090E9465082E
:108FB0008093A30981E080932B028091AB088823E2
:108FC00061F087E090E0909335098093340980E167
:108FD0008093A30981E080932B028091EA08882383
:108FE00061F083E090E0909335098093340980E14B
:108FF0008093A30981E080932B0280916C088823E1
:1090000049F086E090E0909335098093340981E03F
:1090100080932B0280916C088823E1F02091A309B2
:109020002031C1F48091A3088823A1F487E090E067
:10903000909335098093340980911B2F8093AA0A5D
:1090400091E090932B028F5F80931B2F823010F062
:1090500010921B2F8091340990913509079711F0D8
:1090600010921B2F8091EA08882389F0809134099F
:1090700090913509079759F410921B2F83E090E0E7
:10908000909335098093340981E080932B0280917D
:10909000F708882309F4B8C080919D09882309F452
:1090A000B3C0F090A30920919E2E40E1F41609F080
:1090B0003FC080914D0990E030E0FC01EE0FFF1FB2
:1090C000E80FF91F86E299E0B901689F9001699F56
:1090D000300D789F300D1124E20FF31FE05FFC4E3E
:1090E00080818E7F808380914D0990E0FC01EE0F9E
:1090F000FF1FE80FF91FE20FF31FDF01A05FBC4E57
:109100008C918E7F8C93EF5EFC4E80818770808384
:109110009C9111968C911197887F846011968C9305
:109120001197917098619C9381E08093A80A6CC01C
:109130004F2D50E08A01035C164FD801EC9130E0CE
:10914000DA01AA0FBB1FCA0166E0880F991F6A9552
:10915000E1F7A80FB91F83E994E0289FB001299F88
:10916000700D389F700D1124A60FB71FCD018E0F03
:10917000911DFC01EE0FFF1FEB53F54F80818E7F99
:109180008083F801208130E0A20FB31FAA0FBB1F1C
:10919000AB53B54F8C91837C8C938F2D90E0FC0169
:1091A000A6E0EE0FFF1FAA95E1F7880F991FE80FC1
:1091B000F91FE60FF71FE20FF31FEE0FFF1FEB5330
:1091C000F54F80818F7380838181887F8460818364
:1091D0008F2D90E0FC01B6E0EE0FFF1FBA95E1F78E
:1091E000880F991FE80FF91FE60FF71FE20FF31F13
:1091F000EE0FFF1FEA53F54F8081877080834E5535
:10920000514D81E0DA018C9380919C08882369F0AC
:109210008091F808882349F08091A309803119F0E2
:109220000E949D1502C00E9402168091B1088823F9
:1092300009F4FCC08091D508882309F4F7C0809117
:109240009C08882309F44DC000919E2E10E00E94D6
:10925000650826E239E0029FD001039FB00D129FFE
:10926000B00D1124A555B54FE091A309F0E0EC54E1
:10927000F14D90819295907F980F9C9320E030E083
:1092800064E870E046E259E011E080919E2E90E0A3
:10929000269FF001279FF00D369FF00D1124DC0171
:1092A000A49FC001A59F900DB49F900D1124E80FBD
:1092B000F91FEB5BF44FDC01A555B54F8C91808312
:1092C000F901EE55F14D10832F5F3F4F20313105ED
:1092D000E1F6FD01EF59F74F8C9180831093A80AB6
:1092E000A2C08091A30920919E2E8031E9F4022F23
:1092F00010E00E94650826E239E0029FD001039F3A
:10930000B00D129FB00D1124A45FBC4EE091A309D3
:10931000F0E0EC54F14D90819295907F980F9C93E2
:1093200081E08093A80A2BC0022F10E00E946508FC
:10933000A091A309B0E024E830E0A29FA001A39F80
:10934000500DB29F500D112426E239E0F9010E9F15
:1093500090010F9F300D1E9F300D1124420F531F9F
:109360004B5B544FFD01EC54F14D90819295907FF1
:10937000980FFA019083AE55B14D81E08C938091A6
:109380009E2E90E026E239E0829FF001839FF00D4F
:10939000929FF00D1124E555F54F108220E030E04A
:1093A00064E870E046E259E080919E2E90E0269FAE
:1093B000F001279FF00D369FF00D1124DC01A49FD2
:1093C000C001A59F900DB49F900D1124E80FF91FC7
:1093D000EB5BF44FE081DC01A555B54F8C918E1706
:1093E00018F4EC932093B32E2F5F3F4F20313105BB
:1093F000D9F680919E2E90E026E239E0829FF0011E
:10940000839FF00D929FF00D1124E555F54FEF5914
:10941000F74F9081E156F8408081891720F49083BE
:1094200080E18093B32E81E080932B0280919C0891
:10943000882309F45BC08091A408882309F456C0EE
:109440004091A3094E3009F451C04F3009F44EC089
:10945000403109F44BC080919E2E90E026E239E025
:10946000829FF001839FF00D929FF00D1124E5552E
:10947000F54FE40FF11D8781882369F1178240E0E1
:1094800050E063E974E020919E2E30E08091A309C2
:1094900090E0FC0116E0EE0FFF1F1A95E1F7880F30
:1094A000991FE80FF91F269FC001279F900D369F37
:1094B000900D1124E80FF91FE40FF51FEE0FFF1FA9
:1094C000EB53F54F8081826080834F5F5F4F403464
:1094D0005105C9F602C081E0878381E080932B02A9
:1094E000E091A309F0E0EE55F14D808380913409BD
:1094F000909135098330910539F08730910521F03D
:109500008930910509F077C08091D608882311F041
:10951000109200098091B1088823E9F48091A30892
:109520008823C9F480919C088823A9F48091340988
:1095300090913509039779F48091A309209101094D
:1095400030910209803121F4C9010E94F40603C060
:10955000C9010E94FA058091B108882311F5809114
:10956000A3088823F1F480919C088823D1F080918E
:10957000D5088823B1F089E090E090933509809375
:1095800034090E946508E091A309F0E0EC54F14D24
:1095900090819295907F980F90933B0981E0809302
:1095A0002B028091B108882309F0E1C18091A308C2
:1095B000882309F0DCC18091D508882309F4D7C13C
:1095C00080913409909135098930910519F00797F8
:1095D00009F0CDC10E946508E091A309F0E0EC54C8
:1095E000F14D90819295907F980F90933B0981E087
:1095F00080932B02BCC18430910509F035C1809164
:109600009D09882361F08091AB08882341F090E0A8
:109610008091A209882309F491E09093A209809196
:10962000F708882309F44EC0A091A30920919E2E2B
:10963000A031F1F480914D0990E030E0FC01EE0F93
:10964000FF1FE80FF91F86E299E0AC01249FC001DB
:10965000259F900D349F900D1124E80FF91FE05FB6
:10966000FC4E80818E7F808381E08093A80A2AC08F
:10967000B0E0FD01E35CF64F408130E0FD01EE0F0C
:10968000FF1FCD0156E0880F991F5A95E1F7E80FAB
:10969000F91F83E994E0BC01269FC001279F900D2C
:1096A000369F900D1124E80FF91FE40FF11DEE0F06
:1096B000FF1FEB53F54F80818E7F8083AE55B14DF8
:1096C00081E08C938091B108882351F48091A308A4
:1096D000882331F48091DF2E882389F00E94150DB4
:1096E00020E030E084E8482E512C06E2602E09E0AC
:1096F000702E13E9812E14E0912E01E056C00BE08C
:1097000017E0C0E0D0E0B1E0EB2EF12C8091010930
:10971000909102090C2E02C0969587950A94E2F763
:10972000982F9170D8019C9311968C91119798174E
:1097300089F112968C91882369F5913059F5C7010A
:109740000C2E02C0880F991F0A94E2F70E94D409D8
:1097500080ED97E00E946A6080E090E00E94D4096A
:1097600080919D098823B1F08091A209813091F404
:10977000FE01E15AF64F8081FE01A6E0EE0FFF1FC9
:10978000AA95E1F7E80FF11DEE0FFF1FE25EF94D1C
:10979000F182E082F801808181832196095F1F4F69
:1097A000C031D10509F0B2CF9BCFF901E25BF64F92
:1097B0008081882309F051C010E0249D5001259D2F
:1097C000B00C349DB00C1124790166E0EE0CFF1C46
:1097D0006A95E1F7B901660F771F6E0D7F1D42EAAA
:1097E000C42E4EE2D42EC20ED31E25C0412F50E00F
:1097F000D701A40FB51FAA0FBB1FA25EB94D8D9153
:109800009C911197892BB1F0C89DF001C99DF00D75
:10981000D89DF00D1124E60FF71FE40FF51FEE0F92
:10982000FF1FEB53F54F808183608083F601008337
:109830001D921C921F5F80919E2EC82FD0E0C69D66
:10984000F001C79DF00DD69DF00D1124EA0DFB1D12
:10985000EB5BF44F8081181748F22F5F3F4F2031A8
:10986000310509F0A2CF83C00C9709F080C0809128
:1098700001099091020990938B2F80938A2F8091F8
:109880009D09882309F473C08091AB08882341F0B7
:1098900090E08091A209882309F491E09093A209B5
:1098A0008091A209882309F462C0A0E0B0E003E936
:1098B00014E0FF24F39457E080918A2F90918B2F2E
:1098C0000A2E02C0969587950A94E2F780FF4AC057
:1098D000ED01C35CD64F488120919E2E30E0BD0142
:1098E000660F771FCD01E6E0880F991FEA95E1F733
:1098F000680F791F209FC001219F900D309F900D10
:109900001124680F791FFB01E40FF11DEE0FFF1FFB
:10991000EB53F54F8081816080839091892F99234B
:1099200091F08881FB01E80FF11DEE0FFF1FEA5354
:10993000F54F452F491B942F990F990F990F80814F
:109940008770892B0AC08881FB01E80FF11DEE0F9B
:10995000FF1FEA53F54F808187708083FD01EE552C
:10996000F14DF0821196A031B10509F0A5CF80919B
:10997000340990913509029709F01FC18091A3081D
:10998000882389F08091D508882369F083E090E0EE
:1099900090933509809334090E9465088093A30948
:1099A00081E080932B028091B108882309F455C08F
:1099B0008091D508882309F450C000919E2E10E0B4
:1099C0000E94650826E239E0029FD001039FB00D96
:1099D000129FB00D1124A555B54FE091A309F0E0F9
:1099E000EC54F14D90819295907F980F9C9320E0DC
:1099F00030E0C4E8D0E066E279E041E080919E2E5C
:109A000090E02C9FF0012D9FF00D3C9FF00D112454
:109A1000DC01A69FC001A79F900DB69F900D112459
:109A2000E80FF91FEB5BF44FDC01A555B54F8C91A6
:109A30008083E091A309F0E0EE55F14D40832F5F64
:109A40003F4F20313105D1F6FD01EF59F74F8C9191
:109A500080834093A80A40932B028091B208882308
:109A600021F081E080931F2F07C08091B3088823E5
:109A700029F010921F2F81E080932B028091F8082B
:109A8000882361F08091D408882341F09091A50942
:109A90008091A609981711F40E94EC168091D608BF
:109AA000882331F08091B108882311F410920009C5
:109AB0008091010990910209892B09F45AC0809183
:109AC000B108882309F055C08091CD088823C1F0E2
:109AD0000E946508873010F087E002C00E94650888
:109AE0008093A4098091A4098295807F2091A50983
:109AF000922F9F70890F8093A6092817B9F539C056
:109B00008091A3088823A9F50E9480088823B9F0D2
:109B10000E948008182F0E946508181B1093D72EEA
:109B20000E9465089091A4099295907F980F909358
:109B3000D82E9093A60981E0809300090FC08091F0
:109B40000009882369F40E9465089091A409929500
:109B5000907F980F9093A6091092D72E1092D92E2D
:109B60009091A5098091A609981719F081E080933A
:109B70009F2E8091C909882301F18091D72E8823D7
:109B8000E1F01092C9098091D92E9091D82E890FB9
:109B90008093A6099091A509981719F081E0809308
:109BA0009F2E8091D92E9091D72E8F5F8093D92EA2
:109BB0008150891710F01092D92E80919F2E882302
:109BC000B1F110929F2E81E080932B02E2EAFEE237
:109BD0001192BEE2E23BFB07D9F71092A12E109240
:109BE000A80A80919C08882369F08091A609609159
:109BF0009E2E0E9412438091A6098093A5090E947F
:109C0000241C11C060E080919E2E882309F461E03D
:109C10008091A6090E9412438091A6098093A5090C
:109C200081E08093A02E8091A5090E94AC2C8091A8
:109C3000A02E882381F080919D09882361F41092E1
:109C4000A02E90E080919E2E882309F491E09093BD
:109C50009E2E0E94241C8091AB088823B1F0809135
:109C6000A308882391F4C2EADEE210E08881882309
:109C700041F018828091A509612F0E948C3E0E94BC
:109C8000142F1F5F2196103189F78091A80A88232D
:109C9000B9F08091AB08882399F08091A3088823BC
:109CA00079F48091340990913509049749F0109224
:109CB000A80A8091A50960E10E948C3E0E94142FA1
:109CC00080910F2F8823A1F08091AB08882381F029
:109CD0008091A308882361F480913409909135091B
:109CE000049731F010920F2F8091A5090E94262C25
:109CF0008091AC08882319F081E080932B02809139
:109D0000340990913509059709F099C08091A3080D
:109D1000882309F05FC080910109909102090E9497
:109D2000C70780919C088823A9F18091C7088823E0
:109D300021F48091F808882339F01092DC2E1092DB
:109D4000DB2E1092F62E15C08091EA08882311F1BF
:109D50008091DD2E882381F08091E509882349F4E4
:109D60001092DC2E1092DB2E1092E5091092DD2E5F
:109D70000EC01092E5090BC01092E50981E08093B6
:109D8000DD2E8FEF9FEF9093DC2E8093DB2E81E012
:109D900080932B0280916C08882359F090E0809189
:109DA000F62E882309F491E09093F62E81E08093BB
:109DB0002B028091EA088823F1F080919C08882387
:109DC000D1F490E08091E509882309F491E0909323
:109DD000E5090EC08091D508882369F083E090E002
:109DE00090933509809334090E9465088093A309F4
:109DF00081E080932B028091C909882301F1809131
:109E0000D72E8823E1F01092C9098091D92E909124
:109E1000D82E890F8093A6099091A509981719F05B
:109E200081E080939F2E8091D92E9091D72E8F5FC5
:109E30008093D92E8150891710F01092D92EDF917E
:109E4000CF911F910F91FF90EF90DF90CF90BF9037
:109E5000AF909F908F907F906F905F904F900895FC
:109E600080919D09882311F410925B2F0E94012B91
:109E70000E94291D0E94410F0E94523D0E948B4565
:109E80000E9433310895AF92BF92CF92DF92EF924A
:109E9000FF920F931F938F3708F08FE700D000D009
:109EA000682F70E080E090E02AEF3FE040E050E073
:109EB000EDB7FEB7218332834383548320E030E043
:109EC00040E050E01FE7E12EF12C012D112DAA24D6
:109ED000BB2465010E9401667F7070694091102F5C
:109EE0003091112F2091C42F0F900F900F900F9051
:109EF000222381F0213051F48DB38093C62F9DB37E
:109F00008091C52F809589238DBB04C08FB7F894AD
:109F10008093C62F4CBD3DBD12987EBD00000DB490
:109F200007FEFDCF8EB56EBD00000DB407FEFDCF60
:109F30008EB5129A222339F08091C62F213011F468
:109F40008DBB01C08FBF1F910F91FF90EF90DF90ED
:109F5000CF90BF90AF900895EF92FF920F931F9311
:109F6000CF93DF938C01C8E0D0E093E9E92E94E031
:109F7000F92EC8010C2E02C0969587950A94E2F737
:109F800080FF37C0599AFE01E35CF64F4081209173
:109F90009E2E30E0FE01EE0FFF1FCE01B6E0880FCF
:109FA000991FBA95E1F7E80FF91F2E9DC0012F9D6B
:109FB000900D3E9D900D1124E80FF91FE40FF11D47
:109FC000EE0FFF1FEB53F54F808181FD02C084E14E
:109FD00001C08FE70E94434F82B18F71FE01E55EA1
:109FE000FD4F9081892B82B988E290E00E946A60DF
:109FF00059982196CC30D10509F0BBCF88E290E08A
:10A000000E946A60599AC0E0D0E073E9E72E74E0DC
:10A01000F72EC8010C2E02C0969587950A94E2F798
:10A0200080FF37C0149AFE01E35CF64F4081209117
:10A030009E2E30E0FE01EE0FFF1FCE0156E0880F8E
:10A04000991F5A95E1F7E80FF91F2E9DC0012F9D2A
:10A05000900D3E9D900D1124E80FF91FE40FF11DA6
:10A06000EE0FFF1FEB53F54F808181FD02C084E1AD
:10A0700001C08FE70E94434F82B18F71FE01ED5DF9
:10A08000FD4F9081892B82B988E290E00E946A603E
:10A0900014982196C830D10509F0BBCF88E290E032
:10A0A0000E946A60149ADF91CF911F910F91FF90E7
:10A0B000EF9008952F923F924F925F926F927F920E
:10A0C0008F929F92AF92BF92CF92DF92EF92FF92C8
:10A0D0000F931F93DF93CF9300D000D000D0CDB764
:10A0E000DEB78091DB09882361F18091A70A88237C
:10A0F00041F54091A60A80914D0950E090E02091F1
:10A100009E2E30E0FC01EE0FFF1FE80FF91F86E2E4
:10A1100099E0BC01269FC001279F900D369F900DAE
:10A120001124E80FF91FE05FFC4E808186958F7146
:10A1300090E0481759072CF05F981092DB091092B5
:10A14000A60A80910C0990E0882309F491E090938D
:10A150000C0980913C0960E30E94476B992339F414
:10A1600080912901882309F491E09093290180913D
:10A170003C096CE00E94476B992371F4E091A309BC
:10A18000F0E0E65DFE4F108210929509109294095E
:10A19000109297091092960980919D09882309F4DD
:10A1A000DCC5EEEEFEE28481882319F186818330DE
:10A1B00081F0843028F4813081F08230D1F405C000
:10A1C000843059F08530A9F40CC080919C0981300D
:10A1D00081F480913C0960E307C080913C0960E60E
:10A1E00003C080913C0968E10E94476B992309F400
:10A1F000108231967EE2E03FF707A9F680912909A7
:10A20000823028F580912D09813059F0813028F075
:10A21000823059F08330D9F40CC080913C0960E65B
:10A220000BC080913C0960E307C080913C0968E164
:10A2300003C080913C096CE00E94476B992339F47C
:10A2400080913809882309F491E09093380910929D
:10A250009309109292091092A90A8EE59FE29A83BF
:10A260008983A5ECBEE2BC83AB8307EA802E09E0BC
:10A27000902E18EBA12E19E0B12E1C0100E010E089
:10A28000B1E04B2E512C612C712CD02E20919E2EA2
:10A29000B0E10B1791F4822F90E026E239E0829F23
:10A2A000F001839FF00D929FF00D1124E555F54FBD
:10A2B000E05AF74FC190F0801DC0822F90E044E833
:10A2C00050E0049FF001059FF00D149FF00D112444
:10A2D000BC01A6E2B9E06A9FC0016B9F900D7A9F16
:10A2E000900D1124E80FF91FE555F54FE556FF4F86
:10A2F000C080F2903296E08080913C099C2D96952A
:10A30000292F30E090E06C2D70E00E94536B821793
:10A31000930729F4F801EF57F64FB1E0B08380912D
:10A320003C0990E06C2D70E00E94536B82179307FC
:10A3300009F060C0F801E059F64F80818F5F80839B
:10A340008081F81608F41082E1E0EE1679F0EE163E
:10A3500040F0F2E0EF16B1F023E0E21609F04AC057
:10A3600037C0F801E059F64F808107C0F801E05985
:10A37000F64F80813F2D381B832FF801E15AF64FAD
:10A38000808338C0F801E15AF64F80818F1509F0BB
:10A390003BC5D5018C91813009F036C51C9206C0B1
:10A3A000F5018081882311F421E02083D5018C916F
:10A3B000F801E059F64FD801A15AB64F882311F0A1
:10A3C000808104C08081EF2DE81B8E2F8C9312C0FA
:10A3D0002F2D30E02F5F3F4F442737FD4095542FFE
:10A3E00060E070E080E090E00E946C66F801E15A65
:10A3F000F64F608320919E2E4F2D50E0F0E1DF1646
:10A4000091F530E080914D0990E0841795071CF09C
:10A4100080E090E004C080914D0990E00196FC013D
:10A42000EE0FFF1FE80FF91F46E259E0249FD0010D
:10A43000259FB00D349FB00D1124EA0FFB1FE05F84
:10A44000FC4E908192959695969593708181877038
:10A45000880F880F892B482F50E040515040A35F50
:10A46000BC4EAC9152C030E0F801E35CF64F808105
:10A4700090E0841795071CF040E050E005C0808113
:10A48000482F50E04F5F5F4FF801EE0FFF1FC801EC
:10A4900066E0880F991F6A95E1F7E80FF91F63E9F5
:10A4A00074E0269FC001279F900D369F900D1124C8
:10A4B000E80FF91FE40FF51FEE0FFF1FEB53F54FE9
:10A4C0009081929596959695937081818770880F6B
:10A4D000880F892B482F50E04051504084E890E08D
:10A4E000089FF001099FF00D189FF00D1124A6E2BE
:10A4F000B9E02A9FC0012B9F900D3A9F900D112427
:10A50000E80FF91FE85BF44FA081A15020913C09AE
:10A51000F801E653F64FFE83ED838081EA2FF0E0E9
:10A52000EE0FFF1FE80FF11DEE0FFF1FE35AFE4F66
:10A5300080819181820F911D841B950B6C2D70E0A1
:10A540000E94676B892B09F02CC2F801EF57F64F78
:10A550008081882309F425C21082AD81BE818C914F
:10A5600090E0882309F491E0F801E653F64F9083D8
:10A57000F801E65DFE4FB1E0B083EB1691F0EB160B
:10A5800040F0E2E0EE16B1F0F3E0EF1609F049C05A
:10A5900036C0F801E25BF64F8081F801E35CF64FCC
:10A5A00028C0F801E25BF64F8081F81AF801E35CFD
:10A5B000F64F23C0F801E35CF64F80818F1508F455
:10A5C0002BC4D4018C91813009F026C41C9206C0A2
:10A5D000F4018081882311F421E02083D4018C913F
:10A5E000F801E35CF64FD801A25BB64F882319F05F
:10A5F0008C91808316C08C91F81AF08212C02F2D96
:10A6000030E02F5F3F4F442737FD4095542F60E0E7
:10A6100070E080E090E00E946C66F801E35CF64F29
:10A62000608320919E2EF801E35CF64FB0E1DB16CB
:10A63000D1F4808190E030E0FC01EE0FFF1FE80FC5
:10A64000F91F46E259E0249FC001259F900D349FD9
:10A65000900D1124E80FF91FEF5EFC4E60816695A6
:10A660006695669522C0408130E0F801EE0FFF1F2D
:10A67000C80166E0880F991F6A95E1F7E80FF91F96
:10A6800063E974E0269FC001279F900D369F900DCF
:10A690001124E80FF91FE40FF11DEE0FFF1FEB531C
:10A6A000F54F6081669566956F70F801E35CF64F33
:10A6B000808182958F70AB81BC819C918917A9F0B4
:10A6C000908192959F709C938091D62E882321F043
:10A6D000F801EC54F14D9083809134099091350943
:10A6E000039719F4B1E0B0932B0220919E2EE0E184
:10A6F000DE16D9F480914D0990E030E0FC01EE0FB8
:10A70000FF1FE80FF91F46E259E0249FC001259F73
:10A71000900D349F900D1124E80FF91FE05FFC4E5F
:10A72000808181708093A90A36C0F801E35CF64FFE
:10A73000408130E0F801EE0FFF1FC801B6E0880F3E
:10A74000991FBA95E1F7E80FF91FA3E9B4E02A9F32
:10A75000C0012B9F900D3A9F900D1124E80FF91F17
:10A76000E40FF11DEE0FFF1FEB53F54F808180FFCB
:10A7700012C0209192093091930981E090E0002E5F
:10A7800002C0880F991F0A94E2F7822B932B9093B3
:10A79000930980939209F801E25BF64F80818F5F05
:10A7A00080836B3008F4AAC0B0E1DB16B9F02091C9
:10A7B000920930919309D301C201002E04C0880F81
:10A7C000991FAA1FBB1F0A94D2F7809590958223E8
:10A7D0009323909393098093920902C01092A90A3F
:10A7E0006D3091F16E3030F46B3059F06C3009F00F
:10A7F000D0C010C06E3009F440C06F3009F0C9C03D
:10A8000055C060E070E080E090E029E030E040E09A
:10A8100050E054C060E070E080E090E027E030E07D
:10A8200040E050E00E946C669B01AC016130710514
:10A830008105910509F0ADC060E1D61609F04BC065
:10A8400071E07093A90AA5C060E070E080E090E03C
:10A8500024E030E040E050E00E946C669B01AC01D7
:10A86000613071058105910509F093C080E1D8162A
:10A8700091F591E09093A90A8CC060E070E080E0CF
:10A8800090E023E030E040E050E00E946C669B01E5
:10A89000AC01613071058105910509F07AC0A0E134
:10A8A000DA16C9F4B1E0B093A90A73C060E070E0B1
:10A8B00080E090E022E030E040E050E00E946C66F2
:10A8C0009B01AC01613071058105910509F061C002
:10A8D000E0E1DE1679F08091920990919309002EC3
:10A8E00004C0220F331F441F551F0A94D2F7822B36
:10A8F000932B48C0F1E0F093A90A4BC0862F8150FA
:10A90000873058F470E06F5F7F4FD1018C9190E0F9
:10A910000E94676B892BE9F113C0683041F4F101A3
:10A92000808163E00E94476B992399F516C06930D6
:10A9300059F4D1018C9190E083709070892B49F586
:10A94000B0E1DB1669F423C06A3019F5F1018081AA
:10A9500090E087709070892BE1F4F0E1DF16B9F098
:10A960002091920930919309D301C201002E04C0B5
:10A97000880F991FAA1FBB1F0A94D2F78095909544
:10A9800082239323909393098093920902C010929B
:10A99000A90A8091920990919309909399098093C3
:10A9A000980920E1D21609F477C020919E2E30E05C
:10A9B000EDE3EE2EE9E0FE2EE00EF11ED7019C91B4
:10A9C00080913C09E3E9F4E02E9F60012F9FD00CB9
:10A9D0003E9FD00C11249801220F331FA80166E07E
:10A9E000440F551F6A95E1F7240F351FC20ED31E81
:10A9F000F601E90FF11DEE0FFF1FEA53F54FE0815D
:10AA0000E695E695E695F0E0E15BFE4FE08190E0AB
:10AA10006E2F70E00E94536B892BF1F5EE23E1F16C
:10AA20008091980990919909002E02C0969587957A
:10AA30000A94E2F780FF30C0D7018C91C80ED11C78
:10AA4000CC0CDD1CE5ECFAE0CE0EDF1ED6018C91BD
:10AA500080FF22C040919209509193092091920960
:10AA600030919309D301C201002E04C0880F991FB1
:10AA7000AA1FBB1F0A94D2F7282B392B30939309B6
:10AA8000209392098091920990919309842B952BA0
:10AA900090939309809392090F5F1F4F0894211C94
:10AAA000311CEB81FC813196FC83EB830894811C83
:10AAB000911C0894A11CB11C0131110509F0E5CBD2
:10AAC00080912909823038F480913809882311F067
:10AAD0002C9A01C02C988091A90A882309F459C0A6
:10AAE0008091E509882309F054C08091A70A882342
:10AAF00009F04FC020919E2E30E080914D09409189
:10AB00004D0990E0FC01EE0FFF1FE80FF91F86E2F0
:10AB100099E0289FB001299F700D389F700D112476
:10AB2000E60FF71FEE5EFC4E20812F70FB01E65F03
:10AB3000FC4E808190E0FC01EE0FFF1FE80FF91F33
:10AB4000EE0FFF1FEE0FFF1FE20FF11DE356FE4F4A
:10AB5000A081B0E0AA0FBB1FA958BE4F50E0FA0178
:10AB6000EE0FFF1FE40FF51FE60FF71FEE5EFC4E22
:10AB70002081269526952695922F9E7080E02D9116
:10AB80003C91820F931F0E943A0A5F9A81E0809362
:10AB9000DB098091920990919309892B39F1809179
:10ABA00092099091930990939509809394098091CB
:10ABB00094099091950990939709809396098091B3
:10ABC0009209909193090E94AC4F20919209309183
:10ABD00093098091DB2E9091DC2E809590958223B5
:10ABE00093230E94D40981E080933909E091B32E28
:10ABF000F0E0E25BF64F808190E090934E0180930D
:10AC00004D0170919E2E472F50E086E299E0489FBB
:10AC1000F001499FF00D589FF00D1124EB5BF44FAC
:10AC200020E030E061E0D901A25BB64F9C918081C9
:10AC3000891750F41C92A981BA818C918F5F8C93F3
:10AC40008150833D08F06C932F5F3F4FEC57FF4FCF
:10AC500089819A8101969A8389832031310519F778
:10AC600020915E0986E299E0489FF001499FF00D2E
:10AC7000589FF00D1124E45FFC4E8081821768F428
:10AC800010925E0980916E2F8F5F80936E2F81509E
:10AC9000833D18F081E080936E2F20914D0130911B
:10ACA0004E0186E299E0489FF001499FF00D589FC0
:10ACB000F00D1124E555F54F808190E08217930740
:10ACC0005CF51092BD2F81E08093DE2E10924E0134
:10ACD00010924D018091A02E8823F1F080913409CB
:10ACE000909135098230910511F00597A9F41092E1
:10ACF000A02E10929E2E772319F481E080939E2E31
:10AD00000E94241C80E090E0FC01E25BF64F108280
:10AD1000019681319105C1F740914D0150914E014D
:10AD200080919E2E90E026E239E0829FF001839F81
:10AD3000F00D929FF00D1124E555F54F808190E0C4
:10AD400001974817590749F48091BD2F882329F4AA
:10AD500081E08093C9098093BD2F20918A2F309183
:10AD60008B2F21153105A1F080913C09E091892FAD
:10AD7000F0E0E35CFD4F608190E070E00E94536B77
:10AD8000892B31F4C9010E94D40981E080933909EB
:10AD900080913C098F5F80933C098150803650F14F
:10ADA00081E080933C0980919C09823010F01092E0
:10ADB0009C098091F22E882351F080919C0981306A
:10ADC00031F48091F42E882311F41092EE2E8091AC
:10ADD000F32E882351F080919C09813031F48091C9
:10ADE000F52E882311F41092EF2E80919C098F5F2D
:10ADF00080939C098091DB098823B1F08091A60A99
:10AE00008F5F8093A60A10C0F801E15AF64F808147
:10AE1000882309F0CBCAC4CAF801E35CF64F8081ED
:10AE2000882309F0DBCBD4CB26960FB6F894DEBF8F
:10AE30000FBECDBFCF91DF911F910F91FF90EF908B
:10AE4000DF90CF90BF90AF909F908F907F906F904A
:10AE50005F904F903F902F90089580ED84B982EFDE
:10AE60008AB98CEF81B989E061E00E94DE6012B896
:10AE70005F980E94265A8FEF0E94045A81ED90E35A
:10AE80000E94315D08951F920F920FB60F920BB67C
:10AE90000F9211241F932F933F934F935F936F93C0
:10AEA0007F938F939F93AF93BF93EF93FF931091F3
:10AEB0002909113031F01130D8F0123009F002C1F7
:10AEC00070C08AEA93E30E942C63181619060CF0EE
:10AED000F9C08AEA93E30E945D63883F08F4F2C0F8
:10AEE000883F49F40E945A500E945A500E945A507A
:10AEF0000E945A50E7C08A3F09F04DC010939D0947
:10AF000010925B011092882F10923C0981E090E032
:10AF1000A0E0B0E08093732F9093742FA093752FCF
:10AF2000B093762F1093D92E2C982C9A1092380922
:10AF300010924E0110924D011092680880E090E04E
:10AF400021E0FC01E25BF64F1082FC01E653F64F74
:10AF50001082FC01E955F64F2083FC01E059F64FC1
:10AF60001082FC01EF57F64F2083FC01E25AF04DAE
:10AF7000208301968131910521F78091F22E88235B
:10AF800011F01092EE2E8091F32E882309F49AC0CE
:10AF90001092EF2E97C08C3F09F094C010935B2F56
:10AFA00091C080917D2F8823A1F11092732F109270
:10AFB000742F1092752F1092762F10927D2F809102
:10AFC0003C0980913C09883118F48CE080933C095D
:10AFD00080913C09883138F080913C09803318F425
:10AFE00084E280933C0980913C09803338F0809161
:10AFF0003C09883418F48CE380933C0980913C0927
:10B00000883438F080913C09803618F484E58093C8
:10B010003C0960913102709132028091330290912B
:10B02000340228E130E040E050E00E947A6B40E0DA
:10B0300050E08091732F9091742FA091752FB09153
:10B04000762F82179307A407B50740F01092732F4D
:10B050001092742F1092752F1092762F8091732F6B
:10B060009091742FA091752FB091762F0097A10524
:10B07000B10511F40E945A5080916F2F9091702F5A
:10B08000A091712FB091722F0196A11DB11D8093D7
:10B090006F2F9093702FA093712FB093722F809188
:10B0A000732F9091742FA091752FB091762F0196E8
:10B0B000A11DB11D8093732F9093742FA093752FB2
:10B0C000B093762FFF91EF91BF91AF919F918F91A8
:10B0D0007F916F915F914F913F912F911F910F90B1
:10B0E0000BBE0F900FBE0F901F901895FF920F93FD
:10B0F0001F938AEA93E342E15AE760E070E00E941E
:10B10000A6620E942D57E1E1F7E01082379687E0B2
:10B11000E138F807D1F7109268081092760810927B
:10B120007D0810926F081092CA0881ED90E367E5E0
:10B1300070E00E94535C81ED90E36FEF0E94D55C5C
:10B1400081ED90E36DEF0E94D55C81ED90E30E946C
:10B15000185D81ED90E367E570E043E050E00E9408
:10B16000295D81ED90E30E94665C082F81ED90E3FC
:10B170000E94665CF82E81ED90E30E94665C10E010
:10B180000F0D111D080F111D0430110531F00E9423
:10B19000512F0E94F5400E94F32B0E94D90A809102
:10B1A0005D2F843051F40E942F2F8FE70E94434F70
:10B1B00080E094E00E943A0AF8CF80915C2F8330BF
:10B1C00031F40E94512F0E94F5400E94F32B0E94FF
:10B1D000C44280916800816080936800D89A809111
:10B1E0006B00836080936B0080E060919E2E0E94D4
:10B1F00012430E94241C80E090E00E94D4090E9427
:10B2000057161092B1008091B1008093B0008091E8
:10B21000B00082608093B0008091B1008260809322
:10B22000B1008FE78093B3008091700082608093BB
:10B2300070000E94412D78948CE89FE260E044E821
:10B2400052E00E94FD5A8CE89FE261E04CE852E037
:10B250000E94FD5A8CE89FE262E044E952E00E94BD
:10B26000FD5A8CE89FE263E04CE952E00E94FD5AEF
:10B270008CE89FE264E044EA52E00E94FD5A8CE8C8
:10B280009FE265E04CEA52E00E94FD5A8CE89FE2A2
:10B2900060E142E020E00E94535B8CE89FE260E0C6
:10B2A0000E94F35A8CE89FE261E00E94F35A8CE816
:10B2B0009FE262E00E94F35A8CE89FE264E040E083
:10B2C0000E94255B8CE89FE264EC0E94C6648CE8D7
:10B2D0009FE26EED0E94C6648CE89FE267ED0E94DB
:10B2E000C6648CE89FE261ED0E94C6648CE89FE230
:10B2F00069E040E00E94255B8CE89FE26CEB0E94D5
:10B30000C6648CE89FE260EB0E94C6648CE89FE212
:10B3100069EB0E94C6648CE89FE26FEB0E94C664F2
:10B320008CE89FE26BEB0E94C6648CE89FE260EBC6
:10B330000E94C6648CE89FE260E041E00E94255BC9
:10B340008CE89FE263E00E94F35A8CE89FE264E09D
:10B350000E94F35A8CE89FE265E00E94F35A8CE861
:10B360009FE266E041E00E94255B8CE89FE264EA90
:10B3700074E00E94A36460ED77E080E090E00E94BA
:10B3800011608CE89FE260E044E452E00E94FD5AC4
:10B390008CE89FE261E04CE452E00E94FD5A8CE8A8
:10B3A0009FE262E044E552E00E94FD5A8CE89FE291
:10B3B00063E04CE552E00E94FD5A8CE89FE264E0B5
:10B3C00044E652E00E94FD5A8CE89FE265E04CE6BC
:10B3D00052E00E94FD5A8CE89FE266E044E752E0AA
:10B3E0000E94FD5A8CE89FE267E04CE752E00E9421
:10B3F000FD5A8CE89FE260E142E020E00E94535B4E
:10B400001F910F91FF900895982F8091C42F823043
:10B41000E0F42FB7F894913029F0913060F0923039
:10B4200029F402C092E008C094E006C082E0809354
:10B43000C42F2FBF089591E081E08093C42F8091A5
:10B44000C52F892B8093C52F2FBF089584E061E01D
:10B450000E94426184E061E00E94DE608CB5806100
:10B460008CBD8CB580648CBD87E061E00E94DE609D
:10B4700085E061E00E94DE6008950F931F938C01C8
:10B48000FC01868160E00E94426181E090E00E94C0
:10B490006A60F801868161E00E94426181E090E08B
:10B4A0000E946A60F801868160E00E94426184E641
:10B4B00090E00E946A601F910F910895CF92DF92F1
:10B4C000EF92FF920F931F93CF93DF93D82EC92E45
:10B4D000282F392FC9018C01C0E0D0E0E62EFF24CF
:10B4E000F801878161E00E94DE60B7010C2E02C086
:10B4F000759567950A94E2F76170F80187810E945B
:10B50000426121960F5F1F4FC830D10549F78D2D3D
:10B510009C2D0E943D5ADF91CF911F910F91FF907A
:10B52000EF90DF90CF900895CF92DF92EF92FF924D
:10B530000F931F93CF93DF93D82EC92E282F392F27
:10B54000C9018C01C0E0D0E0E62EFF24F80187811C
:10B5500061E00E94DE60B7010C2E02C07595679510
:10B560000A94E2F76170F80187810E944261219696
:10B570000F5F1F4FC430D10549F78D2D9C2D0E94C0
:10B580003D5ADF91CF911F910F91FF90EF90DF9087
:10B59000CF9008951F93CF93DF93EC01162F8C81EA
:10B5A000642F0E9442618D818F3F19F060E00E94FC
:10B5B00042618F8584FF05C0CE01612F0E945E5AD3
:10B5C0000EC0612F70E084E0759567958A95E1F76C
:10B5D000CE010E94945ACE01612F0E94945ADF91AD
:10B5E000CF911F91089541E00E94CA5A81E090E0F6
:10B5F000089540E00E94CA5A0895EF92FF920F9377
:10B600001F93CF93DF938C017A016770660F660FEB
:10B61000660F60640E94F95AC0E0D0E0D801ED9155
:10B62000FC91D701AC0FBD1F0190F081E02DC80146
:10B630006C9109952196C830D10581F7DF91CF91A2
:10B640001F910F91FF90EF900895DF93CF93CDB7A7
:10B65000DEB728970FB6F894DEBF0FBECDBF9C01B2
:10B66000FE013196AFECB6E088E00D90019281507A
:10B67000E1F7F9018389481708F040E0E42FF0E092
:10B68000EE0FFF1FEC0FFD1F8181680F6068C9017D
:10B690000E94F95A28960FB6F894DEBF0FBECDBFB0
:10B6A000CF91DF910895CF93DF93EC01423018F0F2
:10B6B0008F8588608F874B8B1C8A222329F041302D
:10B6C00019F48F8584608F8780E593EC0E946A600F
:10B6D0008C8160E00E9442618E8160E00E94426144
:10B6E0008D818F3F19F060E00E944261CE0163E0DE
:10B6F0000E94945A88E893E10E946A60CE0168E053
:10B700000E94945A88E893E10E946A60CE0162E048
:10B710000E94945A88E893E10E946A60CE0162E038
:10B720000E94945A88E893E10E946A60CE0168E022
:10B730000E94945A88E893E10E946A60CE0168E012
:10B740000E94F95A88E893E10E946A60CE0161E0A4
:10B750000E94F95A88E893E10E946A60CE0166E08F
:10B760000E94F95A88E893E10E946A60CE0162E083
:10B770000E94F95A88E893E10E946A60CE016CE069
:10B780000E94F95A88E893E10E946A60DF91CF91A4
:10B7900008956F927F928F92AF92CF92EF920F9314
:10B7A0001F93DF93CF93CDB7DEB73C01162F842FC5
:10B7B000F301448325830683E782C086A1868286BF
:10B7C0009D8593879E8594879F8595879889968781
:10B7D00061E00E94DE60F30185818F3F19F061E036
:10B7E0000E94DE60F301868161E00E94DE60112329
:10B7F00019F0F301178603C080E1F3018787C301C5
:10B8000060E141E020E00E94535BCF91DF911F9106
:10B810000F91EF90CF90AF908F907F906F900895A1
:10B820008F92AF92CF92EF920F931F93CF93DF93AC
:10B83000DC01362F542F722F102FAE2C8C2C139628
:10B840001C921E9212978BEC96E011969C938E930D
:10B8500000D000D0EDB7FEB73196CDB7DEB7198274
:10B86000118212821382CD0161E0432F2FEF052F49
:10B87000E72EC12E0E94C95B0F900F900F900F9082
:10B88000DF91CF911F910F91EF90CF90AF908F905C
:10B89000089581E08093D03060934B301092CE3089
:10B8A0001092CF30089581E08093D03060934B3078
:10B8B0001092CE301092CF30089520914A3030E06F
:10B8C00080914930281B3109C901089540914930C0
:10B8D00080914A30481718F02FEF3FEF0AC0E42F4D
:10B8E000F0E0E953F04D8081282F30E04F5F409326
:10B8F0004930C9010895E091493080914A30E817F4
:10B9000018F0EFEFFFEF06C0F0E0E953F04D808153
:10B91000E82FF0E0CF01089508951092D4301092EE
:10B92000D33088EE93E0A0E0B0E08093D5309093E0
:10B93000D630A093D730B093D8308BED96E090936B
:10B94000D2308093D1300895CF92DF92EF92FF9260
:10B950000F931F93CF93DF937C016B018A0180913A
:10B96000D0308823A1F0C0E0D0E00DC0D701ED9128
:10B97000FC91D601AC0FBD1F0190F081E02DC701F5
:10B980006C9109952196C017D10780F304C0CB01B3
:10B99000642F0E94DA5DC801DF91CF911F910F9152
:10B9A000FF90EF90DF90CF900895DF93CF930F92A9
:10B9B000CDB7DEB7FC0169838091D0308823C9F010
:10B9C0008091CF30823838F081E090E09383828399
:10B9D00020E030E015C08091CE30E82FF0E0E45B4D
:10B9E000FF4C998190838F5F8093CE308093CF30CE
:10B9F00005C0CE01019661E00E94DA5D21E030E0F1
:10BA0000C9010F90CF91DF9108950F93062F809178
:10BA10004B306CE470E34091CF3021E00E94855DB3
:10BA20001092CE301092CF301092D0300F910895F6
:10BA300061E00E94055D0895433808F042E8862FD2
:10BA400067EC7FE20E943C5D1092493080934A305F
:10BA5000089521E00E941C5D089521E00E941C5D74
:10BA600008951092493010924A301092CE301092C0
:10BA7000CF300E948A5F0895382F433810F040E09D
:10BA800042C08091DD308823E1F791E09093DD3072
:10BA90002093DF308FEF80937032109267314150E6
:10BAA000409368314F5F9093DE308091DE30330FEA
:10BAB000832B8093DE308091E030813041F410920E
:10BAC000E0308091DE308093BB0085EC01C085EED4
:10BAD0008093BC008091DD308130E1F3809167314B
:10BAE000841710F44091673120E030E00AC0FB0178
:10BAF000E20FF31FD901AB51BF4C8C9180832F5FB4
:10BB00003F4F2417A0F3842F08950F931F93582FAE
:10BB1000122F433810F081E04AC08091DD30882335
:10BB2000E1F782E08093DD300093DF308FEF809388
:10BB300070321092673140936831A5EEB0E3FB019B
:10BB400002C081918D938E2F861B8417D0F31092A3
:10BB5000DE308091DE30550F852B8093DE30809172
:10BB6000E030813041F41092E0308091DE308093FB
:10BB7000BB0085EC01C085EE8093BC00112321F051
:10BB80008091DD308230E1F3809170328F3F11F48B
:10BB900080E00DC080917032803211F482E007C0E5
:10BBA00080917032803311F084E001C083E01F91F6
:10BBB0000F910895482F633810F081E00895809127
:10BBC000DD30843011F082E008956093EC31A9E615
:10BBD000B1E3842F9C01F90102C081918D938E2FD6
:10BBE000841B8617D0F380E008951F920F920FB642
:10BBF0000F920BB60F9211242F933F934F935F93A5
:10BC00006F937F938F939F93AF93BF93EF93FF9324
:10BC10008091B90090E0887F90708036910509F49A
:10BC2000F2C081369105CCF58832910509F47BC0CC
:10BC300089329105B4F48031910509F46FC08131E6
:10BC400091053CF4009709F447C1089709F04FC1EA
:10BC500065C08831910509F466C0809709F047C135
:10BC600082C08034910509F4A4C08134910544F464
:10BC70008033910509F482C0C89709F038C189C0A2
:10BC80008035910509F489C08835910509F496C07D
:10BC90008834910509F02BC1AEC08839910509F4AB
:10BCA00013C189399105ECF48837910509F4ABC0CB
:10BCB000893791054CF48836910509F4A4C0803782
:10BCC000910509F014C19FC08838910509F4FCC0A2
:10BCD0008039910509F49DC08038910509F007C1AC
:10BCE00098C0803B910509F4C6C0813B91054CF496
:10BCF000803A910509F49FC0883A910509F0F7C090
:10BD0000BAC0803C910509F4E3C0883C910509F470
:10BD1000DFC0883B910509F0EAC0C2C08091DE30E7
:10BD20008093BB00CFC090916731809168319817A4
:10BD300068F490916731E92FF0E0EB51FF4C80817E
:10BD40008093BB009F5F90936731BCC08091DF30D0
:10BD5000882309F44BC085ED8093BC008091BC0022
:10BD600084FDFCCFC2C080E28093703285ED809369
:10BD7000BC008091BC0084FDFCCFB7C080E3809301
:10BD8000703285ED8093BC008091BC0084FDFCCFB7
:10BD9000ACC088E3809370329BC0809167319091F2
:10BDA000BB00E82FF0E0EB51FF4C90838F5F809356
:10BDB0006731909167318091683182C0809167319D
:10BDC0009091BB00E82FF0E0EB51FF4C90838F5F28
:10BDD000809367318091DF30882341F085ED809337
:10BDE000BC008091BC0084FDFCCF7FC081E08093CB
:10BDF000E03084EA6EC085ED8093BC008091BC0089
:10BE000084FDFCCF72C083E08093DD3010926F32EE
:10BE100059C080916F32823808F056C080916F32DD
:10BE20009091BB00E82FF0E0E351FE4C90838F5FD0
:10BE300080936F3247C080916F32823830F4E09146
:10BE40006F32F0E0E351FE4C108285ED8093BC0030
:10BE50008091BC0084FDFCCF1092DD3060916F3288
:10BE6000E091E330F091E4308DEE91E370E00995DC
:10BE700010926F322DC084E08093DD301092EB3150
:10BE80001092EC31E091E130F091E230099580912F
:10BE9000EC31882329F481E08093EC3110926931F0
:10BEA0009091EB31E92FF0E0E759FE4C80818093CF
:10BEB000BB009F5F9093EB319091EB318091EC311F
:10BEC000981710F485EC01C085E88093BC000FC082
:10BED00085EC8093BC0009C01092703285ED809390
:10BEE000BC008091BC0084FDFCCF1092DD30FF913E
:10BEF000EF91BF91AF919F918F917F916F915F91E2
:10BF00004F913F912F910F900BBE0F900FBE0F904E
:10BF10001F9018951092DD3081E08093DF301092F1
:10BF2000E03081E161E00E94426180E161E00E94D5
:10BF30004261E9EBF0E080818E7F808380818D7F9C
:10BF4000808388E48093B80085E48093BC000895E2
:10BF5000F999FECF72BD61BDF89A80B50895F9993F
:10BF6000FECF1FBA72BD61BD40BD0FB6F894FA9AFC
:10BF7000F99A0FBE08951F920F920FB60F921124D7
:10BF80002F933F938F939F93AF93BF93809176327C
:10BF900090917732A0917832B091793230917A32A3
:10BFA0000196A11DB11D232F2D5F2D3720F02D5798
:10BFB0000196A11DB11D20937A3280937632909321
:10BFC0007732A0937832B093793280917232909127
:10BFD0007332A0917432B09175320196A11DB11DDA
:10BFE0008093723290937332A0937432B09375320F
:10BFF000BF91AF919F918F913F912F910F900FBE65
:10C000000F901F9018958FB7F89420917632309149
:10C01000773240917832509179328FBFB901CA019D
:10C0200008959B01AC017FB7F89480917232909192
:10C030007332A0917432B091753266B5A89B05C079
:10C040006F3F19F00196A11DB11D7FBFBA2FA92F17
:10C05000982F8827860F911DA11DB11D62E0880FC2
:10C06000991FAA1FBB1F6A95D1F7BC012DC0FFB74E
:10C07000F8948091723290917332A0917432B091A1
:10C080007532E6B5A89B05C0EF3F19F00196A11DDA
:10C09000B11DFFBFBA2FA92F982F88278E0F911D92
:10C0A000A11DB11DE2E0880F991FAA1FBB1FEA95D1
:10C0B000D1F7861B970B885E9340C8F22150304021
:10C0C0004040504068517C4F2115310541055105D4
:10C0D00071F60895019739F0880F991F880F991FFD
:10C0E00002970197F1F70895789484B5826084BD32
:10C0F00084B5816084BD85B5826085BD85B581606C
:10C1000085BDEEE6F0E0808181608083E1E8F0E0CB
:10C110001082808182608083808181608083E0E8FA
:10C12000F0E0808181608083E1EBF0E080818460D9
:10C130008083E0EBF0E0808181608083E1E9F0E0E2
:10C14000808182608083808181608083E0E9F0E08B
:10C15000808181608083EAE7F0E080818460808371
:10C16000808182608083808181608083808180681B
:10C1700080831092C1000895982F883108F098515B
:10C1800097708091B4028295880F880F807C892BEC
:10C1900080937C0080917A00806480937A00809103
:10C1A0007A0086FDFCCF2091780040917900942F91
:10C1B00080E030E0282B392BC9010895482F50E04A
:10C1C000CA0187519B4FFC01249147535B4FFA01F1
:10C1D00084918823C1F0E82FF0E0EE0FFF1FE555B2
:10C1E000FB4FA591B491662341F49FB7F8948C91CD
:10C1F000209582238C939FBF08959FB7F8948C91CC
:10C20000822B8C939FBF08958430C9F0853038F419
:10C210008230F1F0833078F4813099F516C08730A0
:10C22000F9F0883018F4863061F516C08830F1F0E6
:10C23000893039F521C0809180008F7703C08091CB
:10C2400080008F7D80938000089584B58F7702C031
:10C2500084B58F7D84BD08958091B0008F7703C031
:10C260008091B0008F7D8093B00008958091900000
:10C270008F77809390000895809190008F7D8093B8
:10C2800090000895FF920F931F93F62E482F50E0D1
:10C29000CA01875F9A4FFC012491CA0187519B4FC5
:10C2A000FC01149147535B4FFA0104910023C9F03C
:10C2B000222319F0822F0E940461E02FF0E0EE0F9C
:10C2C000FF1FEB54FB4FA591B4919FB7F894FF204B
:10C2D00021F48C911095812302C08C91812B8C9339
:10C2E0009FBF1F910F91FF90089508951F920F9285
:10C2F0000FB60F920BB60F9211242F933F934F93CB
:10C300008F939F93EF93FF934091C6002091BB3290
:10C310003091BC322F5F3F4F2F7330708091BD3210
:10C320009091BE322817390759F0E091BB32F09155
:10C33000BC32E558FD4C40833093BC322093BB3275
:10C34000FF91EF919F918F914F913F912F910F907E
:10C350000BBE0F900FBE0F901F90189508951F925F
:10C360000F920FB60F920BB60F9211242F933F939B
:10C370004F938F939F93EF93FF934091CE00209123
:10C380004333309144332F5F3F4F2F733070809190
:10C390004533909146332817390759F0E0914333DC
:10C3A000F0914433ED5FFC4C408330934433209351
:10C3B0004333FF91EF919F918F914F913F912F9137
:10C3C0000F900BBE0F900FBE0F901F901895E0912D
:10C3D0009733F0919833E05CFF4F819191912081E8
:10C3E0003181821B930B8F739070892B11F00E9407
:10C3F0007561E091B633F091B733E05CFF4F819106
:10C40000919120813181821B930B8F739070892BC6
:10C4100011F00E94AE6108951F920F920FB60F9215
:10C420000BB60F9211242F933F934F935F936F930B
:10C430007F938F939F93AF93BF93EF93FF9320913D
:10C44000FF323091003380910133909102332817ED
:10C45000390731F48091C1008F7D8093C10016C0EF
:10C46000E0910133F0910233E154FD4C4081809121
:10C47000013390910233019660E470E00E94676B93
:10C4800090930233809301334093C600FF91EF9164
:10C49000BF91AF919F918F917F916F915F914F91DC
:10C4A0003F912F910F900BBE0F900FBE0F901F90DA
:10C4B00018951F920F920FB60F920BB60F92112480
:10C4C0002F933F934F935F936F937F938F939F939C
:10C4D000AF93BF93EF93FF932091873330918833CD
:10C4E0008091893390918A332817390731F48091EC
:10C4F000C9008F7D8093C90016C0E0918933F09107
:10C500008A33E95BFC4C40818091893390918A3376
:10C51000019660E470E00E94676B90938A33809389
:10C5200089334093CE00FF91EF91BF91AF919F91DE
:10C530008F917F916F915F914F913F912F910F90CC
:10C540000BBE0F900FBE0F901F901895AF92BF9229
:10C55000DF92EF92FF920F931F93CF93DF93EC0143
:10C560007A018B01DD24403081EE580780E06807B6
:10C5700080E0780711F0DD24D39491E0A92EB12C4E
:10C58000EC89FD89DD2069F0C5010E8C02C0880FA1
:10C59000991F0A94E2F7808360E079E08DE390E0F0
:10C5A00005C0108260E874E88EE190E0A801970170
:10C5B0000E947A6B2150304040405040569547953C
:10C5C0003795279580E12030380720F0DD2011F0E5
:10C5D000DD24D6CFE889F9893083EA89FB89208375
:10C5E000EE89FF89408121E030E0C9010A8C02C058
:10C5F000880F991F0A94E2F7482B4083EE89FF8940
:10C600004081C9010B8C02C0880F991F0A94E2F780
:10C61000482B4083EE89FF894081C9010C8C02C000
:10C62000880F991F0A94E2F7482B4083EE89FF890F
:10C6300080810D8C02C0220F331F0A94E2F72095EF
:10C6400028232083DF91CF911F910F91FF90EF90CE
:10C65000DF90BF90AF900895DC011C96ED91FC91A6
:10C660001D97E05CFF4F2191319180819181281BC2
:10C67000390B2F733070C9010895DC011C96ED91C0
:10C68000FC911D97E05CFF4F20813181E054F04028
:10C69000DF01AE5BBF4F8D919C9111972817390731
:10C6A00019F42FEF3FEF07C08D919C91E80FF91F10
:10C6B0008081282F30E0C9010895DC011C96ED919E
:10C6C000FC911D97E05CFF4F20813181E054F040E8
:10C6D000DF01AE5BBF4F8D919C91119728173907F1
:10C6E00019F42FEF3FEF10C08D919C911197E80F37
:10C6F000F91F20818D919C91119701968F739070F5
:10C7000011969C938E9330E0C9010895FC018685B3
:10C710009785DC01A05CBF4FFC01EE5BFF4F2D91C4
:10C720003C9111978081918128173907C1F70895AD
:10C73000CF93DF93EC01462FEE85FF85E05CFF4F42
:10C7400080819181E054F040019660E470E00E94A5
:10C75000676B9C01DF01AE5BBF4F8D919C91119780
:10C7600028173907D1F3E05CFF4F80819181E054B5
:10C77000F040E80FF91F4083EE85FF85E05CFF4F36
:10C7800031832083EE89FF89208181E090E00D8C48
:10C7900002C0880F991F0A94E2F7282B208381E0BA
:10C7A00090E0DF91CF9108951F9310928E331092F5
:10C7B0008D3328EE33E040E050E020938F33309308
:10C7C000903340939133509392336BEE76E07093B5
:10C7D0008C3360938B338BE792E390939833809301
:10C7E00097338FEB92E390939A338093993385EC50
:10C7F00090E090939C3380939B3384EC90E09093F3
:10C800009E3380939D3380EC90E09093A03380938F
:10C810009F3381EC90E09093A2338093A13386EC18
:10C8200090E09093A4338093A33314E01093A53346
:10C83000B3E0B093A633A7E0A093A733F5E0F0935D
:10C84000A833E1E0E093A9331092AD331092AC33FA
:10C850002093AE333093AF334093B0335093B13322
:10C860007093AB336093AA3383E093E39093B73331
:10C870008093B63387E493E39093B9338093B833CE
:10C880008DEC90E09093BB338093BA338CEC90E0C6
:10C890009093BD338093BC3388EC90E09093BF338A
:10C8A0008093BE3389EC90E09093C1338093C03382
:10C8B0008EEC90E09093C3338093C2331093C433D3
:10C8C000B093C533A093C633F093C733E093C83316
:10C8D0001F910895CF93DF930E9474600E94765851
:10C8E000C7EED1E60E94304F2097E1F30E94E76146
:10C8F000F9CFCF92DF92EF92FF920F931F93CF93D6
:10C90000DF937C016B018A01C0E0D0E00FC0D6014B
:10C910006D916D01D701ED91FC910190F081E02DB9
:10C92000C7010995C80FD91F015010400115110505
:10C9300071F7CE01DF91CF911F910F91FF90EF9092
:10C94000DF90CF900895EF92FF920F931F93CF93B4
:10C95000DF937C018B01C0E0D0E0F8010F5F1F4F37
:10C960006491662359F0D701ED91FC910190F0811B
:10C97000E02DC7010995C80FD91FEFCFCE01DF9178
:10C98000CF911F910F91FF90EF900895DC01ED91F1
:10C99000FC910190F081E02D09950895CF93DF93EC
:10C9A000DB010D900020E9F71197A61BB70BEC01F6
:10C9B000E881F9810280F381E02DAD010995DF91D5
:10C9C000CF9108954F925F927F928F929F92AF92F4
:10C9D000BF92CF92DF92EF92FF920F931F93DF935C
:10C9E000CF93CDB7DEB7A1970FB6F894DEBF0FBED9
:10C9F000CDBF2C01742ECB01223008F42AE019A2FD
:10CA000031E2C32ED12CCC0EDD1E822E9924AA2415
:10CA1000BB24672D752FA50194010E947A6B7901C3
:10CA20008A01C801B701A50194010E94286B472D16
:10CA3000461B0894C108D1084A3014F4405D01C077
:10CA4000495CF6014083E114F1040105110521F070
:10CA50007E2C5F2DC801DDCFC201B6010E94CE64DD
:10CA6000A1960FB6F894DEBF0FBECDBFCF91DF9178
:10CA70001F910F91FF90EF90DF90CF90BF90AF90FC
:10CA80009F908F907F905F904F900895DC012115CB
:10CA9000310541F4ED91FC910190F081E02D642F7E
:10CAA000099508950E94E2640895EF92FF920F9312
:10CAB0001F939A017B0100E010E0B801A7010E94DA
:10CAC00046651F910F91FF90EF900895EF92FF92AE
:10CAD0000F931F939A01E62EFF2400E010E0B801A7
:10CAE000A7010E9446651F910F91FF90EF90089556
:10CAF000CF92DF92EF92FF920F931F93CF93DF932A
:10CB0000EC016A017B012115310541F4E881F981CD
:10CB10000190F081E02D642F09951FC02A30310566
:10CB2000D1F477FF17C0E881F9810190F081E02D01
:10CB30006DE209958C0144275527BA014C195D090E
:10CB40006E097F09CE012AE00E94E2649801280F55
:10CB5000391F04C02AE00E94E2649C01C901DF91F0
:10CB6000CF911F910F91FF90EF90DF90CF9008959C
:10CB7000EF92FF920F931F937B019A010027F7FC1E
:10CB80000095102FB801A7010E9478651F910F91A1
:10CB9000FF90EF9008950E94CE640895AF92BF92E7
:10CBA000CF92DF92EF92FF920F931F93CF93DF9379
:10CBB0005C016B01EE24FF24C0E0D0E010C0D50181
:10CBC000ED91FC9100811181C601BE010E94926627
:10CBD000682FC501F8010995E80EF91E2196F601A6
:10CBE00084819581C817D90750F3C701DF91CF9190
:10CBF0001F910F91FF90EF90DF90CF90BF90AF907B
:10CC000008952F923F924F925F926F927F928F92F0
:10CC10009F92AF92BF92CF92DF92EF92FF920F93CB
:10CC20001F93DF93CF93CDB7DEB73B014C011901C2
:10CC30002A016D897E898F89988D6A197B098C09F3
:10CC40009D09621A730A840A950AA40193010E943D
:10CC5000286BE218F30804091509A80197010E943E
:10CC60009C6B2A0D3B1D4C1D5D1DB901CA01CF9166
:10CC7000DF911F910F91FF90EF90DF90CF90BF90C9
:10CC8000AF909F908F907F906F905F904F903F906C
:10CC90002F900895EF92FF920F931F937B018C01C9
:10CCA000611571058105910529F420E030E040E02F
:10CCB00050E00BC00E941B04A80197010E949C6BCE
:10CCC000AC01CB01DA019C01AD01B901CA011F9190
:10CCD0000F91FF90EF900895EF92FF920F931F93A3
:10CCE0007B018C01621773078407950764F4261B88
:10CCF000370B480B590BCA01B9010E944A66E60E70
:10CD0000F71E081F191FB701C8011F910F91FF904F
:10CD1000EF900895009729F0BC0180E090E00E9418
:10CD200020040895FC01848195816817790748F4EF
:10CD30000190F081E02D309721F0E60FF71F808100
:10CD4000089580E00895DC01FB0114968D919C917B
:10CD50001597892B31F461157105A9F090E0808158
:10CD600008C00D90BC91A02D6115710529F490E0CB
:10CD70008C91882349F407C0CD010E940E059C01C7
:10CD800090E0232B09F491E0892F0895CF93DF934E
:10CD90009C01FB01EC01A881B981109729F0608109
:10CDA000718161157105D1F4C081D181209759F04D
:10CDB00084819581892B39F0888190E0222733275F
:10CDC000281B390B12C0109771F0F90184819581ED
:10CDD000892B49F08C91282F30E007C0CD010E94AB
:10CDE0000E059C0102C020E030E0C901DF91CF9127
:10CDF0000895FC01DB012481358114968D919C916D
:10CE000015972817390711F020E007C0CF010E94BD
:10CE1000C66620E0892B09F421E0822F08950F9344
:10CE20001F93CF93DF93EC018B016F5F7F4F88815E
:10CE300099810E942904009711F480E005C099832C
:10CE400088831B830A8381E0DF91CF911F910F912B
:10CE50000895CF93DF93EC0188819981892B29F084
:10CE60008A819B818617970760F4CE010E940F6725
:10CE7000882341F08C819D81892B19F4E881F98107
:10CE8000108281E0DF91CF910895EF92FF920F938E
:10CE90001F93CF93DF93EC017B016C817D81E114C3
:10CEA000F104C1F04115510599F08A01060F171FD1
:10CEB000B8010E942967882369F0888199812C81B3
:10CEC0003D81820F931FB7010E9417051D830C83BC
:10CED00081E001C080E0DF91CF911F910F91FF9021
:10CEE000EF900895DF93CF9300D0CDB7DEB769837D
:10CEF0001A82BE016F5F7F4F41E050E00E9445679C
:10CF00000F900F90CF91DF910895CF93DF93EC01B5
:10CF100088819981009711F00E947003198218820C
:10CF20001D821C821B821A82DF91CF9108950F937C
:10CF30001F93182F092F0E947267882321F4812FD5
:10CF4000902F0E948567812F902F1F910F91089538
:10CF50000F931F93182F092FFB016081718144816A
:10CF600055810E944567882321F4812F902F0E94CC
:10CF70008567812F902F1F910F910895EF92FF9257
:10CF80000F931F93CF93DF93EC017B018A01BA01CA
:10CF90000E942967882321F4CE010E94856707C07B
:10CFA0001D830C8388819981B7010E941705CE01EA
:10CFB000DF91CF911F910F91FF90EF900895CF9344
:10CFC000DF93EC01198218821B821A821D821C8257
:10CFD0001E826115710551F0DB010D900020E9F70B
:10CFE0001197A61BB70BAD010E94BE67DF91CF91D1
:10CFF0000895CF93DF93EC01198218821B821A8265
:10D000001D821C821E826115710551F0DB010D909D
:10D010000020E9F71197A61BB70BAD010E94BE6770
:10D02000DF91CF9108950F931F93182F092F61154A
:10D03000710559F0DB010D900020E9F71197A61B4F
:10D04000B70BAD010E94BE6702C00E948567812FA9
:10D05000902F1F910F910895EF92FF920F931F93BE
:10D06000DF93CF93CDB7DEB761970FB6F894DEBFED
:10D070000FBECDBF8C01CB01F8011182108213824B
:10D0800012821582148216827E010894E11CF11C22
:10D09000B70150E00E943F05C801B7010E94136824
:10D0A00061960FB6F894DEBF0FBECDBFCF91DF9172
:10D0B0001F910F91FF90EF900895EF92FF920F93C1
:10D0C0001F93DF93CF93CDB7DEB762970FB6F89477
:10D0D000DEBF0FBECDBF8C01CB01F80111821082E3
:10D0E000138212821582148216827E010894E11C3A
:10D0F000F11CB70150E00E941E05C801B7010E9453
:10D10000136862960FB6F894DEBF0FBECDBFCF9105
:10D11000DF911F910F91FF90EF900895EF92FF9292
:10D120000F931F93DF93CF93CDB7DEB729970FB639
:10D13000F894DEBF0FBECDBF8C01862FF80111829F
:10D1400010821382128215821482168290E07E0170
:10D150000894E11CF11CB70150E00E943F05C80192
:10D16000B7010E94136829960FB6F894DEBF0FBE70
:10D17000CDBFCF91DF911F910F91FF90EF90089558
:10D18000DF93CF9300D0CDB7DEB7FC0111821082C0
:10D190001382128215821482168269831A82BE015A
:10D1A0006F5F7F4F0E9413680F900F90CF91DF91B8
:10D1B0000895CF93DF93EC01FB018617970761F089
:10D1C000608171816115710529F0448155810E944A
:10D1D000BE6702C00E948567CE01DF91CF9108959E
:10D1E000FC0111821082138212821582148216822F
:10D1F0000E94D9680895FC01118210821382128264
:10D200001582148216820E94D9680895FC018081DB
:10D2100091810E9470030895FC01808191810E9498
:10D22000700308955058BB27AA270ED070C161D152
:10D2300030F066D120F031F49F3F11F41EF456C156
:10D240000EF4E095E7FB4CC1E92F72D180F3BA17D9
:10D25000620773078407950718F071F49EF58AC179
:10D260000EF4E0950B2EBA2FA02D0B01B901900101
:10D270000C01CA01A0011124FF27591B99F0593F45
:10D2800050F4503E68F11A16F040A22F232F342F8D
:10D290004427585FF3CF469537952795A795F040DB
:10D2A0005395C9F77EF41F16BA0B620B730B840BF0
:10D2B000BAF09150A1F0FF0FBB1F661F771F881FA8
:10D2C000C2F70EC0BA0F621F731F841F48F4879500
:10D2D00077956795B795F7959E3F08F0B3CF9395EF
:10D2E000880F08F09927EE0F979587950895D4D069
:10D2F00008F481E008950CD00AC102D140F0F9D0C1
:10D3000030F021F45F3F19F0EBC0511134C1EEC091
:10D310000FD198F39923C9F35523B1F3951B550BFE
:10D32000BB27AA2762177307840738F09F5F5F4FF8
:10D33000220F331F441FAA1FA9F333D00E2E3AF039
:10D34000E0E830D091505040E695001CCAF729D053
:10D35000FE2F27D0660F771F881FBB1F26173707A2
:10D360004807AB07B0E809F0BB0B802DBF01FF27D2
:10D3700093585F4F2AF09E3F510568F0B1C0FBC043
:10D380005F3FECF3983EDCF3869577956795B7950C
:10D39000F7959F5FC9F7880F911D9695879597F927
:10D3A0000895E1E0660F771F881FBB1F62177307A0
:10D3B0008407BA0720F0621B730B840BBA0BEE1FB5
:10D3C00088F7E0950895BCD088F09F5790F0B92F6A
:10D3D0009927B751A0F0D1F0660F771F881F991FCA
:10D3E0001AF0BA95C9F712C0B13081F0C3D0B1E0DC
:10D3F0000895C0C0672F782F8827B85F39F0B93FEC
:10D40000CCF3869577956795B395D9F73EF49095CB
:10D410008095709561957F4F8F4F9F4F0895E89449
:10D4200009C097FB3EF490958095709561957F4F6C
:10D430008F4F9F4F9923A9F0F92F96E9BB2793951A
:10D44000F695879577956795B795F111F8CFFAF42A
:10D45000BB0F11F460FF1BC06F5F7F4F8F4F9F4F5B
:10D4600016C0882311F096E911C0772321F09EE8B9
:10D47000872F762F05C0662371F096E8862F70E01F
:10D4800060E02AF09A95660F771F881FDAF7880FF9
:10D490009695879597F90895990F0008550FAA0B4F
:10D4A000E0E8FEEF16161706E807F907C0F01216B7
:10D4B0001306E407F50798F0621B730B840B950BBA
:10D4C00039F40A2661F0232B242B252B21F408950F
:10D4D0000A2609F4A140A6958FEF811D811D0895AC
:10D4E00097F99F6780E870E060E008959FEF80EC17
:10D4F000089500240A9416161706180609060895BA
:10D5000000240A9412161306140605060895092E1F
:10D510000394000C11F4882352F0BB0F40F4BF2B8E
:10D5200011F460FF04C06F5F7F4F8F4F9F4F0895CE
:10D5300057FD9058440F551F59F05F3F71F04795C4
:10D54000880F97FB991F61F09F3F79F087950895A9
:10D55000121613061406551FF2CF4695F1DF08C0C8
:10D56000161617061806991FF1CF869571056105E5
:10D5700008940895E894BB2766277727CB0197F98D
:10D5800008958ADF08F48FEF08950BD0C0CFB1DF84
:10D5900028F0B6DF18F0952309F0A2CFA7CF112409
:10D5A000EACFC6DFA0F3959FD1F3950F50E0551F4A
:10D5B000629FF001729FBB27F00DB11D639FAA27E8
:10D5C000F00DB11DAA1F649F6627B00DA11D661F37
:10D5D000829F2227B00DA11D621F739FB00DA11D58
:10D5E000621F839FA00D611D221F749F3327A00D12
:10D5F000611D231F849F600D211D822F762F6A2FAE
:10D6000011249F5750408AF0E1F088234AF0EE0F32
:10D61000FF1FBB1F661F771F881F91505040A9F73F
:10D620009E3F510570F05CCFA6CF5F3FECF3983E74
:10D63000DCF3869577956795B795F795E7959F5FA6
:10D64000C1F7FE2B880F911D9695879597F9089540
:10D65000629FD001739FF001829FE00DF11D649FD6
:10D66000E00DF11D929FF00D839FF00D749FF00D62
:10D67000659FF00D9927729FB00DE11DF91F639F03
:10D68000B00DE11DF91FBD01CF0111240895991BB3
:10D6900079E004C0991F961708F0961B881F7A95A9
:10D6A000C9F780950895AA1BBB1B51E107C0AA1FAB
:10D6B000BB1FA617B70710F0A61BB70B881F991F33
:10D6C0005A95A9F780959095BC01CD01089597FBD7
:10D6D000092E07260AD077FD04D0E5DF06D000200A
:10D6E0001AF4709561957F4F0895F6F7909581959E
:10D6F0009F4F0895A1E21A2EAA1BBB1BFD010DC06E
:10D70000AA1FBB1FEE1FFF1FA217B307E407F507F1
:10D7100020F0A21BB30BE40BF50B661F771F881FCD
:10D72000991F1A9469F760957095809590959B0163
:10D73000AC01BD01CF01089597FB092E05260ED03F
:10D7400057FD04D0D7DF0AD0001C38F4509540951F
:10D75000309521953F4F4F4F5F4F0895F6F79095C5
:10D760008095709561957F4F8F4F9F4F0895EE0F75
:10D77000FF1F0590F491E02D09942F923F924F9254
:10D780005F926F927F928F929F92AF92BF92CF9251
:10D79000DF92EF92FF920F931F93CF93DF93CDB75A
:10D7A000DEB7CA1BDB0B0FB6F894DEBF0FBECDBFD2
:10D7B00009942A88398848885F846E847D848C84A3
:10D7C0009B84AA84B984C884DF80EE80FD800C81AC
:10D7D0001B81AA81B981CE0FD11D0FB6F894DEBF8F
:10D7E0000FBECDBFED01089515E0C0E3D5E004C044
:10D7F000FE010E94B96B2296C233D107C9F7F89493
:02D80000FFCF58
:10D80200002D0078004356004F666600323A33001E
:10D81200333A3400373A3800313A002B002F0020D7
:10D8220000CD3300000100000001010000000000F3
:10D832000000000000000000000000200028003767
:10D8420000460055006400730082009100FFFF0053
:10D85200030406080C101820304060010400000088
:10D86200000000FFFF0000FEFF0000FDFF0000FCC3
:10D87200FF0000FBFF0000FAFF00002B00550080B4
:10D8820000AB00D50000012B0155018001AB01D591
:10D89200010002040507090B000205070901020342
:10D8A2000405060708090A0B0C0101030305060615
:10D8B20008080A0A0C0101030304060608080909FC
:10D8C2000B0101030303050508080A0A0A01010303
:10D8D2000304060608080A0A0B01010202040606EE
:10D8E200080809090B0101030305070708080A0ACA
:10D8F2000C0101030305060608080A0A0B010102CE
:10D9020002040606070709090B03030000003F0093
:10D9120000803F713DAA3F00000040713D2A400057
:10D92200008040E0C0A080604020000101000408A7
:10D932000C20030000011018203040608018100CE9
:10D942000806040310101112040810000000171436
:10D95200171517000000101810100C0000000E0A16
:10D962000E0A0E0000001B091B0A1B000101010127
:10D97200010F1F0E00000A0A0E02020000000E0232
:10D982000E080E0000030408121313111F000000FA
:10D9920000000000001804020919191110080601FC
:10D9A200000000000004001F0000000001020C1033
:10D9B2000000000001808386898C8F9295989C9F3D
:10D9C200A2A5A8ABAEB0B3B6B9BCBFC1C4C7C9CCDF
:10D9D200CED1D3D5D8DADCDEE0E2E4E6E8EAECED5B
:10D9E200EFF0F2F3F5F6F7F8F9FAFBFCFCFDFEFEB8
:10D9F200FFFFFFFFFFFFFFFFFFFFFFFEFEFDFCFC3F
:10DA0200FBFAF9F8F7F6F5F3F2F0EFEDECEAE8E6F7
:10DA1200E4E2E0DEDCDAD8D5D3D1CECCC9C7C4C1CA
:10DA2200BFBCB9B6B3B0AEABA8A5A29F9C98959265
:10DA32008F8C898683807C797673706D6A67636068
:10DA42005D5A5754514F4C494643403E3B3836335A
:10DA5200312E2C2A272523211F1D1B1917151312BE
:10DA6200100F0D0C0A090807060504030302010141
:10DA7200000000000000000000000001010203039A
:10DA82000405060708090A0C0D0F101213151719C1
:10DA92001B1D1F212325272A2C2E313336383B3ECE
:10DAA200404346494C4F5154575A5D6063676A6D13
:10DAB200707376797C828486888A8C8E9092949612
:10DAC200989A9C9EA0A2A4A6A8AAACAEB0B2B4B6E4
:10DAD200B8BABCBEC0C2C4C6C8CACCCED0D2D4D6D4
:10DAE200D8DADCDEE0E2E4E6E8EAECEEF0F2F4F6C4
:10DAF200F8FAFCFEFEFCFAF8F6F4F2F0EEECEAE8D4
:10DB0200E6E4E2E0DEDCDAD8D6D4D2D0CECCCAC8A3
:10DB1200C6C4C2C0BEBCBAB8B6B4B2B0AEACAAA893
:10DB2200A6A4A2A09E9C9A98969492908E8C8A8883
:10DB3200868482807E7C7A78767472706E6C6A6873
:10DB4200666462605E5C5A58565452504E4C4A4863
:10DB5200464442403E3C3A38363432302E2C2A2853
:10DB6200262422201E1C1A18161412100E0C0A0843
:10DB7200060402010000020406080A0C0E10121428
:10DB820016181A1C1E20222426282A2C2E30323443
:10DB920036383A3C3E40424446484A4C4E50525433
:10DBA20056585A5C5E60626466686A6C6E70727423
:10DBB20076787A7C7E800102030405060708090A4A
:10DBC2000B0C0D0E0F101112131415161718191A2B
:10DBD2001B1C1D1E1F202122232425262728292A1B
:10DBE2002B2C2D2E2F303132333435363738393A0B
:10DBF2003B3C3D3E3F404142434445464748494AFB
:10DC02004B4C4D4E4F505152535455565758595AEA
:10DC12005B5C5D5E5F606162636465666768696ADA
:10DC22006B6C6D6E6F707172737475767778797ACA
:10DC32007B7C7D7E7F808182838485868788898ABA
:10DC42008B8C8D8E8F909192939495969798999AAA
:10DC52009B9C9D9E9FA0A1A2A3A4A5A6A7A8A9AA9A
:10DC6200ABACADAEAFB0B1B2B3B4B5B6B7B8B9BA8A
:10DC7200BBBCBDBEBFC0C1C2C3C4C5C6C7C8C9CA7A
:10DC8200CBCCCDCECFD0D1D2D3D4D5D6D7D8D9DA6A
:10DC9200DBDCDDDEDFE0E1E2E3E4E5E6E7E8E9EA5A
:10DCA200EBECEDEEEFF0F1F2F3F4F5F6F7F8F9FA4A
:10DCB200FBFCFDFEFF00FFFFFFFFFFFFFFFFFFFF7B
:10DCC200FFFFFFFFFFFFFFFFFFFFFFFFFFFFFFFF62
:10DCD200FFFFFFFFFFFFFFFFFFFFFFFFFFFFFFFF52
:10DCE200FFFFFFFFFFFFFFFFFFFFFFFFFFFFFFFF42
:10DCF200FFFFFFFFFFFFFFFFFFFFFFFFFFFFFFFF32
:10DD0200FFFFFFFFFFFFFFFFFFFFFFFFFFFFFFFF21
:10DD1200FFFFFFFFFFFFFFFFFFFFFFFFFFFFFFFF11
:10DD2200FFFFFFFFFFFFFFFFFFFFFFFFFFFFFFFF01
:10DD3200FFFFFFFFFFFF00000000000000000000E7
:10DD420000000000000000000000000000000000D1
:10DD520000000000000000000000000000000000C1
:10DD620000000000000000000000000000000000B1
:10DD720000000000000000000000000000000000A1
:10DD82000000000000000000000000000000000091
:10DD92000000000000000000000000000000000081
:10DDA2000000000000000000000000000000000071
:10DDB200000000000000000C0D0E0F08090A0B0401
:10DDC2000506070001020300000000F35A7964000F
:10DDD2000040001400540000000000D55CA45C5D0B
:10DDE2005C665C7B5C8C5C00000000986379642C50
:08DDF200635D633D638663007D
:00000001FF
